:020000024000BC
:100000006FC0620B000000000018011800280128D2
:100010000228032800290129022903290429052986
:10002000062907290829002A012A022A032A042A64
:10003000052AA62AE8C806000A1F0400F0020020CC
:1000400076030020C00200208E0200201C02002047
:10005000122104005A210400002304008C2504000E
:100060007A260400681D0400261C0400E81C040015
:10007000781C04006A2C04000C050020E820040011
:10008000362904003A680600326A0600AA6A0600A9
:10009000F2190600261A0600DC680500865C0500D9
:1000A000F06106006C2904009C2406002AE3040089
:1000B000B8E3040010E40400FA34040046350400F8
:1000C000B0330400229F0400DC990400C0A804009F
:1000D00090AC04003CB00400F88B0400968B040044
:1000E000808F0400448C04006C8B0400F08B0400AF
:1000F0001E8B0400C88C0400208D0400D08C0400EA
:10010000D48C04006E8D0400288D04005A8D0400E8
:100110007C92040084920400C48C0400CC8C040003
:100120006C8D0400809204001C8E0400F293040085
:1001300084BE040002BF040040BF040086A1040086
:100140009EA10400DAA10400508504006E8604001C
:10015000E4860400F85304009E4E04005A7A04001A
:100160001C4F04008675040092A50600BA9D060087
:10017000C4A20600ECBA0600B2B9060036BE0600FC
:10018000EEBD06002EBE0600DEBE06002E8C06006A
:100190006EBE0600F4B006001AB1060042B10600B9
:1001A0004EBF0600AEB7060044B70600BEBF06004D
:1001B000CA8E0600668F06008E8F0600308F0600FE
:1001C000F6450600EA2F06007033060048310600A7
:1001D0009E3B0600986206008E610600628C060057
:1001E000F82D0400621B06007C240600742506001E
:1001F00050580600E2580600965A06008AA50400E8
:10020000CE440600463C0600B02D06002A3F0600FC
:100210009A2F06001C0700203A1C06005ABE060052
:10022000F2BD06002ABE060026BE06001825040000
:10023000D8A2040062BE0600CC4606009A4706001B
:10024000144806002AA306005EBE060066BE06002D
:10025000125C05006ABE06000A120020D0110020C0
:100260000AA30600B0A406009C450600000000009A
:10027000000000000000000000000000000000007E
:100280006373B60082801C419105110523AEF5FE13
:10029000C5BFB7270020372700209387079913078A
:1002A00087F56373F700828023A007009107D5BF0D
:1002B0004111B7E700E022C480433707200006C69B
:1002C000798C23A0E7180F10000011C199E5B7E75A
:1002D00000E023A08710014545A893073500C20719
:1002E000C183F19BC207C183130740036366F70212
:1002F00037270020032547AD372700208326C7ACCA
:100300006391A60237270020032747B669D3C207A7
:10031000DD8D0545029765BF37270020032507AD12
:10032000E1BF035765002DE7035745006362F706F9
:10033000B72600203306F74021489386C6AD637880
:10034000C8028328050003D86600138687001D8F26
:100350002A9661172312E6002320160123130600B4
:1003600010C12312F500130788FF2393E60023131F
:10037000B50083D566002105B387F5402393F600C9
:10038000B7E700E023A08710B240224441018280F9
:100390000841BDB7B7E700E003A807003707200012
:1003A00023A0E7183378E8000F10000001E523A030
:1003B00007118280B727002003AE47ADB727002082
:1003C00003A3C7AC8146F28763FC670A83A80700D2
:1003D000636BF50A63E9A80A138787006362E50A7D
:1003E00003D66700216705076319E600372600205A
:1003F000034746A205072302E6A23726002013057D
:10040000C6AD83D547000357650023930700130645
:10041000C6AD2E97420741832313E5006387C703C8
:1004200037250020032505AD6301F50203D56600DD
:1004300009ED83D7460023A016012107BE95A1052B
:100440002392B6002313E600B6879843630A670237
:10045000B726002083A606AD6304D7028356670043
:1004600085E283D64700835547001843A106AE9620
:100470002392D70098C383576600A1072313F60081
:10048000B7E700E02DB7BE86C6873DBFB7E700E0FF
:100490009843B706200023A0D718758F0F100000CF
:1004A00001C599C1814711E6B7E700E023A0E71035
:1004B0008280B386F50003C80600B306F500850701
:1004C00023800601E317F6FEC5B737E700E01C43BB
:1004D000B70620002320D718F58F0F10000019C190
:1004E00091C111E637E700E02320F71082809105E3
:1004F00003A7C5FF11057D16232EE5FEDDB737E7FF
:1005000000E01C43B70620002320D718F58F0F10FA
:10051000000001C53307C50011E637E700E02320DE
:10052000F71082800505A30FB5FEE31DE5FEF5B7C4
:10053000B7E700E09843B706200023A0D718758FCF
:100540000F1000008147B306F5008386060099E688
:10055000B7E600E023A0E6103E8582808507E5B778
:1005600037E700E01C43B70620002320D718F58F9B
:100570000F10000001C599C1014711EA37E700E0FB
:100580002320F710054582800507E309E6FE3308BE
:10059000E500B386E5000348080083C60600E305CE
:1005A000D8FE37E700E02320F7100145828037E7C7
:1005B00000E01C43B70620002320D718F58F0F104A
:1005C00000001307F6FFBA952A966317C50037E7B0
:1005D00000E02320F7108280FD1503C715000505F4
:1005E000A30FE5FEDDB737E700E01C43B7062000A8
:1005F0002320D718F58F0F10000001C53307C50061
:1006000019E637E700E02320F71001458280050551
:100610008346F5FFE397B6FEE31BE5FE37E700E010
:100620002320F71005458280797126D2B724002057
:1006300022D403A404B306D64AD04ECE52CC56CA16
:100640005AC85EC662C44DC8372A00203729002028
:10065000B7290020814BB72A002037CBC901130AE4
:100660004AB31309C9AD938909B88357240099EF98
:100670005C44639A0B0023A8F4B2032CC4002285C7
:10068000113B6284B9A823A6FB00C5BF83A78AB229
:1006900082971C443307F5406376F50003A74900B1
:1006A0001D8F2A979306FB3763ECE6062328090083
:1006B0008355240003450400972004E0E780A0CC84
:1006C0005C405844B1C70C4403A64900AE97BE86AF
:1006D00063E4B70063E4C700B386C74014C4A28BC9
:1006E0003A8441F4B72700209387C7AD984B8946D9
:1006F00063FCE604791798CBB25022549254025905
:10070000F249624AD24A424BB24B224C4561828046
:1007100063950B0023A8E4B28DB723A6EB00B1BF0D
:1007200003274A0219CB63EDA7003385A74083272F
:1007300009016374F5002328A900A28B404455B732
:1007400003A74900BA97D5B723A8070075B7B727FD
:10075000002003A787B7411122C406C63E8411C3F7
:100760000297B727002083C767B293F7F70F99E383
:10077000232C04B6B24022444101828001114EC6AE
:10078000B729002083A789B006CE22CC26CA4AC842
:1007900052C456C281C7829723A409B0B72400204F
:1007A000938784E583C7570037240020938484E52A
:1007B000858B130484B081CF83C7740019476316F7
:1007C000F70EA3820400EF00706F5C4482971C4414
:1007D00091C3829737240020372900209307C4ADA6
:1007E0000327C9B203C61700130AC4AD8347C4ADBB
:1007F00093961700BA9683D60600F9C28347C4AD14
:1008000063E8C70C83A789B0230E04AC6394071276
:10081000B727002083A787B2638E0710B727002071
:1008200083A747B82328FA00013583C7B400639330
:10083000071083C7940081CF83C7740093F7F70F25
:1008400099E7A3840400972006E0E780A09AB727E1
:10085000002083A787B5F9CF83270A01E1CF83C79B
:10086000740015476368F70CB7270020938747EAA1
:1008700083C7C700918BDDEFB727002083C767B21E
:1008800093F7F70FC5EB83461A000326C9B263CC72
:10089000D70A6244F240D2444249B249224A924ABB
:1008A0000561172304E06700830C83C774001D47AC
:1008B000E31FF7F0A3820400EF0050601C4839B733
:1008C000850793F7F70F230EF4ACE3E1C7F23DB7CA
:1008D00086073E9783550700231007000345C4ADE4
:1008E000B727002083A747B013172500B72A002099
:1008F000BA979C4323920AB2829783D74AB203479E
:10090000C4AD93C7F7FF7D8D931717000327C9B2B6
:100910003E97835707005D8D2310A7008347C4AD22
:1009200081C78507230EF4AC0347C4AD83471A0083
:10093000E37AF7ECF2406244D2444249B249224A97
:10094000924A056182801397170032970357070078
:1009500075F385072DBF37C700408326C720B7072B
:10096000FCFFFD17F58F2326F72001000100B727B4
:1009700000209387C7ADC84F832787262326D7201B
:100980006A0593C7F7FF99835D8D8280B7270020A2
:1009900003A347B96303030002831305F00F8280AA
:1009A0000327851163000712411122C406C683473D
:1009B000C5008345E5042A8493F7C70F2306F50095
:1009C000834697000356C70013958601618563F13E
:1009D000C508635A05060345870093F6F607A30486
:1009E000D700054693E627006314C50093E6170079
:1009F0002306D4005C4389075CC3A30AB400032523
:100A000004112E864C430905513483278411034673
:100A10005401D44303D7C700B296118FD4C3239691
:100A2000E7008947A30DF400B727002003476403BC
:100A300083C767B46378F7048347C40093E707016B
:100A40002306F40081A093E717002306F40075B78E
:100A50009376F60F635D050203458700854513E62F
:100A600027006314B50013E617002306C400A30A89
:100A7000D400A30407008547A30DF4008327841145
:100A80009C43DDF3B240224401454101828093E75B
:100A900017002306F400A30AD400A30407000325CB
:100AA00004114C430905DD328327841103465401A8
:100AB000D44303D7C700B296118FD4C32396E7005F
:100AC0008D475DBF05458280B727002083A747E398
:100AD000411122C406C6858B2A84DDEB41651305CE
:100AE00025F5977005E0E780A0185DC18347A50054
:100AF0002315F50083270412B5E72320A41223222F
:100B0000A41285472311F4042320050083476401C0
:100B100054412316F5000347D4002304E50005479C
:100B2000A304E500372700200327C7E71385170232
:100B300015811C437D151375F50F9CC25C43DCC207
:100B40001C479CC65C47DCC61C4B9CCA5C4BDCCA81
:100B50001C4F9CCE5C4FDCCE19CD9386060213074A
:100B60000702C1BF8327441288C38357240423226A
:100B7000A412850741BFB7270020938787D003D7EA
:100B8000870005072394E700B24022444101828098
:100B90008347C40023090400054593C74700230683
:100BA000F400DDB78347850193F7E70FDDEB83475B
:100BB0009501C5EB034625018346C50009CA3727C1
:100BC000002083456503034777B463E7E50013F727
:100BD000060149CB014709C6C18A0357651C81C676
:100BE0008356A51C36973DCFB727002003D587B87D
:100BF0001307C71237460F00B335A702411113067A
:100C00000624814622C426C206C67D543305A702A7
:100C100097B006E0E780207BB727002083C7B7B4F2
:100C2000B384A700B727002003A707DA83270709A3
:100C300063F387003E84184375FBB727002083A722
:100C400087B2829781476364A400B307A440B2408F
:100C50002244B3B7970093C7170092443E854101E1
:100C6000828081473E858280B727002003A707E85E
:100C70003C5BFDFF010001008280011122CC4AC8CB
:100C80004EC606CE26CA52C456C25AC00347B50045
:100C900085472A842E8983290509631AF71E8357FD
:100CA0000508035BC503372A002093060AB883DAD8
:100CB0008600130A0AB863F4671B83460501639034
:100CC000E61A03278511631C07180327450A6318D2
:100CD00007188346F5001D476393E6180355A503DF
:100CE000330BFB409307204E3305650383244409EF
:100CF00037460F008146130606243305F502B72751
:100D0000002083C7A7B4B3549502B3B5AA02BE941A
:100D1000C204C180231394083385AA0297B006E069
:100D2000E780606AB307350133B5A7002E953E878B
:100D300083264A0019E163E4D7003387D740B384A0
:100D40005403B7460F009387F62393860624232087
:100D5000E900A697B3D7D702DA97636CF70E1D8F19
:100D60002320E900B729002083A789B28324090042
:100D7000829763E1A4123385A4406350050C83A7D6
:100D800089B2372B0020130B0BB882970327090079
:100D90006368E510198D8357E40303578B008E07B2
:100DA000B387E7021307003293870719B3D7E70227
:100DB00063EDA70E374A0F00930AFA23130A0A2499
:100DC0008357040485072310F4048347041499E32C
:100DD0002285512A2285976005E0E78060E07DE169
:100DE000832604098327C40803274B00B6973E8552
:100DF00063E4D70063E4E7003385E7408347F40109
:100E0000835464082328A4088507A30FF40083579C
:100E10008B00B384F402D694B3D444036363950C7B
:100E2000B304954083A789B223209900829763EE8B
:100E3000A40A3385A440E34505F8B727002083C7FB
:100E4000B7B463E2A708B727002023A487DA0145D7
:100E50009DA883264A00B387F6403E9711B7835476
:100E6000640837470F009307F723B3845403BE94F5
:100E700093070724B3D7F40263E7F900B387F94077
:100E80002320F900C5B503274A00BA99C5BF23A09E
:100E90003501C9BDB727002083A747B8BE94E1BD7F
:100EA00083274B00998F3E95FDB5A145228597601C
:100EB00005E0E78000CCA305A402B727002083A7A4
:100EC00047B681EF7D55F2406244D2444249B2496F
:100ED000224A924A024B05618280894515458297D4
:100EE000D5B7B3049740AA9435BF83274B00BE946F
:100EF00089B72DC901116C0022CC06CE2A84B53BDE
:100F000029CDFD576305F50237270020130747B3A6
:100F10005453B2479DC62547637FF700D9173EC695
:100F2000B24503459402971004E0E780C05CF240AC
:100F300062440561828037270020032747B8BA97AB
:100F4000F1BF0347770163E4E700998FC9BFB72674
:100F5000002083A646B8B697CDBF977005E0E7801E
:100F60006084F1B78280797126D206D622D44AD025
:100F70004ECE52CC56CA5AC85EC683475503034468
:100F80007513AA843E941374F40F9307400263F61A
:100F900087001304B4FD1374F40F03AA841383AA07
:100FA000C413A38B841222865285D68597B006E09F
:100FB000E780E03B058915E503CBD412014981495F
:100FC000337B6403930B50024A865285D68597B0D3
:100FD00006E0E780C039058915C56391690313747C
:100FE000F90F238B8412B250225492540259F249C1
:100FF000624AD24A424BB24B456182808509E2097E
:1010000093D989410509E31179FDE1BF832785095A
:1010100003560504797193D60701BD8EC206C182BD
:10102000358E1357764093575640898B058B5D8FCD
:1010300093573640918B5D8F93571640A18B5D8FF0
:1010400093171600C18B5D8F9317360093F7070235
:101050005D8F931756009355860093F707041E067D
:101060005D8F1376F60F518F93D7554013D63540C9
:10107000118A898BD18F13D67540D18F13D6154025
:10108000218AD18F13961500418AD18F139635008E
:1010900013760602D18F13965500137606049E052B
:1010A000D18F93F5F50FCD8FA20745465D8F33079E
:1010B000C70222D42A8426D252CC56CA032A8413C9
:1010C000832AC4135AC806D63697420741839357DA
:1010D0007740135557400989858BC98F1355374081
:1010E0001189C98F135517402189C98F131517000E
:1010F0004189C98F1315370013750502C98F131560
:10110000570093558700137505041E07C98F137781
:10111000F70FD98F13D5354013D755401189098B57
:10112000498F13D57540498F13D515402189498FB3
:10113000139515004189498F1395350013750502E4
:10114000498F13955500137505049E05498F93F536
:10115000F50F4D8F2207D98FB387C7024AD04ECEE5
:101160005EC662C4B697C207C18313D7774013D552
:1011700057400989058B498F13D537401189498F0D
:1011800013D517402189498F139517004189498F3D
:101190001395370013750502498F1395570093D5A2
:1011A0008700137505049E07498F93F7F70FD98FB2
:1011B00013D5354013D755401189098B498F13D565
:1011C0007540498F13D515402189498F1395150016
:1011D0004189498F1395350013750502498F139581
:1011E0005500137505049E05498F93F5F50F4D8F36
:1011F0002207D98FB387C702130650025285D685BE
:10120000B697BD8E93940601C18033F6C402137B5A
:10121000F60F97B006E0E780801505890DED83474E
:10122000D41201498149B3849702130C5002C18042
:101230004A865285D68597B006E0E7804013058937
:10124000937BF90F11C563863403850993F9F90F70
:101250000509E31F89FD230B6413B25022549254F5
:101260000259F249624AD24A424BB24B224C456182
:1012700082805E8BCDB70111B727002022CC03A45A
:1012800007DD26CA4AC84EC606CEAA841309250021
:10129000854915C083C7140003473400858B630458
:1012A000F700405CFDB71946930544004A85EFF00E
:1012B0002FABE31835FF2285F2406244D244424905
:1012C000B249056182804111B727002022C403A4DE
:1012D00007DD26C24AC006C693042500054901E879
:1012E0002285B24022449244024941018280A6856F
:1012F0001305A40297C005E0E7804046E30225FFFE
:10130000405CF1BF4111B727002022C403A407DDD0
:1013100026C24AC006C693042500054901E8228575
:10132000B24022449244024941018280A6851305BD
:10133000A40197C005E0E7806042E30225FF405C1E
:10134000F1BF011122CC604126CA4AC84EC652C420
:1013500006CEAA841D4A130965058549BC44636409
:10136000F400054581A803C7D40083474400631BEC
:10137000470503C784026304F7000040C5B703476D
:10138000540083C75405E31AF7FE1946CA851305AE
:101390006400EFF0EF9CE31235FF0347C40083C7FE
:1013A0009402E31CF7FC0357E40083D7A402E3167E
:1013B000F7FC0145F2406244D2444249B249224A14
:1013C00005618280E31BF7FA0347540083C7540585
:1013D000E315F7FA1946CA8513056400EFF04F9834
:1013E000E31D35F9F9B70111B727002022CC03A47A
:1013F00087DC26CA06CE2AC42EC6854419E40145D8
:10140000F2406244D24405618280834791000347E1
:101410001400858B6304F7000044CDB7194693058B
:10142000A10013052400EFF0AF93E31795FE0545E7
:10143000C1BF0000EFF0AFB173000000000000007A
:1014400097120000938262950383020023800200BA
:10145000630F0300F32510342EC097050000938519
:10146000A5FD73901534EF00A0477300203086DC93
:10147000EF000047E65082800000B726002003A757
:1014800046E501114AC81C5F4EC606CE998322CCA0
:1014900026CA858B3689B7290020ADCF9307000671
:1014A000372400201CDF930784E583C767001307F8
:1014B0000008930484E56319F70083A709E59C43BA
:1014C00093F707042383F400834784E593F7070425
:1014D00089CFB727002083A787B28297C8CC8347DC
:1014E00084E593F7F70B230CF4E483C7440093F7E8
:1014F00007048DE38547A382F400B727002083A764
:1015000007E83707020098C7130700FC2382E400AE
:101510009848F8D3032749E51C5F9183858B95C3D1
:101520001C5F93E707011CDFB727002083A707E8AC
:10153000054723A20706B7270020938787E5238264
:10154000E70083A709E5D8430583058B19C7D8436E
:10155000759BD8C3D843799BD8C3F2406244D24428
:101560004249B24905618280093F730020309317D8
:10157000D50063DF0700B727002083A707E87D5762
:10158000B8D7B72700209387C7ADD84F0507D8CF66
:101590009377850099CFB7270020938787E503C706
:1015A0002700136717002381E700130700F8238241
:1015B000E7009377150099CBB7270020938787E53D
:1015C00003C7170013671700A380E7009377650030
:1015D0008DC713774500B727002059CF03C787E58C
:1015E00013671700238CE7E4B727002003A747E51C
:1015F0005C57F19B93E717005CD79317F50063D214
:101600000702B7270020138787D083468707938771
:1016100087D0C18ABDCA8347870793E70702230C97
:10162000F7069317E50063D60702B72700209387D4
:1016300087E503C7470062076187635507000547D1
:101640002382E700B727002083A707E837070200B7
:1016500098C79317C50063D00702B7270020938768
:1016600087D003C79707058B29C303C7970713675D
:101670002700A38CE7068280938787E503C737009E
:1016800013671700A381E70085B703C7870789465B
:101690003D8B6308D70003C787078D463D8BE31258
:1016A000D7F81147238CE706ADBF03C79707118B07
:1016B00079D303C797071367870065BFB727002053
:1016C000B726002003A607E8938786E503C786E5CB
:1016D000058B11C723820700A3820700828003C7FE
:1016E0001700058B65FB785275F303C75700EDB7FC
:1016F00037270020032847E5832788039583858BB8
:10170000C1E311C683270803BD832300F60085CA01
:10171000832747E5985B46079357670163560700A1
:1017200093E707C0C207C18303970600C207C187BA
:1017300009C7BA970947B3C7E7022390F6009DCDC2
:101740008345150085CDB7270020938787E583C79C
:10175000670013879500894593F7070485C33A9579
:10176000834705000547994593F6F7066398E60019
:10177000E207E187814563D30700B9452E85828062
:101780008545EDBF411126C206C622C44AC0B72412
:10179000002035ED83A604E8AE87F8527DFF372997
:1017A0000020130989E52301090037F400E03E8594
:1017B000832704D1B285ED9B2328F4D0832704D15D
:1017C00093E787022328F4D073005010971006E0A7
:1017D000E780208AB727002083A747E5B706800067
:1017E0009843558F98C3D857719BD8D783A704E8DF
:1017F000A3020900A3000900094798C3832704D165
:1018000093E787002328F4D07300501005A08D477C
:101810006314F504B727002083A747E5B7068000C7
:101820009843558F98C3D857719BD8D783A604E89F
:10183000B7270020938787E503C72700058B19E7A3
:1018400003C73700058B51CB23820700B2402244E7
:1018500092440249410182808547E319F5FCB7F7BC
:1018600000E003A707D16D9B23A8E7D003A707D10A
:101870001367870223A8E7D07300501003A704E87A
:101880008177FD175447F58F5CC70F10000003A741
:1018900004E8B7070200130600F81CC7B7270020AA
:1018A000938787E52382C700B727002083A747E5F2
:1018B0009C439D83858B639FA700930760197CD30E
:1018C00054C737F700E0832707D193E78700232821
:1018D000F7D01DBF9307E01BDDB7F85231FFBDB74E
:1018E000B727002083A707E88847D847798D09C91B
:1018F00088C7B727002003A3C7A26303030002839E
:10190000828037270020B7260020138646E8130779
:1019100047EA8347D7008345B601484AAE97FD8B17
:10192000B355F500A300F600A306F700858995E9F5
:1019300003471701814613080002B3F7E702014786
:10194000B355E50085899378F70F89C96395D7006A
:10195000A30016018280850693F6F60F0507E311B2
:1019600007FF8280B7270020938787E583C757004A
:1019700093F7F70FD1EBB727002083A787B2411168
:1019800022C44AC006C626C2829737290020930780
:1019900049EA8047130949EA6302A406636885049B
:1019A000018DB7240020938744E883C7A70113540F
:1019B0005500938444E86363F404A13783C7A4010A
:1019C000032789009396570036971D8C2324E9003E
:1019D000E375F4FE224403C51400B2409244024968
:1019E00081454101171306E0670003FCB72700207B
:1019F00083A747B833848740229565B7B240224415
:101A000092440249410182808280B727002083A747
:101A100087B2011122CC26CA52C406CE4AC84EC68D
:101A20008297B7240020938744EA8047014A6301E4
:101A3000A406938444EA63668506018D3727002057
:101A4000930747E883C7A70113545500137AF5019C
:101A5000130947E8636BF402B7290020938909B89A
:101A60004D358346A90103A8840083A54900139737
:101A700056004297158C3A86636407016364B70089
:101A80003306B74090C4E37DD4FC1604336A4401A6
:101A9000F24062445285D2444249B249224A056129
:101AA0008280B727002083A747B8338487402295D8
:101AB00071B7B727002003A707E88967938707F462
:101AC0007CD3B727002083A747ED83A60709139689
:101AD00056006358060083A6070913966600634400
:081AE00006007453FDF2828040
:101AE800B72700203727002083A747AD0327C7ACB7
:101AF80001456313F700828083D6670081E683D6A9
:101B0800470036959C43F5B7B727002083A547B310
:101B180037270020938747B313860522232AC7ACAB
:101B280003D74700938785FFB72600204111BA974E
:101B3800056523A6F6AC06C61D05935637006374E3
:101B4800E500930600203307D60037250020232818
:101B5800E5AC23A0E522E1162312D60023130600E4
:101B68001CC3998FE1172312F700231307008D3F39
:101B7800B240B72700202391A7AE41018280B72742
:101B880000203727002083A747AD8326C7AC01452F
:101B98006393F600828003D7670011E703D74700F5
:101BA8006373E5003A859C43E5B7B7270020B7265D
:101BB800002083A747AD03A6C6AC2A87B305B54066
:101BC8006314F6003A8529A8938687009C43E36945
:101BD800D7FEE377F7FE2E85E3E4D5FEE3F2F5FEC4
:101BE800828023AC05FE1C4191E7010001000CC175
:101BF8008280BA8703A787FF6DFF23ACB7FE828078
:101C0800184183A785FF6319B7001CC1FD5723AC92
:101C180005FE238FF5FE8280232CF6FEC5BF4111F9
:101C280022C437E400E026C204403707200006C675
:101C3800F98C2320E4180F10000009E923209410E0
:101C48001545B24022449244410182800347E5FF92
:101C58009307F00F6306F700232094101145D5B7BA
:101C680097E0FB1FE780C04B014523209410D1BFAC
:101C7800411126C2B7E400E04AC003A90400B7072F
:101C8800200006C622C43379F90023A0F4180F10E7
:101C9800000009E923A02411B240224492440249D9
:101CA800410182809565938505D0C98D2A842105D7
:101CB800C2054205C181418197E0FB1FE7800038DA
:101CC80001CDFD5723200500231285002303F500CD
:101CD80023A024112105C9B723A0241101456DBFF4
:101CE8000111B7E700E04AC803A907004EC6370745
:101CF800200006CE22CC26CAAA893379E90023A07F
:101D0800E7180F10000037250020032485AD814413
:101D1800014619E499E8A1654E85EF00B00631A89F
:101D28008347E4FF6397370395C8A685130585ADF8
:101D3800C13D75D0A1654E85C92EF2406244B7E712
:101D480000E023A0271126854249D244B249056103
:101D5800828091E02286032484FF65BFA284E5BFC8
:101D680041114AC037E900E022C4032409003707BB
:101D7800200006C626C2798C2320E9180F1000001F
:101D880089E523208910154515A0B727002083C7AA
:101D9800D7ADAA842E8563F5F400894763EE9700D2
:101DA800BD3DB7E700E023A087100D45B2402244AF
:101DB800924402494101828083A785FF99E703C7BE
:101DC800E5FF9307F00F6308F700913DB7E700E0E0
:101DD80023A087104DBF37250020238F95FE1305BC
:101DE80085AD0135A16526850D260145232089107D
:101DF80075BFB727002023AC07AC8280B727002027
:101E080083A707B399E33E85828003D7270063162B
:101E1800B70003C70700E308A7FEDC47E5B7B9CD5D
:101E2800011106CE22CC26CA8147C14633D7F540D8
:101E3800058B21C312053E9531473305E502372747
:101E48000020832447B705443314F4002EC6420407
:101E58004180AA949C40C8408297B24523A00400C0
:101E680023A20400A18DF2406244D2442E8505616C
:101E780082808507E39CD7FA0144EDB72E858280DE
:101E8800BDCD797122D406D626D24AD04ECE014491
:101E98004147B3D78540858BB1CF1205314722958D
:101EA8003305E502B727002003A947B78544B39453
:101EB8008400C204C180BE892A990327090011C77A
:101EC800032549002EC60297B24531473304E40280
:101ED80083A749B73E941C4489E72320090023229D
:101EE8000900B2502254A58D02599254F2492E8508
:101EF800456182800504E31EE4F88144DDB72E8540
:101F080082804111B7E700E026C2844337072000EA
:101F180006C622C4F98C23A0E7180F100000B727C3
:101F2800002083A747B5372400201304049691C7DF
:101F380082971C403E9508C031A0B727002083A790
:101F480087B2FDF70840B74703009387D73F3305AB
:101F5800F502B7A72600938737ECB2403E9508C034
:101F68002244B7E700E023A0971092444101828001
:101F78000111B7E700E022CC80434AC837072000A8
:101F880006CE26CA2A892E86798C23A0E7180F1038
:101F98000000131506019305F004418132C697E04D
:101FA800FB1FE780A009AA8419C53246CA8597E0B5
:101FB800FB1FE7806026B7E700E023A08710F24008
:101FC800624426854249D244056182807971B7E727
:101FD80000E022D480433708200006D626D24AD013
:101FE8004ECE52CC56CA5AC85EC662C43374040177
:101FF80023A007190F10000005E123A08710094549
:10200800B250225492540259F249624AD24A424B7F
:10201800B24B224C45618280B727002083A787B244
:10202800BA8A368AB28B2E8BAA898297B727002064
:1020380003A747B73E898144B146C147338CD402D0
:1020480033068701104241E6C165938505F0414595
:1020580097E0FB1FE78080FE19EDB727002083A7D4
:1020680047B681C7814511458297B7E700E023A0AD
:1020780087102D4571B7B727002003A707B321E7BD
:1020880023A8A7B223000500832749B705473317BC
:10209800970023260500232475012311E500232238
:1020A8005501E29723A0370123A2670123A4570112
:1020B80063040A0023009A00B7E700E023A0871012
:1020C80001453DBF3E875C47F5FF48C765BF8504AE
:1020D800E396F4F6B7E700E023A0871021450DB793
:1020E800B727002083A7C7B7411122C406C63724E3
:1020F80000201304C4AD89C782975C483E9548C840
:102108004848B240224441018280B7E700E0984342
:10211800B706200023A0D718758F0F100000B72628
:10212800002083C6D6AD6372D502372600209316E9
:1021380015000325C6B2369583560500D58D2310A4
:10214800B50023A0E7100145828023A0E7100D45C4
:102158008280B7E700E09843B706200023A0D7188D
:10216800758F0F100000B726002083C6D6AD6374A4
:10217800D50237260020931615000325C6B293C54D
:10218800F5FF369583560500F58D2310B50023A07D
:10219800E7100145828023A0E7100D4582800111D8
:1021A80037E700E026CA0443B706200006CE22CC53
:1021B8004AC84EC652C4F58C2320D7180F10000009
:1021C800130705FF1377F70FFD4763E2E70AB146E8
:1021D800B306D502B727002003A747B736971C4395
:1021E800D9C71359450005443D893315A400131474
:1021F80005014180AE894A85A28509312A8A39C9F3
:10220800A2854A85B937B727002083A787B237291F
:102218000020130909B88297835789002A848146C8
:10222800B385370313060064B3B737031385053244
:10223800B335B500BE95EF905271B30785003E8760
:102248008326490063E4A70063E4D7003387D740B7
:102258002324EA00B7E700E023A097100145F240E5
:102268006244D2444249B249224A05618280B7E7B2
:1022780000E023A097100945DDB70111B7E700E09A
:1022880026CA84433707200006CE22CC4AC84EC649
:10229800F98C23A0E7180F100000BD4763E8A704D6
:1022A80031473307E502B727002083A747B7BA9716
:1022B8009C438DCF05443314A400420441802E89E9
:1022C8000145A285253EAA8911C5A285014551353A
:1022D80023A42901B7E700E023A097100145F240A5
:1022E8006244D2444249B24905618280B7E700E0BE
:1022F80023A097100945E5B779714AD037E900E07E
:1023080026D283240900B707200006D622D44ECE51
:1023180052CC56CA5AC85EC6FD8C2320F9180F1035
:102328000000B727002083C7D7AD6378F500B7272B
:10233800002083AB87B263970B00B7E700E023A0C8
:10234800971099A0B7290020938909B8AE8A03ABE2
:10235800490083D58900B74736FE938707C83E9B57
:10236800B387C5022A84328A8146B3B5C50213856C
:102378000732B337F50013060064BE95EF90F25CA0
:102388006370AB02232099100145B2502254925435
:102398000259F249624AD24A424BB24B45618280A5
:1023A800829B83D589002A8913060064B387450375
:1023B8008146B3B5450313850732B337F500BE959B
:1023C800EF90B258B30725013E8903A7490063E49B
:1023D800A70063E4E7003389E740D6852285393CC6
:1023E80009C923242501B7E700E023A09710054574
:1023F80069BF936504F0C205C181414597E0FB1FA1
:10240800E780C0C311E9B727002083A747B695D74F
:10241800A2851145829715B737270020832707B370
:1024280095E32328A7B28547232605002324250101
:102438002311550123008500A300F5002322050080
:102448005DB7BA87D84775FFC8C7F1BF7971B7E7D5
:1024580000E026D284433707200006D622D44AD08B
:102468004ECE52CC56CA5AC85EC662C466C26AC04C
:10247800F98C23A0E7180F1000002DC14144B6893C
:10248800B28A2E8A2A89B14C372B0020054D130CAD
:102498000003B30B940303274BB75E971C43A5E3D4
:1024A8009375F400B315BD0013554440C205568614
:1024B800C1811375F50F893539C183274BB7DE976D
:1024C80023A0270123A247016384090023808900F0
:1024D800B7E700E023A09710014521A023A097109B
:1024E8000945B250225492540259F249624AD24ADA
:1024F800424BB24B224C924C024D456182800504FE
:10250800E31984F9B7E700E023A097102145D1BF6C
:102518000111B7E700E026CA844322CC4AC84EC658
:102528003707200006CE2A84AE893289F98C23A089
:10253800E7180F100000C9332285CE85C1302A84E0
:1025480005C5B727002083D587B8130600648146E0
:10255800B3872503B3B5250313850732B337F500D1
:10256800BE95EF90923E48C013351400F240624485
:10257800B7E700E023A097104249D244B2490E05BC
:10258800056182800111B7E700E04AC803A9070086
:1025980022CC4EC63707200006CE26CAAA892E842A
:1025A8003379E90023A0E7180F100000EFF01F852A
:1025B800AA8419C123110500A2854E85593EB72763
:1025C800002083C7C7AD63993701B727002003D719
:1025D80047B2598C239287B2B7E700E023A02711AE
:1025E800014591E01945F2406244D2444249B2495A
:1025F8000561828001114AC837E900E022CC032432
:102608000900B707200006CE26CA4EC67D8C2320B7
:10261800F9180F1000009307F00263E6A704B1470A
:10262800B304F502B729002083A749B7A6979C43AE
:102638009DCB9377F5008545B395F500C205C1811B
:102648001181893783A749B70145A69723A00700B9
:1026580023A2070023208910F2406244D244424951
:10266800B24905618280B7E700E023A087100945D9
:10267800E5B74111B7E700E026C2844306C622C485
:1026880037072000F98C23A0E7180F100000EFF09F
:10269800EFF619E90145B2402244B7E700E023A06C
:1026A8009710924441018280B727002083A787B200
:1026B80000458297B7270020938707B86368A4026C
:1026C800D843B74636FE938606C83305A4403697E6
:1026D800E372E5FC13070064B335E50203D687000F
:1026E80081463305E502EF90522675B7D8433A94F0
:1026F800C1BF411122C426C237240020B7240020BC
:10270800130704B89384C4AD94485843B7270020EE
:1027180006C683A787B2130404B86392E6088297B3
:102728005440B74736FE938707C8B6973387A70044
:102738003A856364F7006364D7003305D740B7244C
:102748000020938784E5DC53938484E599CBB727ED
:10275800002083A647ED3707CDFF7D179C46F98FEC
:102768009CC611E14840B727002083A787B5829708
:1027780019E5DC5085C3EFF05176EFF0213FDC50CE
:1027880091CBB727002003A747EDB70633001C47B6
:10279800D58F1CC7B240224492444101828082975F
:1027A80094485840B387A6003E8563E4D700E3E821
:1027B800E7F83385E74061B74111B727002006C61F
:1027C80023AEA7B60295B240B727002023AAA7AE2A
:1027D800014541018280994763E9B700B727002086
:1027E8008A05938787B0BE9588C18280B727002065
:1027F80023ACA7B611C5B727002005472383E7B246
:102808008280B727002023A807B2B727002023AE6D
:1028180007B6B727002023A407B237250020B7271B
:1028280000204111238307B27146B7270020814554
:10283800130585B006C623AC07B622C426C23724C2
:10284800002097E0FB1FE78040A41305C4AD1306E2
:102858008002814597E0FB1FE78020A3EFF0CFAA15
:10286800B7270020938747B303C5C70383C7D70398
:102878001304C4AD85453E958D473305F502994748
:10288800B724002039051375F50F2301A40033057B
:10289800F5021305052497D0FB1FE780207A23AAA9
:1028A800A4B649C103462400994781453306F60278
:1028B8001306062497E0FB1FE780209D83A744B7F3
:1028C80003472400B7240020938707240A0723A27C
:1028D800F4B0BA97372700202326F7B2EFF06FD16C
:1028E800A5218347140083A644B037260400139714
:1028F80027003697130686E810C313871700137747
:10290800F70F0A07372604003697130666E210C346
:1029180013873700890793F7F70F8A07A300E400A6
:10292800B69790C3B240224492444101828037272F
:1029380000201307C7AD834717008346270063F0BD
:10294800D702B726002083A646B013861700A30037
:10295800C70013972700369708C33E8582809307E0
:10296800F00FE5BF1C41638C071041777D8FB706D8
:10297800002089476316D7100357450063020710E4
:10298800411126C21946AA849305F00F610506C6AF
:1029980022C497E0FB1FE780C09D05478D47630A67
:1029A800E50C9C4491C7D858994761C7985C71C396
:1029B80037240020130600048145130544B397E02B
:1029C800FB1FE780808C13060004A685130544B31B
:1029D80097E0FB1FE7804084930744B303D7C70001
:1029E80009E7130700102396E70003C7E70001E78C
:1029F80005472387E70003D7070101E76D472398B9
:102A0800E70003C7F70001E71547A387E70003C7F7
:102A1800270101E705472389E70003C7370109E7CD
:102A280003C7F700A389E70003C7570101CB9376D3
:102A380037000983238ED702A38EE70203C7470115
:102A480001E75547238AE70003C7640109E713072D
:102A5800C003238BE7009C5791C78297B7270020B4
:102A68002392A7AEB72700207D57A38CE7F2513BEE
:102A78008147B240224492443E8541018280894781
:102A88003E85828001114AC837290020832709B86A
:102A980006CE22CC26CA52C456C24EC68297130A04
:102AA8000064B3354503130909B8835A8900814680
:102AB800568633054503EF904269B72700201387F0
:102AC800C7AD004FAA840145630694029389C7AD38
:102AD80033858440636E94000325490056868146F9
:102AE800B335AA023305AA02EF902266018D269516
:102AF80023AC9900F2406244D2444249B249224A86
:102B0800924A05618280011122CC2E84B7C5060045
:102B18000A8541469385055A06CEEF90921C1808FF
:102B280006043A94B7270020035504FF83D7A7B8B3
:102B3800F2406244AA9737450F0013050524335520
:102B4800F50205618280B727002083D7A7B85147CF
:102B58001D45637CF702794719456378F702130727
:102B6800200315456373F7021307B0041145637E0C
:102B7800F700130740060D456379F700130760094E
:102B880009456374F70013B5B70F8280011122CC91
:102B980006CE2A842EC6EFF0CFB6B245F240818D1C
:102BA80033A5A502229562441375F50F056182804D
:102BB800011122CC06CE2A842EC6EFF08FB4B2457E
:102BC800F240818D33A5A5022295624442054181D8
:102BD80005618280011122CC06CE2A842EC6EFF030
:102BE8004FB2B245F240818D33B5A50222956244B9
:102BF80005618280B7270020138747B318572DC374
:102C0800411122C426C24AC006C6138947B3029797
:102C1800B72700201387C7AD035787002A849384FA
:102C2800C7AD0DCBBA876373A700AA87C207C18354
:102C3800BA866373E400A286C206C182958F5147A3
:102C4800635AF7008327C90291C38297EFF01112E4
:102C580023948400B2402244924402494101828074
:102C680082800111B727002022CC3724002023AA14
:102C780007B8930744B3DC5706CE26CAAA851304BF
:102C880044B381C72AC68297B245C9C19C4105454C
:102C9800ADCBDC41BDC783D78500A5C783D7A500C9
:102CA800ADC3B7240020138504B85146938404B8F3
:102CB80097D0FB1FE780405623860400B7270020E3
:102CC80083A607B8372700202324D7B20347740107
:102CD8001DE3938707B803D58700930780573746C6
:102CE8000F003305F5021306062481468145EF904F
:102CF800C245A30BA400373504001305C5A86D3CD5
:102D08000145F2406244D24405618280B727002021
:102D18009387C7AD3707002023AE07001307676EF8
:102D2800B727002023A0E7B837873200938707B872
:102D3800FD56130727A1D4C398C723860700B7C732
:102D4800004023A4D7269DBF011122CC37240020A0
:102D5800930744B3884706CE26CA4AC801E9054501
:102D6800F2406244D244424905618280130444B36C
:102D78005C58F5D7185C65D770008545829718446C
:102D8800B247E30EF7FC0355C4009305E004B724EB
:102D9800002097D0FB1FE780602A1387C4AD08D3B3
:102DA8009384C4AD4DDD0356C4009305F00F01496B
:102DB80097D0FB1FE780604D8347E4009050634D38
:102DC800F900328597D0FB1FE7808035014523A0A5
:102DD800040223A2040269B78355C4000844185C9E
:102DE800B3872503898105093E9508C20297E9B78B
:102DF80001114EC6B7290020938749B39C4726CABC
:102E08004AC852C406CE22CC56C25AC02A8AAE84B8
:102E18003289638D071E938949B303A74903630465
:102E280007121307F01F6362A71237240020130745
:102E3800C4AD832A07021304C4AD639A0A0803D5F4
:102E4800C9009565938515E097D0FB1FE780001FA3
:102E580008D02A866DC983D5C90083A7490303A56D
:102E680089008981829783A78900832A04025CD01C
:102E780089476316FA08C1476397F40C83D5C900DC
:102E88009147938505FCB3C5F5028A05D69503C716
:102E980025009307A0056314F70A83D705006390FC
:102EA800470B4A852686910597D0FB1FE780C036D9
:102EB8001C505685639357130145F2406244D2442F
:102EC8004249B249224A924A024B056182805850CF
:102ED800E380E7FA03D5C9009565938525E097D087
:102EE800FB1FE780A015AA8A39CD83D5C9002A8699
:102EF80083A7490303A589008981829795BF8D47D8
:102F0800631BFA00C1476390F40483D5C900938515
:102F180045FDF199A5BF91476318FA0063954403ED
:102F280083D5C900A115F5B793070010631DFA00F2
:102F3800A14763EA970083D5C900C115D9BF1C50C2
:102F480056856390570D29458DBF9D6A637C550949
:102F5800930A05E01947B3CAEA0203D7C900372B19
:102F68000020B38AEA02BE9A9307CBADDC53130B59
:102F7800CBAD6395570103240B021DE003D5C900AF
:102F88009305E00497D0FB1FE780400B2A8445DDBA
:102F980083D5C90083A749032A86898156858297E4
:102FA80091451307A005898193972500A29783C6A9
:102FB80027006393E60483D60700639C46038505D0
:102FC8008A052686A2954A8597D0FB1FE780C024EC
:102FD80083270B02E38287EE228597D0FB1FE780C9
:102FE8002014D9BD21677917E36FA7F4B30A5541B7
:102FF800ADB783C5370045BF83270B02E38587F448
:10300800228597D0FB1FE780A01135BFB727002086
:1030180083A5C7AF8DD991479306A00589831397D8
:1030280027002E9703462700E31FD6F00356070014
:10303800631C460185078A072686BE954A8597D070
:10304800FB1FE780601D8DBD83473700C1BFB727D1
:103058000020938747B3984729C3985F1DCF8546BB
:10306800631DD502411122C4372400201304C4ADC6
:10307800105006C619CE83D5C700485089810297DB
:10308800085097D0FB1FE780A009232004022322C1
:103098000402B2402244410182808280011122CC84
:1030A80037240020930744B356C283AA870026CA50
:1030B8004AC84EC606CE52C42A89AE84B2891304C1
:1030C80044B3638C0A1C1C5C99EB2945F2406244AA
:1030D800D2444249B249224A924A056182805C58E8
:1030E800EDD79307F01F63E8A70C372A0020930752
:1030F800CAAD9C53130ACAADB9C7084483274A020C
:10310800639FA70489476317F906C147E39FF4FA49
:103118000355C4009147130505FC3345F502931781
:10312800250003250A022686CE853E959307A0052D
:103138002301F50023102501110597D0FB1FE78017
:10314800A00D014561B70355C4009305E00497D06D
:10315800FB1FE780A0EE2320AA0245F1BDB78355E7
:10316800C4005C5803260A02898182971C442322E2
:10317800FA0249BF8D47631CF900C147E397F4F48D
:103188000355C400130545FD9377C5FF59BF914703
:103198006318F900E39B24F30355C4002115EDB728
:1031A80093070010E313F9F2A147E3E097F2035500
:1031B800C4004115D1BF9D676378F506930705E004
:1031C8001947B3C7E7020357C400372A0020B3875B
:1031D800E702BE9A9307CAAD9C53130ACAADA1CFA2
:1031E80083274A026395570703250A029146130865
:1031F800A0059305F00F93D72600139727002A9769
:10320800034627006316060783580700034637005E
:10321800639C2805B306D64063C6960485078A07CB
:103228002686CE853E9511BF21677917E36FA7E8FB
:10323800B307F54049BF0355C4009305E00497D090
:10324800FB1FE780A0DF2320AA0259F9BDBD8355E3
:10325800C4005C5803260A02898156858297232276
:103268005A0359B72310B70093160601C18261B7F4
:103278000356C400B38596009105130606FCE3F6D1
:10328800C5E413863400719A1106B296230107012A
:1032980023102701A301D70051B7372A002093072D
:1032A800CAAD9C53130ACAADA9C303250A029146A5
:1032B8001308A0059305F00F93D72600139727004E
:1032C8002A97034627006314060583580700034618
:1032D800370063982801B306D640E3D196F423104B
:1032E800B70093160601C182C1BF0345E4008357A6
:1032F800C4009305E0043305F5024205418197D0E7
:10330800FB1FE780A0D32320AA0245F17DBB03560B
:10331800C4008345E400B385C502338696001106D0
:10332800E3E5C5DAB9BF0145828083C705002300FC
:10333800F50083D72500A300F50083D72500A183D6
:103348002301F50083C74500A301F50011458280DC
:10335800B727002023AA0798B727002023A8079893
:10336800828029C1411126C206C622C4AA84014509
:103378008DC52E84B7C50600228541469385055B19
:1033880097D0FB1FE78040E983C704000545230663
:10339800F40083C71400A306F400B2402244924408
:1033A8004101828001458280011122CC26CA06CEC5
:1033B8000947AA8432846381E50441468147639BB7
:1033C800C500638FE6006397B6000DA841478147A3
:1033D800638EE600F2406244D2443E8505618280F5
:1033E8008A852285BD3F41468A8519A88A85953FE9
:1033F80041468A85228531A0E39AB6FC2E86A285AD
:10340800268597D0FB1FE78060EEAA87E1B7B7272C
:10341800002023A8A7988280B727002023AAA7986E
:103428008280011122CC0354650006CE26CA4AC800
:103438004EC641C083298500AE842A8803C9090085
:10344800814713178901618763550702B14705450D
:1034580063FA8704511442040355280041803387D6
:103468008900A2864E868545EFC0C00FB337A000FD
:1034780085077D1413556900420405891379F903FA
:1034880041802380F400A380A40023812401239297
:103498008400014719C01387190098C4094763833A
:1034A800E7000145F2406244D2444249B24905610D
:1034B80082800545C5BFC167F917630AF502D94778
:1034C80063F7B702011122CC2EC606CE2A84EF90EC
:1034D800C049B2456368B50022856244F24005617F
:1034E8006FA01070F2406244054505618280054571
:1034F8008280C167F9176314F5006F900047411186
:1035080006C6EFA0B05C11E15D45B2404101828082
:1035180091476394F502834705002300F60083472B
:10352800250003471500A207D98F2311F60083470A
:10353800350001452302F600828011458280411141
:10354800814522C426C206C6AA8405252A8409E91B
:10355800B727002083A7079981C7F9452685829751
:103568002285B240224492444101828039714ED66C
:1035780056D25AD006DE22DC26DA4AD852D4AA8A93
:103588002E8BB28941EF36C6AD379145EF90A04FEB
:10359800AA844D492DC9B246054A23803401054401
:1035A800630A0B00B68513851400029B05051314E6
:1035B80005014180E20993D9894163D30902C145D4
:1035C8005685EFA0F05E654905E933868400A2853B
:1035D8002685EFB0303E2A8905E131044204418056
:1035E80091472C085685231CF10026CE231D810007
:1035F800EFA0A0642A8901C963070A00268597D02D
:10360800FB1FE780E0B1F25062544A85D254425918
:10361800B259225A925A025B21618280BA84014AC5
:10362800ADBF011122CC26CA4AC84EC606CE2A8989
:103638003284B689253FAA840DE1B727002083A7E5
:10364800479981CF05476317E40003C409000504BF
:103658001374F40FA2854A858297F2406244268546
:103668004249D244B24905618280AE86B73504002A
:1036780001470546938525336DB783D70500230099
:10368800F50083D70500A183A300F50009458280D2
:1036980083D705002300F50083D70500A183A30085
:1036A800F50083D725002301F50083D72500A183E2
:1036B800A301F5001145828083D705002300F5009A
:1036C80083D70500A183A300F50083D72500230134
:1036D800F50083D72500A183A301F50083C7550012
:1036E8002302F50083C76500A302F50003D5850012
:1036F800190542054181828083D705002300F50022
:1037080083D70500A183A300F5000945828083D7EC
:1037180005002300F50083D70500A183A300F50069
:1037280083D725002301F50083D72500A183A301B2
:10373800F5001145828003D5450006054205418103
:10374800828083D705002300F50083D70500A18375
:10375800A300F50003D525000905420541818280B3
:1037680083D705002300F50083D70500A183A300B4
:10377800F50083D725002301F50083D72500A18311
:10378800A301F50003D5450011054205418182805A
:1037980083C705002300F5000545828083D705000F
:1037A800411122C406C62300F50083D705002E84E4
:1037B8001105A183A30EF5FE83D725009505230FD8
:1037C800F5FE83D7D5FFA183A30FF5FE03C6F5FF4A
:1037D80097D0FB1FE78040A403454400B240224431
:1037E8001105410182808947639CF50083471500D4
:1037F800034705000145A207D98F2310F6008280F0
:103808001145828003D70500D94763FEE7020111FD
:1038180022CC06CE2EC62A84EF902015B24683D736
:103828000600636DF50022856244F240B735040056
:10383800014709469385256805610DBBF24062443E
:103848000945056182800945828091479DC5834667
:103858000500FD15C2058547C1816392F60213D79D
:1038680025008D89914791E9914701CB05052301F1
:10387800D6002310E60048C281473E85828009476A
:103888009147E39CE6FEC94733D7F502B3F5F50245
:10389800D1BFAE86B73504000147114693858569C7
:1038A800F1B193F7350091EB8981914789C52310D0
:1038B800B60048C281473E8582809147EDBF03C765
:1038C80045008947631AF702011122CC2A84C845AA
:1038D80006CEAE86014719C52EC69D45EFE0EFAC72
:1038E800B2462A8722856244F240B7350400194659
:1038F8009385056C05619DB90945828099E111455B
:1039080082808347050005472311F600E379F7FE17
:10391800FD1593F5F50F33D7F502B387E702E3906A
:10392800F5FE050548C22310E6000145828083C7DD
:1039380045000947AE866385E70041476399E7007C
:10394800B7350400014721469385457A05B10945F5
:1039580082802310B60091E1014548C2014582806A
:10396800AE86B73504000147294693850570FDBE2C
:103978002310B60091E1014548C201458280AE8618
:10398800B73504000147314693856571C5B62310E4
:10399800B60091E1014548C20145828003D7450040
:1039A800854763FDE702011122CC2A84884106CEAF
:1039B8000DC12EC68545EFE04F9F2A8722856244B8
:1039C800B246F240B735040039469385E573056180
:1039D80071BEF240624409450561828009458280D2
:1039E80091479DC5034705008D46914763F2E6025E
:1039F800FD15C205C181B3C6E5023308D702639934
:103A0800050105052310D6002311E60048C28147A9
:103A18003E85828083C745000947AE866385E700F7
:103A280041476399E700B73504000147414693854C
:103A3800457A2DBE09458280B335B000139525001F
:103A48008280011122CC26CA06CE03C7850085478D
:103A5800AA842E8449466310F702613C83572400E8
:103A680049151306200963C8A700F2406244D244EE
:103A78000945056182800347940085476314F70070
:103A880013660604484011C58D4532C6EFE0EF9134
:103A98003246A2866244F2402A872685D244B73548
:103AA80004009385A5740561D1B48D4763FFB702FF
:103AB8008347150003470500F115A207D98F231086
:103AC800F6008347350003472500C205A207C181D8
:103AD800D98F2311F6002312B60089C5110508C62F
:103AE8000145828023240600E5BF1145828001112B
:103AF80022CC2A84884506CEAE8611C52EC69545A9
:103B0800EFE0AF8AB2462A8722856244F240B73591
:103B18000400594693858576056189BCB335B000A4
:103B2800139525008280AE86B735040001476146AB
:103B38009385857925BC8547114563F4D70283476A
:103B4800160083450600A207CD8F2310F700938740
:103B5800E6FF2311F70089476386F600090650C37C
:103B68000145828023220700E5BF01478146794647
:103B78008145EDBA83D705002300F50083D70500FA
:103B8800A183A300F5000945828083C72500054766
:103B98002300F50003D505006397E7000A0505052E
:103BA800420541818280C9473305F502CDBF03D55F
:103BB80005000A0542054181828083D7250023003C
:103BC800F50003D5050083D725003305F502050563
:103BD80042054181828003D50500828003D5050016
:103BE800828003D50500828083D725002300F50055
:103BF80003D5050083D725003305F50205054205E1
:103C08004181828083D705002300F50083D7050012
:103C1800A183A300F50083D725002301F50083D7EE
:103C28002500A183A301F50003D545001105420530
:103C38004181828083D705002300F50083D70500E2
:103C4800A183A300F50003D525000905420541819C
:103C5800828089471145639BF60083471600834697
:103C680006000145A207D58F2310F700828003D7ED
:103C78000500D947AE8663F9E700B7450400014758
:103C88000D469385C5B771BA09458280114563937E
:103C9800A60283471600834606000145A207D58F72
:103CA8002310F7008347360083462600A207D58FE6
:103CB8002311F700828083C725000547FD1793F776
:103CC800F70F6361F70483D705008DCF011122CC6C
:103CD8002A84C84106CE15C12EC68945EFD0FFEC0F
:103CE8002A8722856244B246F240B7450400154649
:103CF800938525B905616FF0DF92F240624409456A
:103D080005618280094582809547114563F9D70688
:103D1800411122C426C24AC006C683471600BA8487
:103D280003470600A2073284D98F2390F400834703
:103D380036000347260093054400A207D98F239134
:103D4800F40089472382F400094613855400368914
:103D580097C0FB1FE780404C9307A9FF2394F4000A
:103D68009947631BF90023A60400B24022449244F9
:103D780002490145410182801904C0C4FDB782800F
:103D880083D705008DCF011122CC2A84C84106CEE5
:103D980015C12EC68545EFD05FE12A87228562448A
:103DA800B246F240B74504001D46938565BB0561E0
:103DB8006FF03F87F24062440945056182800945FA
:103DC800828099476395F6048947411106C6230204
:103DD800F7008347160083460600B285A207D58FF1
:103DE8002310F70083473600834626000346470022
:103DF800A207D58F130557002311F700910597C027
:103E0800FB1FE7806041B240014541018280D147F4
:103E180011456394F600C1474DBF828083D70500E2
:103E28008DCF011122CC2A84C84106CE15C12EC6D9
:103E38008945EFD09FD72A8722856244B246F2404F
:103E4800B74504002546938525BC05616FF06FFDD5
:103E5800F2406244094505618280094582808947AC
:103E68001145639BF600834716008346060001450B
:103E7800A207D58F2310F7008280011122CC2A8453
:103E8800C84106CEAE86014719C52EC68545EFD076
:103E9800DFD1B2462A8722856244F240B745040042
:103EA8002D469385E5BD05616FF0AFF71145639326
:103EB800A60283471600834606000145A207D58F50
:103EC8002310F7008347360083462600A207D58FC4
:103ED8002311F7008280011122CC2A84C84106CE22
:103EE800AE8611C52EC68545EFD03FCCB2462A878F
:103EF80022856244F240B74504003546938545BEA5
:103F080005616FF00FF293F71600114589EB8947A9
:103F18006387F60085822312D70010C3014582808B
:103F2800011122CC2A84C84106CE15C12EC685456A
:103F3800EFD0BFC72A8722856244B246F240B74510
:103F480004003D469385A5BE05616FF08FEDF240F4
:103F5800624409450561828083D705008DCF011130
:103F680022CC2A84C84106CE15C12EC68945EFD079
:103F7800DFC32A8722856244B246F240B74504006F
:103F88004546938505BF05616FF0AFE9F24062448D
:103F980009450561828009458280854763FCD7020F
:103FA8002304A700A304B70083471600834506002F
:103FB800A207CD8F2310F7009387E6FF2311F700A0
:103FC80089476386F600090650C30145828023228B
:103FD8000700E5BF11458280014781464D4681456E
:103FE8006FF02FE48D47114563FBD7028347160016
:103FF80083450600A207CD8F2310F70083473600BC
:1040080083452600A207CD8F2311F7009387C6FFAB
:104018002312F7006386A600110610C701458280A7
:1040280023240700E5BF011122CC2A84884506CE47
:10403800AE8611C52EC69545EFD03FB7B2462A8742
:1040480022856244F240B74504005D469385C5C0A9
:1040580005616FF00FDD854711456397F6008347CB
:10406800060001452300F700828001478146654626
:1040780081456FF00FDB011122CC2A84C84106CE9E
:10408800AE86014719C52EC68D45EFD01FB2B24680
:104098002A8722856244F240B74504006D4693851D
:1040A800C5C305616FF08FCC011122CC2A84C841A9
:1040B80006CEAE86014719C52EC68D45EFD0FFAE98
:1040C800B2462A8722856244F240B7450400754605
:1040D8009385C5C305616FF06FC9011106CE2EC661
:1040E800EFA0E01A01C9B245F24003552500056169
:1040F8006FE0C071F240494505618280B727002012
:10410800A380079CB72700202380079CB72700209F
:1041180023A4079AB727002023A6079AB7270020C9
:1041280023A8079AB727002023AA079AB7270020B1
:1041380023A2079AB727002023A0079AB7270020B1
:10414800239C07BA93064038938787BB2391D702ED
:10415800F1761307400B938606B82391E700239264
:10416800D70211679D46130600059305000A13053B
:10417800007D2392E7002393D70241478546130821
:1041880010F82395E7002396E7002399E700239A80
:10419800E700239BE700239CE7002394E70223938F
:1041A800B7002394B7002397C7002398C700239D1F
:1041B800A700239E0700239F07002390070223954B
:1041C800D70223960703239707029308F00723983B
:1041D80007022392E7042393E704239FE70423902D
:1041E800E7062391E7062392E706239917031307A7
:1041F800C01C239AD702239BD702239C0702239D26
:104208000702239E0702239F070223900704239196
:10421800D70423940704239507042396D7042397E8
:10422800C7042398C7042399A704239A0704239B48
:104238000704239C0704239DC704239EC7042393D4
:10424800A7062394070623950706239607062397B0
:10425800B7062398B70623990706239AE706514716
:10426800239DE7067D57239B0706239C0706239E6D
:10427800D706239F0706239007092391E708828022
:10428800011126CAAA84214522CC06CE2E8432C624
:1042980036C43AC2EFD0DF9D1DC9A2461247324646
:1042A800930700FD2300F5009947A300950023011B
:1042B800F5002303D500A303E5002312C500AA8552
:1042C80022856244F240D24405616FD07FA9F24052
:1042D8006244D24405618280B727002023A4A79AAC
:1042E8008280B727002023A6A79A8280B7270020BC
:1042F80023A8A79A8280B727002023AAA79A82809A
:10430800011122CC4AC806CE26CA2A890144B30420
:1043180089006368B400F2406244D24442490561AE
:1043280082802EC6EFD0FFBD93170501C183A183FC
:10433800B2452380F4009307140093F7F70F850420
:1043480063F9B700CA9709042380A7001374F40F10
:104358007DBF3E847DBF411122C437240020130451
:1043680084B903556400C16706C6FD17630FF500DD
:10437800B727002003C687CFB72500209385859BE4
:10438800EF90904EFD572313F400B24022444101B0
:10439800828009C925151375F50F1335850E134548
:1043A800150082800145828023900500C9C6797175
:1043B80022D426D24ECE52CC5AC806D64AD056CA95
:1043C8005EC63684328AAE892A8B814463F34407F9
:1043D800B307940083C70700138914004209939A0E
:1043E800070193DA0A011359090163840A04CA9779
:1043F8006341FA04B307240183CB07005E85513F6C
:104408000DC99387FAFF2390F90063906B03130596
:1044180019002295B250225492540259F249624A24
:10442800D24A424BB24B45618280D694C204C180C5
:1044380071BF0145C5B701458280011122CC3724DF
:10444800002026CA4AC84EC6930784B906CE2E89CC
:10445800D0CB8CCBC8C7AA8441469305F00F4A85B8
:1044680097C0FB1FE780E0F08549130484B96319FE
:1044780035030848C145693541469305F00F26853F
:1044880097C0FB1FE780E0EE054963152503484404
:104498006244F240D2444249B249C14505618DB5F2
:1044A800414681454A8597C0FB1FE78080ECE315AC
:1044B80035FDC1B741468145268597C0FB1FE7807A
:1044C80040EBE30625FDF2406244D2444249B2493A
:1044D80005618280411122C43724002026C24AC0C7
:1044E800AE842A89130600028145130584B906C6DD
:1044F80097C0FB1FE78060D9930784B9A381270180
:10450800B7270020238E97CEEFE08032854719C168
:1045180081474945230CF4B8B240224492440249E9
:1045280041018280814781CD19C98547631BF50008
:1045380083C7550093E707FCA382F50085473E85AE
:10454800828089476317F50083C7550093F7F703FF
:10455800E5B70D478547E314E5FE03C75500137714
:10456800F70313670704A382E500D1BF81478DC114
:1045780005C103C755009306000C85471377070C40
:104588006308D700930600048D476303D700894763
:104598003E858280411122C4005D06C626C21DC820
:1045A800AA84085009C597C0FB1FE78060B7485028
:1045B80009C597C0FB1FE780A0B6085409C597C076
:1045C800FB1FE780E0B5228597C0FB1FE78040B559
:1045D80023AC0402B240224492444101828019E98A
:1045E800B727002083C7A7B991C73725002013052F
:1045F8008599828037250020130505BB8280B7275F
:10460800002003C5A7B98280B727002003A547BAB1
:104618008280B727002003A587BA8280B7270020A9
:1046280083A7C7BA88438280B7270020938787B9B2
:10463800D44B9842050798C203C537009307F00F7B
:104648006305F50091656FD05FAC8280011122CCC3
:1046580006CE2E8432C6EF9030549147B24563108F
:10466800F502B727002083A7479B95C303A307003C
:10467800630F030022856244F24005610283B72775
:10468800002083A7C79A81C703A34700D5B7F24084
:104698006244054505618280011122CC2A840355B4
:1046A800450006CE26CA4AC84EC6EF90102D25CD25
:1046B8002A89834405008349C500E93D4A85EFA05E
:1046C800C00C03554400EF907048372900201309A7
:1046D800099C83470900A1CF639B9704B727002053
:1046E80083C5179C2685EFF05F9F19E12300090019
:1046F80003554400EF90504A9147631FF500B727D0
:104708000020938787B98356440003D767006395D1
:10471800E6007D572393E700F2406244D2444249C1
:10472800B2490561828081499304F00F79BF9307EC
:10473800F00FE38FF4FA8346640003564400034500
:1047480024004E87A6852D3E65B779715EC6AA8B73
:104758002E8552CC56CA5AC806D622D426D24AD05A
:104768004ECEAE8A328B368AEF9030217DC1045D01
:104778002A89E5C09C50614599C3130540039C54A0
:1047880081C751054205418163050A00710542054B
:104798004181DC5081C75D0542054181EFD04FCD95
:1047A8002A8445C96146814597C0FB1FE780E0AD73
:1047B800B727002083C987BE63940900834909008D
:1047C800930700FD2300F400A947A3007401230107
:1047D800F400230364018C5023125401130584014F
:1047E80091C908C47146930A440397C0FB1FE78028
:1047F800A0A256858C5491C948C45146930A4501D4
:1048080097C0FB1FE78040A15685630C0A0008C8C3
:104818007146D285930AC50197C0FB1FE780C09FE8
:104828005685CC5099C548C85D4697C0FB1FE780A0
:10483800A09EA2854E85EFD0AFD22254B25092549A
:10484800F249624AD24A424BB24B4A850259456103
:1048580091B3B250225492540259F249624AD24A50
:10486800424BB24B4561828001114EC6AA892E8502
:104878004AC806CE22CC26CA2E89EF90101021C92C
:10488800B727002083C487BE99E0834405001945F3
:10489800EFD00FBE2A8405CD8145194697C0FB1F6E
:1048A800E780A09E930700FD2300F400B947A3000A
:1048B80034012301F40023122401A2856244F2404A
:1048C8004249B2492685D24405616FD06FC9F2408A
:1048D8006244D2444249B2490561828039715ECE50
:1048E800AA8B2E8526DA4ED652D456D25AD006DE58
:1048F80022DC4AD8AE84328BB68A3A8ABE8942C64E
:10490800EF90B00721CD2A894145EFD06FB62A84B0
:1049180031C54146814597C0FB1FE7800097B727FF
:10492800002003C587BE19E103450900930700FD70
:104938002300F400BD472301F400B247A30074012B
:104948002312940023046401A304540123054401A1
:10495800A30534015CC4A285EFD08FC0F250625425
:10496800D2544259B259225A925A025BF24B2161EF
:104978008280797126D2AA8439454AD04ECE06D68D
:1049880022D42EC6B2893689EFD08FAE21C1B24566
:104998009307000D2310F500B1472A842312B500B0
:1049A8002301F500CE851905194697C0FB1FE7803E
:1049B800A08623062401A2852254B2500259F24946
:1049C80013F5F40F925445616FD08FB9B250225449
:1049D80092540259F24945618280411126C2B72496
:1049E8000020938484B903C7340006C622C44AC091
:1049F8009307F00F630CF7042A893945EFD04FA7C6
:104A08002A8429C5930700FDB72500202300F50057
:104A1800A300250123010500938505BB0D05194653
:104A280097B0FB1FE780407F83D78400A28503C52A
:104A380034002315F40083C714002306F40022442D
:104A4800B2409244024941016FD08FB1B240224432
:104A5800924402494101828001115AC02A8B314592
:104A680026CA4EC652C456C206CE22CC4AC8AE8406
:104A7800B28A368ABA89EFD0AF9F3DCD2A8426857F
:104A8800EF90A06F11C50347C500A1476314F70451
:104A9800B727002003C9B7B9930700FD2300F40026
:104AA8009D47A30064012301F400231294002313FB
:104AB80054012314440123153401A2856244F240B1
:104AC800D244B249224A924A024B4A854249056178
:104AD8006FD00FA9B727002003C9D7CFE31E0BFA61
:104AE800B727002083A787A79C47DDD7CE865286A5
:104AF800D685268582974DB7F2406244D244424912
:104B0800B249224A924A024B05618280011122CCA5
:104B18002A84214506CE2EC6EFD08F9521C1B245F5
:104B2800930700FD2300F500C5472301F50083C75F
:104B38003500A301F50083D745002312F50083C78C
:104B480065002303F50083C77500AA85A303F50054
:104B580022856244F24005616FD08FA0F240624422
:104B680005618280397162CC2A8C594526DA4AD887
:104B78004ED652D456D25AD05ECE06DE22DCAE8451
:104B880032C636C4BA8B3E8BC28A468A8359010420
:104B980003494104EFD0CF8D25C93246930700FD64
:104BA800A2462300F5009547A301C500A30085018F
:104BB8002301F5002A8419461105A9C2B68597B0C4
:104BC800FB1FE780606523066401230A240123157F
:104BD8007401231754012318440123193401A285B1
:104BE8006254F2504259B259225A925A025BF24B1D
:104BF800624C2685D25421616FD08F96814597B03B
:104C0800FB1FE7808068C1B7F2506254D254425902
:104C1800B259225A925A025BF24B624C216182804D
:104C2800411122C437240020130484B98347240087
:104C380006C626C28DCBB7240020AA85194613853F
:104C4800849997B0FB1FE780205D03452400938576
:104C58008499EFF03F8D2244B240138584999244A1
:104C680041016FD0B03DB240224492440145410118
:104C78008280411126C2B7240020938784B906C6D2
:104C880022C44AC003C737009307F00F938484B93E
:104C98006304F7042A892945EFC09FFD2A840DCDB6
:104CA800930700FD2300F500A147A3002501230178
:104CB800F50083C72400B725002093858599A301B3
:104CC800F5001946110597B0FB1FE780E05403C5AE
:104CD8003400A285EFD0CF8803C724008D47631125
:104CE800F702B727002083A7079B99CB03A3870068
:104CF800630803002244B2409244024941010283FE
:104D0800B24022449244024941018280797122D4FE
:104D180006D626D24AD04ECE52CC56CA09445DCDCC
:104D28002A8903550500AE895144EF900045AA84AD
:104D380055C537270020930787CF83C74700854687
:104D4800BA8AFD1793F7F70F494463F9F608034742
:104D5800C500A1476314F700639209089C5C4544A9
:104D6800B5EF9165938545711305C00297B0FB1F98
:104D7800E780C02C88DC2A8A4D442DC11306C00266
:104D8800814597B0FB1FE780405083570900930681
:104D98004A0036852311FA0071469305490036C644
:104DA80097B0FB1FE780404789472300FA0003C5F7
:104DB800C400B2460356090083C58ACF611513356E
:104DC8001500EFA0006E2A8463860900CE8526852B
:104DD800EF90504B01C42685EFF0CFFB2285B250EF
:104DE800225492540259F249624AD24A4561828059
:104DF800B727002083C7C7CF0547FD1793F7F70FDD
:104E08006378F708894751C6011122CC26CA4AC8D7
:104E18004EC652C406CEAA89368AB2842E89EF902D
:104E2800C0352A84D14729C9485509C597B0FB1F01
:104E3800E780002FF1452685EFD08F9348D4CD47E2
:104E480005CD8346C40021478147639FE600630D73
:104E58000A000347A5010356050193062501AA8503
:104E68004E85EF90D049AA8703474400630F090095
:104E7800136767002302E400F2406244D2444249C7
:104E8800B249224A3E850561828013674700DDB733
:104E9800C9473E8582809307000463EBA700B727C4
:104EA8000020938787BB06053E9503550500828041
:104EB80041657D158280011122CC2A842E8526CA5F
:104EC80006CEAE84EF90602B1DCDB7470F009387B9
:104ED800F723094563E4870281450A85414697B06F
:104EE800FB1FE780803AA685231081000A85418050
:104EF80023018100A3010100EFA0203AF24062449F
:104F0800D244056182804945D5BFB7270020238D4B
:104F1800A7CE82806FA00053797152CC2A8A32853D
:104F280022D426D24AD04ECE56CA5AC85EC606D613
:104F380062C4AE8BB28A368BBA843E89C2894684F3
:104F4800EF90A02315C92A8C63140A0213774B002B
:104F58008347450015CF93E727012302FC008DEC1A
:104F6800631C0902639A090205E8ED9B2302FC0011
:104F7800832B8C03639F0B06B25022549254025920
:104F8800F249624AD24A424BB24B224C4561828076
:104F9800F59B93E70701D1B793E747002302FC008D
:104FA80001CC1C484146A2852324FC0213058C0130
:104FB80097B0FB1FE780402663910B02D5D80325E5
:104FC800CC0209C597B0FB1FE7808015F1452685FF
:104FD800EFC01FFA2326AC0261BFE30B09F80325D3
:104FE800CC0209C597B0FB1FE7808013F1454A85BD
:104FF800C5B79DC483A70B0299EB9165938535715D
:10500800714597B0FB1FE780600323A0AB0203A59F
:105018000B0219C57146A68597B0FB1FE780C01F14
:105028006388090283A74B0299EB916593852571E3
:105038005D4597B0FB1FE780600023A2AB0203A584
:105048004B0219C55D46CE8597B0FB1FE780C01C93
:105058001DC483A78B0299EB916593851571514502
:1050680097B0FB1FE78080FD23A4AB0203A58B024A
:1050780019C55146A28597B0FB1FE780E019225455
:10508800B2509254F249B24B224CCA865A860259FF
:10509800424BD6855285D24A624A45616FF0EFEAA3
:1050A800011126CA52C406CE22CC4AC84EC62A8A44
:1050B800AE84EF90800C25C5AA893945EFC05FBB47
:1050C8002A8431CDB727002003C987BE631409009D
:1050D80003C909009307000D2310F400AD4723010D
:1050E800F4009385690013053400194697B0FB1F37
:1050F800E780801293F71400858085882306F400E2
:10510800A306940023154401A2856244F240D244C8
:10511800B249224A4A85424905616FC07FC4F240BC
:105128006244D2444249B249224A0561828001114F
:105138004EC652C456C206CE22CC26CA4AC8AA8A2D
:105148002E8AB289EF9060032DCD2A891305C002FB
:10515800EFC01FB22A8435C5B727002083C487BE95
:1051680099E0834409009307000D2310F400E947F0
:105178002301F4009305690013053400194697B01C
:10518800FB1FE7806009D285231554011305C4006D
:10519800414697B0FB1FE7802008CE851305C40160
:1051A800414697B0FB1FE7802007A2856244F24082
:1051B8004249B249224A924A2685D24405616FC0C3
:1051C8003FBAF2406244D2444249B249224A924A22
:1051D80005618280411122C4372400201304049AF7
:1051E800084006C619C597B0FB1FE78060F3232067
:1051F8000400B240224441018280011106CE22CC33
:1052080026CA4AC82EC6EF80507739CDB245B7278F
:10521800002003C987BE0CD5AA846314090003497A
:1052280005004145EFC0DFA42A841DCD9307000D7A
:105238002310F500A5472301F50083C75400938583
:1052480064001105A30FF5FE194697B0FB1FE78010
:10525800A0FC9C54A285F2405CC46244D2444A85B6
:10526800424905616FC0DFAFF2406244D24442490F
:10527800056182801D71A2CC86CE2A842EC6EF805D
:10528800D06F05CD8346C5001147AA87494563926B
:10529800E6029C5FB24599C383C56701B70605005E
:1052A8002308B10093862648100889452285EF9087
:1052B8002074F6406644256182805145DDBFB727DA
:1052C800002083C7C7CF0547FD1793F7F70F637A09
:1052D800F704894721CA411122C426C24AC006C61A
:1052E800B2842E89EF8070692A84D14705C5630886
:1052F80009008347450093E727002302F50041464C
:10530800A6851305840197B0FB1FE780E0F09C4851
:105318001CD48147B2402244924402493E8541014F
:105328008280C9473E858280797122D406D62A8434
:105338002EC6EF80906401CDB2452285230EB100C0
:105348006C08EF90A070B25022544561828051459C
:10535800DDBF6F803079C1671387E7FF6395E5028A
:10536800B727002083A7C79A91EB49458280494512
:10537800B2402244924402494101828003A30700BB
:10538800E30503FE0283411122C426C24AC006C6B1
:10539800FD172A892E84B284639AF502B727002064
:1053A80083A7C79A91CF9C4381CF829711E9B727EA
:1053B80000202380279DB7270020A380979C4DBFFE
:1053C800A6854A85EFE07FD145F5D5B72E85EF80D4
:1053D800D05A51DD834705000D45E39B27F9228507
:1053E8002244B2400249A685924441016FD000424E
:1053F8009307000463E2A7064111C16722C406C6E9
:1054080026C2FD172A8409456382F502C547AE8482
:105418006313F4022E85EFD02047372500201305AB
:1054280085BB06042A94231094000145B240224407
:105438009244410182809307A0036316F4002E85ED
:10544800EFD0803DD9BF9307B003E318F4FC13F500
:10545800F50FEFD0A03CD1B709458280011106CEE7
:105468002AC6EFE0BFC9EF202074EF101015EF60D7
:10547800224BB7270020938787B9130700F02391A1
:10548800E70023820700B72700203245138787CF1C
:10549800FD562301D700F240238CA7CE9545056120
:1054A8006F70C058597193970501CAD086D6A2D497
:1054B800A6D2CECED2CCD6CADAC8DEC6E2C4E6C2FE
:1054C800EAC06EDEC1872E8963D40756B724002050
:1054D80003C584CFB7290020372B0020EFC05F8099
:1054E8002A8426CCB72A0020372C0020938489B937
:1054F800B72C00201DE021653345A900B65026547D
:1055080096540659F649664AD64A464BB64B264C37
:10551800964C064DF25D656182808347040013074F
:10552800200A639CE70003CA340003552400C165C0
:105538002286FD15EFF08F918DA26247130787CF62
:10554800034A2700130710096395E71683471400D9
:105558001547639FE7002285EFF00F942285EFC07F
:105568000FECE24703C587CFEFC08FF72A8459B7FE
:1055780039476398E716035544008567A5076315FF
:10558800F5040C4483CB0500639D0B00850591C988
:10559800372500201946130505BB97B0FB1FE78088
:1055A800A0C703C789B985476315F71063880B003F
:1055B800238C09B85E85EFF04FC24DB78947238C1D
:1055C800F9B8EFD0602759BF896713872700631C94
:1055D800E504832B8400638E0B0C83C70B0089EFD3
:1055E80083C72B0003C71B00A207D98F2394F4009D
:1055F80083C73B00A380F40003C789B98947631AAE
:10560800F70A83C70B0091C7238C09B803C50B00A1
:105618005DB783C5140003D584008D47238CF9B882
:10562800EF70C043E5B795076318F5001C4403C540
:105638000700EFF00FE41DB7F9771387A7FF2A9744
:1056480042074183914663F1E6049387A7FCAA9732
:10565800C207C18371476371F70289671387B7006F
:105668006310E50483A78A9AE38A07EE9C43A28520
:10567800E38607EE829715A0370700181307F7701F
:10568800B357F700858BA1CB83270B9BE38807ECE7
:105698009C43E38507EC22858297E31105EC11A86A
:1056A8001387C7006310E5021C4483C70700E3871C
:1056B80007EA9307F00FE303FAEAA2855285EFC0E1
:1056C8002FEA45B5B9076318F50083A7CC9AE38795
:1056D80007E8DC4369BF896793871704E304F5F893
:1056E800C9BF3D476399E704035544008967138799
:1056F800D700E30CE5FC13879701E308E5FCCD0729
:10570800E319F5FA03D76400C167FD17631DF700B5
:1057180083A7CC9AE38407E4DC43E38107E40965C3
:10572800A2854D0581BFB727002083A7479BE38744
:1057380007E29C43DDB71307E003E39CE7F68347E2
:10574800240005476398E70E834764003727002045
:10575800930D079AE1E783A70D00D5CF83CB070008
:10576800214A03457400130D8400EA85EFE01FE029
:1057780083474401A303A400835804010358E400A9
:10578800035744002A86034534003EC28357240148
:10579800EA86DE853EC0D287EFF0CFBC834734006F
:1057A80095E7DD47835804010358E40083467400F5
:1057B800835544003EC2835724016A873EC0D2877E
:1057C80005465E85EF805054A301A40083A70D0011
:1057D80081C71145EFF01FA0930B0C9C03C50B006C
:1057E800E30E05D6B727002083C5179CEFE0FF8E90
:1057F800E30605D68346340093071003638AF60050
:105808000356440083C50B0052873685EFE05FA737
:1058180023000C9CA1B383CB340099B783270B9B3F
:1058280083CB3400114A95DFDC4385DF8145014590
:10583800829705BF29476398E70A8347640037279B
:105848000020930D079AA5EF83A70D00B5C783CB5A
:105858000700214A034574009306840093772500C6
:10586800BDCB137615001303440183470402835804
:10587800C4010358A40103574400034534003EC241
:105888008357E401DE851ACE3EC0D287EFF08FAD94
:105898008347340072439DFBDD478358C401035896
:1058A800A40183467400835544003EC28357E40133
:1058B8001A873EC0D28729B783CB340059BF8327C4
:1058C8000B9B83CB3400114AD1D7DC43C1D7814528
:1058D8000145829741B7B68536CEEFE03FC9F2461B
:1058E8002A86368359B70947639CE70083A78A9AB3
:1058F800E38607C6DC43E38307C622858297B9B9E6
:105908002D476398E70083A78A9AE38907C49C47D1
:10591800DDB70D476397E70022868D4503554400A0
:1059280011B919476395E70693056102130510310C
:10593800EF60A2072C1013052031EF600207035611
:105948006400835781020355440063E8C700835607
:1059580084000357610263F7E60093050002EFC075
:10596800B071EDBE6374E6002313E40063F4D7005E
:105978002314F4000357C4008356A400035684007C
:105988008355640001488147EFC0D06EC1BE1D47F2
:10599800E381E7D231476395E7002286B145BDBF71
:1059A80035476398E70083A78A9AE38907BADC47F3
:1059B80099B739476396E7002285EF00F00779BE6B
:1059C8003D476398E70083A78A9AE38907B89C4B09
:1059D8001DB741476396E7002285EF001011BDBE51
:1059E80045476396E7000145EF00902085BE49478B
:1059F800639DE70083270B9BE38D07CADC43E38A9B
:105A080007CA8145054582976DB14D47639CE700FC
:105A180083270B9BE38F07C8DC43E38C07C8A28569
:105A28000945D5B76147E396E7C82286E145FDB544
:105A380093F7150089CFB727002083A7879A89C7CE
:105A4800DC4399C3014582971345190045BC93F778
:105A5800250091CFB727002083A7079B91C7DC4378
:105A680081C78145054582971345290041BC93F7B5
:105A780045000145E38407A8B727002083A7479A74
:105A880037240020130484B991CF85472302F400FA
:105A9800B727002083A7079B91C7DC4381C78145AF
:105AA8000545829748442C10EF90806B2810EFF042
:105AB8002F97B727002083D7A7BD81CF130600648F
:105AC8003386C702B727002003C587CF9145EFC0AB
:105AD800BF82134549001DB4011122CC2A845545C3
:105AE80006CE26CAEFF02FBBAA8413054002EFF0BA
:105AF8008FBA2AC613055002EFF0EFB9AA8622859D
:105B080062443246F240B3359000D24405616FC01A
:105B1800105D797122D406D68D472E84631FF50057
:105B280003D7A50083D6850003D665000345340056
:105B380083D54500EFE05FF209A889671387D7008E
:105B48006311E50403C5250019E58547B2502254C1
:105B58003E8545618280B727002083A6079AF5D63F
:105B680003C6360083C50600814802C202C0014848
:105B7800814701479106EFE0FFFE0545EFF08FE50D
:105B8800E9B71387E700E302E5FC13873701631AD7
:105B9800E50003C5250055D90147814601468145E1
:105BA80051BFE507E303F5FAB1476319F500B727D5
:105BB800002003C5B7B9EFE07FF541BF41677D1706
:105BC8008147E315E5F803C75500C947E31FF7F612
:105BD80083D6E50003D6C5000355840083D5A50008
:105BE800EFC0705641C95D45EFF0EFAA3335A0000C
:105BF800231CA10083454400035524003008EF808E
:105C0800004883578101B1F36C0813051031EF5038
:105C1800D2599305E10113052031EF5012598357EA
:105C2800C101035784006374F7002314F4008357F9
:105C3800E1010357A40063F4E7002315F400835738
:105C480084000357A4006374F7002315F400035578
:105C58002400EF4091160357E4008356C40003560E
:105C6800A400835584000355240001488147EFC0F0
:105C7800303EE1BD8547231CF100ADBFB7270020AA
:105C8800138787CF834677001307F00F638CE608E6
:105C980051C9411122C426C24AC006C6AA84034576
:105CA800A500138987CF4105EFB09FFC2A842DC535
:105CB8009307000D2310F500D9472301F50083D77A
:105CC80044002312F50083C764002303F50083C74B
:105CD8007400A303F50083C784002304F50083C779
:105CE8009400A304F50003C6A4002305C50015C24B
:105CF800CC44410548C497A0FB1FE780E051A2852A
:105D0800224403457900B2409244024941016FC0E0
:105D18002F8523260500E5B7B24022449244024964
:105D2800410182808280C1671387E7FF639EE50097
:105D3800B727002083A7079A9DC383C707000D478D
:105D4800639DA7006FC01030FD1749476397F500A2
:105D5800B727002083A7079AF5F73A858280494735
:105D6800EDBF397122DC06DE26DA4AD84ED652D487
:105D780056D25AD05ECE62CC0347050085472A84A6
:105D8800630DF70403468500930695009305E1002B
:105D98000545EFE06FE1814719C183470500834658
:105DA800040011476383E604372700200327479C34
:105DB8008D4603471700630AD70285CB1DC70DE13F
:105DC8000145F2506254D2544259B259225A925A59
:105DD800025BF24B624C2161828081470145C1B769
:105DE80085466314D70A8D8BE1DF03451400130A37
:105DF8002400D285EFE08FF737290020A300A40004
:105E08008327899C2A8B1309899C8149C1C7B72A92
:105E180000209304F00F83C72A9C138C2A9C63FDEF
:105E2800F90203250900939B49005E958347050005
:105E38006384970683471500639067071946D285E0
:105E4800090597A0FB1FE780604A39C5832409002C
:105E580003470400DE94B9E4834604009147E381D4
:105E6800F6F683270900A9DF03460C0001479305CE
:105E7800F00FE307E6F4BE84C10703C507FF630913
:105E8800B50C05071377F70FEDB78946E31AD7F274
:105E9800858B99BF054535B7850993F9F90FA5BFD6
:105EA80088C4F5A09147631AF706C84405C5834717
:105EB8008400034605006304F6060347040091477F
:105EC800631DF706C84419C597A0FB1FE780402546
:105ED80023A604000345840091659385E5710505B3
:105EE80097A0FB1FE780801505C50347040091476D
:105EF800631EF704C8C4834784009305940005050E
:105F0800A30FF5FE0346840097A0FB1FE780C0306F
:105F1800034584003335A0006DB5884441BF93051F
:105F28009400050597A0FB1FE780403C8547E316D2
:105F3800F5F85545EFE03FF6BDA8884441DD97A048
:105F4800FB1FE780E01D23A4040069B788C465B778
:105F58002380D40083471400D28513852400A380AE
:105F6800F400194697A0FB1FE780002B0345840027
:105F780091659385F571050597A0FB1FE780000CD7
:105F880005C5034704009147E31CF7F0C8C48347DD
:105F98008400930594000505A30FF5FE03468400CD
:105FA80097A0FB1FE780402783478400E39407EE10
:105FB800034504007D151335150021B5397122DC20
:105FC80026DA4ED652D406DE4AD856D25AD05ECEFB
:105FD8002A849309250003451500CE85B72400209F
:105FE800EFE0CFD8A300A4009384449C9C400D47C5
:105FF8002A8A83C717006390E7043729002083277C
:10600800899C814A1309899C638E0714B72B002049
:1060180003C72B9C93970A01C18303250900138B9F
:106028002B9C63E7E70C83460B0003270900814795
:106038001306F00F79AAF1D3144C034674019305A3
:10604800E1000545EFE04FB605CD9840854683470A
:106058000500034717006310D7028D8BD9FF014550
:10606800F2506254D2544259B259225A925A025B9F
:10607800F24B216182808946858BE310D7F8F9BFFE
:106088008347040011476385E7002D47E399E7FC40
:10609800B724002083A7849C9384849CE9D3814AF5
:1060A8000149B72B00201DA88840139B4A0083474D
:1060B80004005A95034705006311F702834715004A
:1060C800639D47011946CE85090597A0FB1FE78008
:1060D800E02101C503A904005A99850A03C72B9C2E
:1060E80093970A01C183E3E1E7FCE31809F085BF50
:1060F80093944A0026950347050083470400631FCD
:10610800F70A83471500639B470B1946CE85090597
:1061180097A0FB1FE780801D55C183270900114701
:10612800BE94834704006385E7002D47639EE7021A
:1061380003AAC4008347740103460A006309F602F0
:10614800528597A0FB1FE780A0FD03457401916568
:106158009385E571050597A0FB1FE78020EE1DE5F7
:10616800E38304EC0545EDBD03AA8400E1B70C4CBC
:1061780013051A0097A0FB1FE78040178547E31116
:10618800F5FC5545EFE03FD161DDD1BD8347040003
:1061980011476385E7002D476390E702C8C483472A
:1061A80074010505A30FF5FE034674010C4C97A076
:1061B800FB1FE78060066DB788C4D5B7850A89BD1F
:1061C800BA844107834507FF638AC5008507C2076C
:1061D800C183E3E7D7FE79B788C491A08347040059
:1061E800CE85138524002380F400834714001946C4
:1061F800A380F40097A0FB1FE78000020345740109
:1062080091659385F571050597A0FB1FE78000E36D
:1062180031D9034704009147E310F7FCC8C483470A
:1062280074010505A30FF5FE034674010C4C97A0F5
:10623800FB1FE78060FE3DB701114AC837290020DF
:10624800130989CF0347790006CE22CC26CA4EC649
:106258009307F00F6304F70851C1AA845145EFB0C2
:106268003FA12A8425CD9307000D2310F500D547BB
:106278002301F50083C7340093898400CE85A301E8
:10628800F50083D744002312F50083C76400230375
:10629800F50003C57400EFE06FADA303A400CE853D
:1062A80013058400194697A0FB1FE780E0F683C713
:1062B800E400A285034579002307F40083D704018D
:1062C8002318F40083C724012309F4006244F24030
:1062D800D2444249B24905616FB09FA8F240624476
:1062E800D2444249B24905618280411122C437240F
:1062F8000020130484CF0347740006C626C2930700
:10630800F00F630CF70215C9AA841945EFB05F9620
:10631800AA8505C59307000D2310F500DD47230165
:10632800F50083D74400B24092442312F500034598
:106338007400224441016FB0BFA2B240224492448B
:1063480041018280011122CC372400208327849CBC
:1063580006CE26CA4AC84EC652C48DC31304849CAE
:106368002E8AAA840149084063129902630C0A0420
:1063780097A0FB1FE780C0DA23200400F2406244A4
:10638800D2444249B249224A0561828093194900A0
:10639800B3073501884709C997A0FB1FE78040D894
:1063A8001C40CE9723A407001C40CE97C84709C9B4
:1063B80097A0FB1FE780C0D61C40BE9923A6090002
:1063C800050955B745DD13964400814597A0FB1F85
:1063D800E780A0EB144081477D5613F7F70FE37F62
:1063E80097F81397470036972300C7008507F5B736
:1063F80079714AD0372900208327499C06D622D4B0
:1064080026D24ECE52CC56CA5AC85EC6C5C7B72A7F
:106418000020AA891309499C938A2A9C014405E112
:10642800B727002083A6879C99CA03C60A002A8436
:1064380081479305F00F13F7F70F6368C708131523
:1064480034002105EFB0DF82AA8401E92145EFB0CD
:106458003F82AA8421C50144CD49930700FD2380CA
:10646800F4008547A38034012381F400A3818400CC
:1064780045C89389840023A23401014A372B0020A0
:10648800930BF00F83C70A006373FA0039E8832778
:106498000900A68503C50700EFB09F8C03C50A0055
:1064A80081454D350325090097A0FB1FE78040C7AC
:1064B80023200900B250225492540259F249624AE8
:1064C800D24A424BB24B45618280139747003697B8
:1064D800034707006305B70005041374F40F850725
:1064E80099BF83278B9C93154A00BE9583C70500E7
:1064F800638477032380F90083C715001385290077
:106508007D14A380F900194689051374F40F97A028
:10651800FB1FE78060D0A109050A137AFA0F9DB71F
:1065280023A20400ADB7B727002083A7479CB1C7B3
:10653800411122C406C62A841DE10945EFE0BF9532
:106548002A8601C9B727002003C587CF8545EFB044
:10655800BFDA0545EFF04FD82A84054519C8B72793
:10656800002003C587CF8545EFC0CF8122854935F7
:106578000545B240224441018280014582808967F5
:106588009386B7006316D5009C4503C5070061BF15
:106598009386C7006318D5009C45854603C5070048
:1065A80019C9F5B793861704E300D5FE9387270426
:1065B8008146E303F5FE36858280797106D622D4BA
:1065C80026D24AD04ECE52CC56CA5AC85EC662C4EB
:1065D80071CD83473500AA8985C7404115C0594503
:1065E800EFE07F8B931A850193DA8A410149372AB4
:1065F8000020130B000DB54B83C73900636EF900FB
:10660800B250225492540259F249624AD24A424B39
:10661800B24B224C456182808307840263CF5707BF
:1066280083274A9C130C4A9CADCB2285EFF06FF36D
:106638002DC5034584005105EFB08FE3AA8431CD01
:10664800231065012301750183470400194693054A
:106658002400A301F5008307840215052303F50030
:1066680083471400A30FF5FE97A0FB1FE780C0BA6D
:10667800034684002386C4001DC61385440188C8C8
:106688009305940097A0FB1FE78000B983270C00AF
:10669800A68503C50700EFB0AFEC05091304940203
:1066A8001379F90F91BF23A80400CDB7B7270020AD
:1066B80083A7479CB1D72D3B2254B250925402591C
:1066C800F249624AD24A424BB24B224C01454561DB
:1066D8006FF08FC0797106D622D426D24AD04ECE1A
:1066E80052CC56CA5AC85EC662C469C583473500CB
:1066F800AA8985C7444195C05945EFE0CFF9931A57
:10670800850193DA8A410149372B0020930B00FD5C
:10671800414C83C73900636EF900B2502254925439
:106728000259F249624AD24A424BB24B224C456165
:1067380082808387F40063CA5707130A4B9C832718
:106748000A00A5C75145EFB0AFD22A8439CD23003E
:106758007501A30005002301850183C704001946BC
:1067680093852400A301F5008387F4001505A3068B
:10677800F50083C71400A30FF5FE97A0FB1FE78061
:10678800A0A983C78400938594001305C400A305BA
:10679800F400194697A0FB1FE78000A883270A008A
:1067A800A28503C50700EFB0AFDB0509C104137963
:1067B800F90F85B7B727002083A7479CB9DFEFF00B
:1067C8003FC32254B25092540259F249624AD24A03
:1067D800424BB24B224C014545616FF0EFAF5D7102
:1067E80086C6A2C4A6C2CAC04EDE52DC56DA5AD841
:1067F8005ED662D466D26AD06ECE6301052883471E
:106808003500AA8495CB832A450063870A02594537
:10681800EFE06FE893178501E1873EC60144B72989
:106828000020130A000D054CB54C130D00FDC14D99
:1068380003C734006361E402B6402644964406491F
:10684800F259625AD25A425BB25B225C925C025D98
:10685800F24D616182800387CA00B2476349F71627
:1068680003A7499C1389499C6303071683CB0A0035
:1068780013F70B014DCF4D47639EEB0623800A00AB
:106888005685EFF0AFF36304051403C70A00914778
:1068980063E4E7146319870D5145EFB06FBD2A8B88
:1068A800630705122300A501A30005002301B50114
:1068B80083C60A00194693852A00A301D50083865A
:1068C800CA001505A306D50083C61A00A30FD5FE76
:1068D80097A0FB1FE780409483C60A011946938559
:1068E8001A01A305DB001305CB0097A0FB1FE78067
:1068F800A092F9A055476398EB0005472380EA006A
:10690800A38B0A00B5BF7547E389EBFE4947639639
:10691800EB0009472380EA00A5B741476394EB00E1
:106928000D47CDBF6D47E39DEBF41147E5B713F76E
:106938008B0019C32D47F9BF13F61B0013F74B0043
:1069480011C619C315475DBF2147E9B713F62B00D8
:1069580011C619C325475DB719476DBF19C3294724
:1069680055BF1D4745BF03C57A015105EFB04FB06C
:106978002A8B31CD231045012301950183C60A00D6
:10698800194693852A00A301D5008386CA001505F8
:106998002303D50083C61A00A30FD5FE97A0FB1FBB
:1069A800E780808703C67A012306CB0001CA130556
:1069B8004B012328AB0083A58A0105BF23280B00C0
:1069C80083260900DA8503C50600EFB06FB9050410
:1069D800F10A1374F40FA9BD03C57A011305050262
:1069E800EFB00FA92A8B65D5C9472301F5002310FD
:1069F800450103C60A0093F60B0693852A00D18E3B
:106A0800A301D50083C61A0019461505A30FD5FEA4
:106A180097A0FB1FE780408083C68A0019469385AC
:106A28001A01A305DB0083C69A0013053B01230660
:106A3800DB0083C6AA00A306DB0083C6BA002307CF
:106A4800DB008386CA00A307DB0083D6EA0023188D
:106A5800DB0083C60A012309DB009790FB1FE78050
:106A6800A07B03C67A01A30CCB0011C613050B0249
:106A7800232EAB0089B7232E0B0099B7B727002028
:106A880083A7479CE38A07DAEFF09F962644B6402F
:106A980096440649F259625AD25A425BB25B225C6A
:106AA800925C025DF24D014561616FF0EF82B7279C
:106AB800002083A7479C85CB03C707008D47631534
:106AC800A702B727002003C587CF4111854506C611
:106AD800EFB05FAB13050003EFF09F91B2400145A3
:106AE80041016FE07FFFC9473E85828079714AD0B6
:106AF800372900201309499C8327090006D622D488
:106B080026D2F9E337240020130484CF0347440036
:106B1800C947298B5DC39165AA849385D5711145B1
:106B28009790FB1FE78080512320A900CD4751C5CE
:106B3800034774009307F00F6316F70083C7040038
:106B4800A303F4001146A6859790FB1FE780C06C4D
:106B5800930531011305F041EF30A225B727002036
:106B6800938787B903C42700034731013334800072
:106B780011C3090413051002EFE0EFB11376F50F06
:106B880013771600E14715CB154532C6EFE0AFB0D5
:106B980083C72400231CA1001945230AF100EFE054
:106BA8008FAF324683C53400231EA1007C08380805
:106BB80054082285EFB07052AA87B25022549254DA
:106BC80002593E8545618280C547C5BF757126C398
:106BD800B724002022C506C74AC1CEDE938484CFDD
:106BE80083C744004944A18B638D0718B727002049
:106BF80083A7479C4144639607182A89EFE06FF5FD
:106C080083C784005544637EF516B724002083A704
:106C1800049AA68945446396071691659385C571BC
:106C280029459790FB1FE780604123A0A49A4D4413
:106C3800630905142946CA859790FB1FE780C05D44
:106C480013056002EFE02FA51375F50F9377150074
:106C58006144638807121306000381451364250005
:106C680088009790FB1FE78040624145EFE0AFA2A4
:106C78002316A1043D45EFE00FA22319A1043545D1
:106C8800EFE06FA1231CA1043945EFE0CFA0231F3B
:106C9800A1042145EFE02FA02312A1061D45EFE036
:106CA8008F9F83A7049A2315A10683C717006382C1
:106CB800070E2D45EFE02F9E2310A1043145EFE08C
:106CC8008F9D2313A1041305C002EFE0CF9C231767
:106CD800A1041305B002EFE00F9C231AA1041305C9
:106CE8009002EFE04F9B231DA1041305A002EFE0E3
:106CF8008F9A2310A10613058002EFE0CF99231382
:106D0800A10613057002EFE00F9983A7099A2316CD
:106D1800A10603C5370093854700EFD0BF802AD668
:106D28009305F1031305F041EF30A208B7270020BF
:106D3800938787B983C527000347F1033256B335D4
:106D4800B00011C3890583A6099AFC00228703C5F0
:106D580026003EC8930721053EC6BC083EC49307DB
:106D6800E1053EC2DC103EC09308A1061308610489
:106D78009C009106EFB0F0362A8401C50D45EFE07E
:106D88006FC52285BA402A449A440A49F65949618E
:106D980082802545EFE02F902310A104294505B7EF
:106DA800B727002083C7C7CF0145A18B89C73725DF
:106DB8000020130505C56FD0CFD2B72700207D5717
:106DC8002381079CB7270020A38FE7CEB727002091
:106DD80023A4079C37670400B727002013076758C8
:106DE80023A2079CB727002023AEE7C23767040019
:106DF8009387C7C31307275CD8C3376704001307F3
:106E0800C76D98C7376704001307677ED8C7376709
:106E18000400130747C898CB37670400B72700203A
:106E28001307E7D223A8E7C437670400938707C589
:106E38001307A7B1D8C38280411122C43724002088
:106E48001304249C26C2AA8403450400854506C66B
:106E5800EFF04FCFB727002083C7C7CFA98BA5CFA7
:106E680037250020230094001305C5C3B72400204C
:106E7800EFD08FC69384849C9C4099C74D45B240FF
:106E880022449244410182800345040019E10145EE
:106E9800FDB791659385B57112059790FB1FE78043
:106EA800E01988C061DD0346040081451206979009
:106EB800FB1FE780803D8346040090408147FD55D5
:106EC80013F7F70FE375D7FC1397470032972300A2
:106ED800B7008507F5B7014523000400EFD0CFBF01
:106EE8007DB7411122C4372400200325449A06C6E1
:106EF80019C59790FB1FE780A0222322049AB2406D
:106F080022444101828001111305700306CEEFD09F
:106F18009FF82AC613058003EFD0FFF72AC413058C
:106F28009003EFD05FF72246B245F240AA860545A6
:106F380005616FB0D0195D711305D00386C6A2C470
:106F4800A6C2CAC0EFD03FF52A841305C003EFD00C
:106F58009FF4AA841305E003EFD0FFF32A891305F1
:106F6800F003EFD05FF38A871377F50F9376F90F65
:106F780013F6F40F9375F40F0545EFB09017B6406C
:106F8800264496440649616182805971A2D4372407
:106F980000208327449A86D6A6D2CAD0CECED2CC99
:106FA800D6CADAC80545638D070C9305F1041305A5
:106FB800F041EF2012609305F1041305F041EF2032
:106FC800525FB7270020938787B983C727000347F5
:106FD800F104B337F00011C389070327449A3EDE52
:106FE8000345370093054700EFD0CFD30327449AD2
:106FF8002ADC0D45834527002EDAEFD0DFE92AD8B1
:107008001145EFD05FE90324449A2AD66545034722
:10701800A400034BB4003AD4EFD0FFE7AA84694533
:10702800EFD07FE72A897145EFD0FFE6AA896D4541
:10703800EFD07FE62A8A7545EFD0FFE5AA8A794521
:10704800EFD07FE5E2046258F2572257B256425613
:10705800D2551375F50F93FAFA0F137AFA0F93F9BD
:10706800F90F1379F90FE1842ACC56CA52C84EC6D3
:107078004AC426C25AC0930844000545EFB090019F
:10708800B650265496540659F649664AD64A464B8F
:1070980065618280011122CC06CE26CA8D472E84D6
:1070A8006315F50603C73500B7240020E94703D563
:1070B8004500938484B96316F70083D7640063821C
:1070C800A706EF70800B09C5835764002317F500E6
:1070D8000357A40083568400035664008355440074
:1070E80003453400EFD05F970357440083D764000B
:1070F8006309F7008547F2406244D2443E85056142
:107108008280FD572393F400F5B78967CD07631D87
:10711800F50083C7250031476385E7004547E39BB2
:10712800E7FCEFD04FA3F9B7B1476319F500B727CC
:10713800002003C5D7CFEFD07F9D6DBF41677D1776
:107148008147E31AE5FA83C655004947E395E6FA0D
:1071580083C5450003552400300023140100EF6067
:10716800F06C49BF411122C4372400208347C49CD6
:1071780026C206C64AC01307E00FAE846386E7043A
:107188001307F00F1304C49C6387E7021145EFA0AF
:107198003FAE15C1930700FD2300F5008947230181
:1071A800F5008547A3009500A301F500AA850345CE
:1071B8000400EFA0FFBAF9572300F400B2402244BC
:1071C80092440249410182802A891145EFA05FAAB1
:1071D80075D5930700FD2300F50089472301F500C5
:1071E800A3009500A30125012244B7270020B2403F
:1071F80092440249AA8503C5D79C41016FA05FB696
:1072080079714AD0372900208327499A22D406D693
:1072180026D24ECE52CC56CA4544D5EFB7240020CC
:10722800938784CF83C747004944958BCDC7B72739
:1072380000202E8A9165A386A79CAA8993857571DB
:1072480031459790FB1FE78060DF2322A99A4D44C0
:1072580059C123003501A30005002946D285090537
:107268009790FB1FE78040FB8327499A914603C705
:10727800270063EDE60835EB4D472381E70003C798
:107288002700136707012381E700930571001305A1
:10729800F041EF20123283477100F1EBB72700204D
:1072A80003C7A7B98D476314F70CEFD0EFB52C00CF
:1072B800EF70106B2800EFD0BF964545EFD0BFBDEB
:1072C800014411C9130600643306C50203C584CFFF
:1072D8009145EFB06F822285B250225492540259E0
:1072E800F249624AD24A4561828085466314D700D2
:1072F800754761B789466314D7004947BDBF8D46B6
:107308006314D700414795BF554785BF9546CA8A3C
:10731800630ED70099466316D70009472381E70013
:1073280031A01D466314C702238107006545EFD0CD
:107338009FB69307F007E30AF5F403A74A9A834731
:10734800270093E707042301F70081B72146631458
:10735800C7000547E1B725466315C7002381D70055
:10736800F1B7A9460544E318D7F6114745BFEFF032
:10737800DFC12A842DD1EFF0DFB6B1BF011126CAD3
:10738800B724002083A7449A22CC06CE4AC8494491
:10739800B1C783C707000D446392A70437290020AB
:1073A800034589CF8945EFB0EF9D034589CFB727BE
:1073B800002091452398079CEFB0CF9C83A7449A5F
:1073C80001478146A38087001306F100854785455C
:1073D8000145A307F100EFB0404F2A842285F2400F
:1073E8006244D244424905618280011106CE22CC12
:1073F80026CA4AC88547631EF506372400201304A9
:10740800049D83570400A9CB372700200347C7B939
:1074180021E71307B003636CF702B724002003C504
:1074280084CF8945EFB00F96035604009307006494
:1074380003C584CF3306F6028945EFA0FFEB23107E
:107448000400F2406244D244424905618280938735
:1074580047FC2310F400F5B7B727002083A7479A05
:10746800EDD36244F240D244424903C507000561A6
:1074780031B7B724002083A7449AE1D737270020E3
:10748800130987CF83474900918BC5DF8947631369
:10749800F5062D452EC6EFA0AFFD2A845DD1B24575
:1074A800930700FD2300F500E547A300050023012D
:1074B800F50083C7350015051946230FF5FE83C768
:1074C80045009505A30FF5FE9790FB1FE780C0D4F4
:1074D800034559009307F00F6316F50083A7449AF4
:1074E80003C50700A2856244F240D24442490561BF
:1074F8006FA01F87034587CF8945EFB0AF886244E7
:10750800F240D2444249B72700202398079C0561DE
:107518006FF03F9DB727002083C7C7CF958B89CFD2
:10752800B727002083A7C79D91CBB7270020054721
:10753800238CE7C46FF03F9D494582804145828096
:10754800B727002085450145238C07C46FB0A038B4
:10755800B727002083C7C7CF958B81CBB7270020DB
:1075680005472387E79C6FF01F9D49458280B72711
:107578000020814505452387079C6FB0C037B72792
:10758800002083C7C7CF958B638F07129307C01C52
:1075980063FCC70009458280F2406244D2444249F4
:1075A800B249094505618280B727002083A7479A19
:1075B800638B0710B72700209387C79C03C8070071
:1075C8001307E00F6311E810011122CC4AC806CE58
:1075D80026CA4EC62380A7001305860042053689B1
:1075E80032844181ADC99165938565719790FB1F80
:1075F800E780C0A4AA894DD1B724002003A5849DA3
:107608009384849D09C59790FB1FE78060B113851B
:10761800890023A0A9002286814523A034019790E0
:10762800FB1FE78080C69C402286CA8588439790C6
:10763800FB1FE78060BE9C40A286F2402392870031
:107648006244D2444249B249984305468D450545AE
:1076580005616FB000279165938555719790FB1F61
:10766800E780C09DAA890DD9B724002003A5049EF0
:107678009384049E09C59790FB1FE78060AA138531
:10768800890023A0A9002286814523A03401979070
:10769800FB1FE78080BF9C402286CA85884397905D
:1076A800FB1FE78060B79C40A286F24023928700C8
:1076B8006244D2444249B249984305468D4505453E
:1076C80005616FB04020494582809307C01C63FC68
:1076D800A700094582800945F2406244D2444249E4
:1076E800B2490561828045CD011122CC2A84210549
:1076F8004EC64205AE8991659385657141814AC838
:1077080006CE26CA9790FB1FE78040932A8961D549
:10771800B724002003A5849D9384849D09C5979070
:10772800FB1FE780E09F130589002320A90022861C
:10773800814523A024019790FB1FE78000B59C405A
:107748002286CE8588439790FB1FE780E0AC9C405B
:1077580023928700B727002083A7479A8DCFB727A2
:10776800002083C7C7CF958B8DCBB727002083A771
:10777800879D99CF984383D647006244F240D2440C
:107788004249B24905468D45054505616FB060130C
:1077980001478146DDB7014581B7494535BFB72760
:1077A800002083A7479A95C7B727002083C7C7CF6C
:1077B800958B95C3B727002083A7879D81CB9843D6
:1077C80083D6470005468D450545C9B7014781461B
:1077D800D5BF01458280494582809307C01C63FC60
:1077E800A700094582800945F2406244D2444249D3
:1077F800B2490561828045CD011122CC2A84210538
:107808004EC64205AE8991659385557141814AC836
:1078180006CE26CA9790FB1FE78040822A8961D549
:10782800B724002003A5049E9384049E09C597905D
:10783800FB1FE780E08E130589002320A90022861C
:10784800814523A024019790FB1FE78000A49C405A
:107858002286CE8588439790FB1FE780E09B9C405B
:1078680023928700B727002083A7479A8DCFB72791
:10787800002083C7C7CF958B8DCBB727002083A760
:10788800079E99CF984383D647006244F240D2447A
:107898004249B24905468D45054505616FB0A002CC
:1078A80001478146DDB7014581B7494535BFB7274F
:1078B800002083A7479A95C7B727002083C7C7CF5B
:1078C800958B95C3B727002083A7079E81CB984344
:1078D80083D6470005468D450545C9B7014781460A
:1078E800D5BF01458280494582809307C01C63F457
:1078F800A70009458280797122D44ECE06D626D2B9
:107908004AD0AE892A842DC1210591654205938507
:10791800757141819780FB1FE78040722A8909456C
:1079280063060908B724002003A5C49D9384C49D59
:1079380009C59780FB1FE780A07E130589002320D7
:10794800A9002286814523A024019790FB1FE78088
:10795800C0939C402286CE8588439790FB1FE78082
:10796800A08B9C4023928700B727002083A7479AC3
:1079780001458DCFB727002083C7C7CF4945958BD1
:1079880095C76C001305D030EF402202B24701457D
:1079980093F7070F81CFB727002083A7C79D8D4591
:1079A8000545944303D64700EFA0B072B250225465
:1079B80092540259F24945618280B727002083A773
:1079C800879D91CF03D647008C43411106C69790F7
:1079D800FB1FE7806084B240014541018280094570
:1079E8008280B727002083A7879D8DC7B7270020EF
:1079F80003A7079E894705C3035647000C43411157
:107A080006C69790FB1FE7802081B24081473E85DC
:107A18004101828089473E858280B727002083A75D
:107A2800879D8DC7B727002003A7C79D894705C332
:107A3800035647000C43411106C69780FB1FE78099
:107A4800A07DB24081473E854101828089473E85BD
:107A58008280797106D622D426D24AD04ECE52CC14
:107A68008D4763FCA7008944B250225426850259E9
:107A78009254F249624A45618280372900200347BF
:107A880089B9C144E312F7FE9307F5FF930989B951
:107A980093F7F70F8546AE842A8403CA2900130991
:107AA80089B963EAF6068DE199452800EFC05F853C
:107AB800B729002003C589CF914523018900EFA08C
:107AC8007FAC35E481444DB719468145280097803D
:107AD800FB1FE780807B19462C0026859790FB1FAB
:107AE800E780C08049F119469305F00F2800978078
:107AF800FB1FE780807919462C0026859780FB1F9D
:107B0800E780C07E2DF11946A68528009780FB1FC7
:107B1800E780807071BFE31DE5F803A5C9002C005C
:107B2800EF700064AA8449D52381490135BF280034
:107B3800EFD00F8FAA840DED930571001305F04166
:107B4800EF20222783447100B5FC8D47E31CF4F62F
:107B58004545EFD04FB43DD5B7771800938707A0B8
:107B68003306F50203C589CF9145EFA07F9AEDBD95
:107B780023014901D5BDB727002083C7C7CF918B03
:107B88008DC33725002041111305459D06C6EFC05A
:107B98008FF6B240B72700207D57239FE7B84101F1
:107BA800828001456FC02FF5B72700207D57A38637
:107BB800E79CB727002079572386E79CB727002042
:107BC800238C07C4B72700202387079CB7270020EA
:107BD8002398079CB727002023AC079CB7270020D1
:107BE80023A0079EB727002023AE079C37870400F1
:107BF800B7270020938707A8130747E298C337776A
:107C080004001307273FD8C337770400130727F961
:107C180098C7377704001307E7F0D8C73777040009
:107C28001307E7F398CBB77704003727002093872B
:107C3800C709232AF79C8280411126C2B724002055
:107C480083A7449A06C622C48DCF2A840D45EFA087
:107C58002F82AA8505C1930700FD2300F5008D47F3
:107C6800A30085002301F50083A7449A03C50700F4
:107C7800EFA00F8F19C42244B240924441016FF023
:107C88004FA6B2402244924441018280797152CC7D
:107C9800372A002083274A9A4AD006D622D426D2E9
:107CA8004ECE56CA0149B1C703C91700B7240020F0
:107CB8008547AA89938484B96307F90483C7440074
:107CC800054985EB0D45EF90BFFAAA8505C19307D5
:107CD80000FD2300F5009147A30035012301F500BD
:107CE80083274A9A03C50700EFA08F87EFF06F9F9D
:107CF8000549B25022544A8592540259F249624ABF
:107D0800D24A45618280B727002083A7879DD28AFF
:107D180085E30145EFD02F982A8601CAB7270020AE
:107D280003C587CF8945EFA02FDD83A74A9A81A88D
:107D3800944303D647009305E1000545EFC0CFE61D
:107D480069D983470500858BE9D70545EFD0AF94FE
:107D58009307B0032A8463F0A704B727002003C55C
:107D680087CF5D66130606708945EFA06FFAB727BF
:107D78000020130444FC2398879C83274A9A0947C8
:107D8800A380E70083C7440081C72382040095B716
:107D98004E855D35B9BF130600643306C502B5BF0D
:107DA800411122C42A840D4506C6EF907FEC05C513
:107DB800930700FD2300F500CD472301F500A3003C
:107DC80085002244B7270020B240AA8503C5D79C66
:107DD80041016F90FFF8B240224441018280411175
:107DE80022C42A840D4506C6EF909FE805C593076F
:107DF80000FD2300F500ED472301F500A3008500F1
:107E08002244B7270020B240AA8503C5D79C410168
:107E18006F901FF5B240224441018280035745000C
:107E28000111896606CE22CC26CA13866600AA8767
:107E38006317C7009C47014583C5070009A8138637
:107E48008600631AC7009C47054583C50700EFF005
:107E58006FB105453DA8138696006313C7023727FF
:107E680000200327479A01450DC79C4703C5070013
:107E780065E18547A300F7000545EFA0701CD1BF59
:107E88001386A600631CC7009C4703C50700EFF0D4
:107E9800FFDFF2406244D2440561828013866603A4
:107EA800E30AC7F813867603E30FC7F81386860339
:107EB8006313C70A1C45372400201307E00F83C447
:107EC80007008347C49C1304C49C638EE70213070E
:107ED800F00F6386E7021145EF909FD9AA8505C187
:107EE800930700FD2300F5008947A30095002301AF
:107EF800F500A301050003450400EF907FE6F9575C
:107F08002300F400B9B7B727002003A7479A3E8497
:107F1800014541D38DEC85447D4523059100EFC093
:107F28009FF72316A10013050002EFC0DFF6832791
:107F3800449AA305A1001307B100A3809700740019
:107F48001306A10085450545EFA0301819B7268509
:107F5800EFF09FCEFDBD13869603E307C7F21386A5
:107F6800E6036317C7001C45094583C50700C5B567
:107F78009386F603631DD7021C4503C5070035ED3C
:107F88006C001305D030EF305222B247414793F7C7
:107F9800070FE380E7EC9305B10013056031EF307C
:107FA800D2200345B1008545EFA0F0125DB5896682
:107FB800138606046316C7041C4503C40700B727C5
:107FC800002083C787C522858DEB0D45EF905FCADA
:107FD800AA85E30005E8930700FD2300F500D147D3
:107FE8002301F500A3008500B727002083A7479A3F
:107FF80003C50700EF90DFD6A9BDEFF07FDA91BD8A
:1080080013861605631BC7001C4503C5070021E935
:1080180085450545EFA0300E2DBD93862605014503
:10802800E319D7E69C4703C40700B727002083C796
:10803800E79C22858DE70D45EF909FC3AA85E30A4B
:1080480005E0930700FD2300F500F1472301F50043
:10805800B7270020A300850003C5D79C61BFEFF0B8
:108068001FD8C5BBB727002083C7C7CF411106C695
:10807800958B99CB37250020130505A8EFC00FA7CE
:108088004D45B240410182800145EFC02FA6014510
:10809800CDBF03C70500937625009377D70F99C204
:1080A80093672700131885011358884113F7F707BA
:1080B8006354080013E70708937685009377770FD2
:1080C80099C2936787001377050293F6F70D19C3D2
:1080D80093E607022380D500634508009377A5023D
:1080E80081CB8347060093E7C7002300F600828010
:1080F8007DFD83470600CD9BCDBF2D456319071431
:1081080003C8050009476310E814C8410347150070
:10811800034505002207498F42070D6541879308EB
:1081280025A0630B170B011122CC26CA4AC84EC6DC
:1081380006CEBE89B68432842E8963CEE8009307C2
:1081480005A0630DF702130515A06300A706239089
:1081580004000545B5A0930745A06309F7086348DF
:10816800F706130565AAE314A7FE85472390F600D2
:10817800DC4583C707002300F60091A0C845978017
:10818800FB1FE780A013420541814E8663733501CA
:108198002A862390C400420641828325C90022858D
:1081A8009780FB1FE780400719A8DC4583D70700A5
:1081B800239006012300F600A183A300F6000145E1
:1081C800F2406244D2444249B249056182809947EB
:1081D8002390F6001946D1B785472390F600DC4571
:1081E800014583C707002300F6008280DC45A9CB40
:1081F80021472390E60003D707002300E60003D7B2
:1082080007002183A300E60003D727002301E60027
:1082180003D727002183A301E60003D747002302E1
:10822800E60003D747002183A302E60003D76700CF
:108238002303E60083D76700A183A303F60041B7B1
:1082480023900600ADBF23900600054582808280FA
:1082580083C8050089476394F816DC41797122D4F4
:1082680006D626D24AD04ECE52CC56CA03C81700DC
:1082780083C707002E8422083368F80042088D67F8
:1082880013580841138327A0630C68102A8A3A8977
:10829800B684B285634C0301138707A0630BE80219
:1082A800938717A06301F80A854711A8138737A099
:1082B8006303E80C138767AA8D47E317E8FEB250FB
:1082C800225492540259F249624AD24A3E85456183
:1082D8008280484432C69780FB1FE78020FE420513
:1082E80041819D47E36D25FDB72A0020938A6A9E48
:1082F80083C70A00B3099900B24563D43701B5476B
:108308007DBF48442686C2094A959780FB1FE780AF
:10831800A0F003C60A00484493D9090105063306AC
:10832800364181454E959780FB1FE78000F6B727B9
:10833800002083A7879E99E3814751B79C438145D5
:10834800E5DF52853DA0AD47E31B09F6E39916FB2F
:1083580083471600834606005844A207D58F23108A
:10836800F700B727002083A7879EF9D79C43854548
:10837800E1D78297D1B7AD47E31309F49947E39062
:10838800F6F8484419469780FB1FE780E0E8B727CE
:10839800002083A7879ECDD39C43D9DF8D4555B751
:1083A800AD4711FF8547E39CF6F4034706009307A2
:1083B8000008E3E6E6F0DC452380E700B5BF854723
:1083C8003E858280B727002023A4079EB727002078
:1083D800A383079EB72700202383079EB725002085
:1083E800B707A0009385C596938707059CC1B70773
:1083F800E803DCC137D60600B727002093878787B4
:108408001306C6CCD0C3B72E002037D606000947BE
:10841800938E7E96130606CA372E00202380EE0020
:10842800130E4E96D0C723AED70137230020B728A6
:108438000020372800203725002037D60600B7DE71
:1084480006008546130606CB2300EE00938888961F
:1084580023AEC7031303439E130868961305559666
:10846800938E8ECB37DE06002380E8002380E7005A
:108478002388E7002380E7022388E7022380E704B4
:108488002300E8002384D70023950700D0CB238C52
:10849800D700239D070023A2D7032384D70223955F
:1084A800070223A60702D0DB238CD702239D0702ED
:1084B800231003002300D500130E8ECA23A2C7057C
:1084C8002388E70423AE17052380E7062388E706F9
:1084D8002380E708B7D8060037D706001307C7CAAE
:1084E800938888CC23A2E7082384D704239507041C
:1084F80023A66704F0CB238CD704239D070423A26B
:1085080017072384D70623950706ECD7F0DB238CBF
:10851800D706239D070623AE07072384D70823958C
:10852800070823A6A70837870400B72700209387E2
:1085380087901307271098C33787040013078725E8
:10854800D8C323A407008280A54763ECA710B7C748
:1085580006009387075C0A053E951C41011122CC51
:1085680026CA06CE4AC8B2842E8482879307800F13
:1085780063F9B7006145F2406244D244424905615B
:1085880082803729002093078987C857130989876C
:1085980009C99780FB1FE780A0B8B727002023836D
:1085A800079E13061400916593850571328532C6BE
:1085B8009780FB1FE78080A82326A90245DD324665
:1085C80081459780FB1FE78040CC0325C90222869E
:1085D800A6859780FB1FE78020C4B7270020238348
:1085E800879E014549BF8947E396F5F8035706007A
:1085F800B72700202392E79EEDB7A147E39CF5F645
:10860800372500202146A6851305C5969780FB1FB0
:10861800E78080C0F9B78547E39EF5F4B7250020C9
:1086280093858587D04D9385850203C50400EFF0B7
:108638005FA645BF8547E39FF5F2B72500209385E0
:108648008587D05D93858504CDB78547E394F5F29A
:1086580003470600B7270020A382E79659B70945C4
:1086680019BF0945828005476302E5044111AA87BD
:1086780006C62E8581CF11476383E70425476388A3
:10868800E7048947B2403E8541018280B727002030
:1086980083A5478A8947FDD5B727002003C6679E6B
:1086A8009780FB1FE78040B78147E9BFB7270020C5
:1086B80083D7479E2390F50081473E858280B72562
:1086C800002021469385C596EF30B261F1BFB727E8
:1086D800002083C757962380F500F9B7B7270020F5
:1086E8009387779E03C7070015E305472380E700B4
:1086F800058909CDB7260020372500209386869066
:108708004146A545130585876F304077014582802E
:1087180001111388F5FF06CE22CC26CA4AC84EC6D8
:1087280052C41378F80FAD4563ED050BB7C50600C5
:108738000A089385855E2E983E8A83270800BA89A1
:108748003689B28482878545EFB0DFD82A8419E15B
:10875800EFF05F912285F2406244D2444249B24927
:10876800224A056182808945EFB0DFD62A847DF1EF
:108778002685EFE06FECF9BF9145EFB0BFD52A84AD
:1087880071F95286CE854A85EFB03FCBEFF09F8DC9
:10879800EFF06FBEEF70E00575BFA145EFB09FD356
:1087A8002A844DF95286CE854A85EFB01FC92685A1
:1087B800EFE08FE8EFE0CFDEEF70A00161BFB145D9
:1087C800EFB05FD12A8459F55286CE854A85EFB03D
:1087D800DFC62685EFE04FE6EFE08FDCEF60707FC5
:1087E80075B7094485BF79714ECEAE896C0022D425
:1087F80026D24AD006D62A89B284EF00707B2A8412
:108808000DE1CE854A85EFB0AF952A8419E9324546
:10881800B746040026879386A6952D468145EF1016
:1088280040142285B250225492540259F2494561AB
:10883800828079714ECEAE896C0022D426D24AD07D
:1088480006D62A89B284EF00B0762A840DE1CE8557
:108858004A85EFB00F9F2A8419E93245B7460400CC
:108868002687938606A44D468145EF10800F228502
:10887800B250225492540259F249456182803971AA
:1088880026DAAE844C0022DC4AD84ED652D406DE14
:10889800AA893289368AEF00B0712A8431EDA6851B
:1088A8006303090283D704002C002314F10083D743
:1088B80024002315F100930720302316F1009307B5
:1088C80080022307F1004E85EFB06F862A840DE5FC
:1088D8005946A6851305A100230421019780FB1F93
:1088E800E78080931245B7460400528793864690E6
:1088F80025462C00EF10E0062285F2506254D2542F
:108908004259B259225A21618280797126D2AE84A5
:108918006C0022D44AD04ECE06D6AA893289EF00FE
:1089280030692A840DE1A6854E85EFB04F852A84EB
:1089380019E93245B74604004A8793868697354633
:10894800A685EF1000022285B25022549254025993
:10895800F24945618280BD47638CF50663E9B70239
:10896800A5476387F50663EDB7009947638CF5045F
:108978009D47638FF5049547638CF5040145828014
:10898800B5476387F50463E1B704AD47F5B7DD473D
:10899800638EF50263EAB700C947638BF502D947CE
:1089A8006386F502C547C9BFF5476383F50263E4EB
:1089B800B700ED47D1B793072005638BF500930700
:1089C800200D5DBF4845828008418280084582802D
:1089D800484182809307F00F630EF506011126CAFD
:1089E800AA841305000222CC4AC84EC652C456C2F5
:1089F80006CE3A89B689B28A2E8AEF906FA72A8462
:108A08004D4515C8930700FB2300F400A30054014B
:108A180023114401230234011305840061466305D0
:108A28000902CA859770FB1FE780007FA28526850B
:108A3800EF900FB30145F2406244D2444249B24933
:108A4800224A924A0561828081459780FB1FE78010
:108A5800C083E9BF09458280011122CC06CE2A8451
:108A68002306B100A306C100EF50207115C183464B
:108A7800C500B72700202147938787CF639EE6006C
:108A880003C5670078009306E0070146A285993779
:108A9800F24062440561828078009306E00701464F
:108AA800A28503C55700E5B7930700643306F602AD
:108AB8006F90DF9905C9034705008546930727008E
:108AC80093F7F70F63F0F602411122C42A843A851E
:108AD80006C6EF903FB2FD572300F400B24022448F
:108AE800410182808280035705009307000B6313BE
:108AF800F702834745004947639CE7000347150190
:108B080085476399E7000355250085456F309066D2
:108B18006D47C5BF828001112314B1006C0022CCBF
:108B280026CA4AC806CE2A89B6842315C100EF0092
:108B380030482A840DE12C004A85EFA09FD52A846D
:108B480019E93245B74604002687938626851546D7
:108B58002C00EF0010612285F2406244D244424961
:108B6800056182807971930720302314B1002315A1
:108B7800C1002316F1002C0093078002014606D697
:108B88002307F100EFF0BFCFB25045618280C17773
:108B9800797185073EC4894726D22316F100AE8431
:108BA800930780024C0022D44AD006D62A8923078C
:108BB800F100EF00F03F2A840DE12C004A85EFA078
:108BC8007FE52A8419E91245B7460400268793866B
:108BD800869E45462C00EF00D0582285B25022547C
:108BE8009254025945618280B28605466FF03FC9AA
:108BF800797126D2AE846C0022D44AD04ECE06D6E5
:108C0800AA893289EF00D03A2A840DE1A6854E85DB
:108C1800EFA05FBF2A8419E93245B73604004A87B6
:108C28009386E67E0D46A685EF00B0532285B250A6
:108C3800225492540259F24945618280797193070E
:108C480020202314B1002315C1002316F1002C00A5
:108C580093078002014606D62307F100EFF03FC2D2
:108C6800B25045618280011122CC06CE2A842EC6DC
:108C780032C436C2EF5060500DCD0345C500B7274A
:108C88000020A146938787CF12472246B245631C2E
:108C9800D50003C56700B2862E86A2856244F240DD
:108CA80005616FF03FD3B28603C557002E86A285B3
:108CB800F5B7F24062440545056182806FF0BFB2A6
:108CC8006FF07FB26FF07FC46FF03FC479714ECE02
:108CD800AE896C0022D426D24AD006D62A89B2841C
:108CE800EF00102D2A840DE1CE854A85EFA01FCB19
:108CF8002A8419E93245B74604002687938666997F
:108D08003D468145EF00F0452285B25022549254E9
:108D18000259F24945618280B28601466FF03FB63A
:108D2800011122CC2E846C0026CA06CEAA84EF003C
:108D38003028DD47630AF500930710102314F40068
:108D4800A2852685EFA0FFCFF2406244D244056198
:108D580082802394050083D7850099E36FF07FAD67
:108D680009458280FDB7B727002003C727A285479A
:108D780063F9E702011122CC2E846C0026CA06CEC4
:108D8800AA84EF00F02209E9930700102314F400E5
:108D9800A2852685EFA0FFCAF2406244D24405614D
:108DA800828059458280B727002023A6A79E82800B
:108DB800B727002023A8A79E8280011122CC26CAAB
:108DC80006CE2A84AE84EF50403BA6852285EFA0CC
:108DD8008FEE0DE9228523169100EF50003A1DC150
:108DE8008346C500B72700202147938787CF639024
:108DF800E60203C5670078009306F0070146A285DE
:108E0800EFF05FBDF2406244D2440561828003C541
:108E18005700D5B7011126CA06CEB68422CCDD4646
:108E280063E2B608D94663FED50AA5466381D50A2A
:108E380063EEB6049546638CD50899466387D50AD0
:108E4800054441687D18631606093AC6EFA06FEA23
:108E58003306854032474206418242044180330549
:108E6800C4004205BA85418132C6EF30D041AA8795
:108E780049C181C432462390C400B305804062448E
:108E8800F240D2443E8505616F803FD2C54663807B
:108E9800D504C9460D44E395D5FAC167FD17E31E0D
:108EA800F6FA65B7F5466380D50463E4B600ED4687
:108EB800D5B7930620056388D5029306200DE39164
:108EC800D5F8C167FD170D446319F600BDBF094405
:108ED8008DBF9306200DE392D5F8310642064182F4
:108EE800ADBF15445DBF0D444DBFC167FD171D449F
:108EF8007DB7F2406244D24405618280011122CCE0
:108F080026CA06CE03C645002E84130700028146F2
:108F18009945AA84EFF01FF02AC629CD835704008B
:108F280003464400930554002310F100835724009E
:108F38002311F10089472312F100930780022303CC
:108F4800F1009770FB1FE780202D834744008A8536
:108F580026852314F100EFA09F962A8411C5324577
:108F68009770FB1FE780C01B2285F2406244D24401
:108F7800056182804D44CDBF5D7186C6A2C4A6C27C
:108F8800CAC04EDE89476306F600C1470944631A22
:108F9800F6040144B9C52E894C0832C6B689AA849C
:108FA800EF0010012A8432460DEDC1778507CA8586
:108FB8001305D1013ECC230EC1009770FB1FE7803B
:108FC800A0252C082685EFF07FF32A8419E952455D
:108FD800B74604004E879386A68A1D462C08EF00E4
:108FE80050182285B640264496440649F2596161D4
:108FF8008280797122D436844AD04ECE52CCB2893E
:109008002E8A3A898146130710022286D94526D22C
:1090180006D6AA84EFF01FE02AC629C12286CA858F
:109028002314810023124101231331019770FB1F80
:10903800E780801E4C002685EFA07FAB2A8411C5EF
:1090480032459770FB1FE780A00D2285B25022544D
:1090580092540259F249624A456182804D44F5B7FB
:10906800011122CC26CA06CE4AC8DD472A84AE841E
:10907800638DF5028147035504006C002306F10057
:10908800EFA07FAA0545638EA40803458400B16557
:10909800938505B8EF90AF90E5472301F400B747F3
:1090A8000400938747B25CC0A5A80347550131491E
:1090B800B2863306270318499C4232971043E31BB4
:1090C800F6FA83D7460003564700E315F6FA8C46AE
:1090D80008479770FB1FE780602149DD83475401EB
:1090E80003474401850793F7F70FA30AF40063F0D9
:1090F800E704B3872703184803550400BA9798472D
:1091080083D6470003D6270083D50700EFF07FEE0C
:1091180035F103458400B165938505B8EF902F8834
:109128005945F2406244D2444249056182808347EE
:10913800640191B7011122CC26CA06CEDD472A84E4
:10914800AE84639CF50603550500EFA08FBA03565D
:10915800C40183562401035744016D162A9642061A
:109168004182B307D640C207231EC400C18363F1FE
:10917800E7089305C5FF3308F740635CB802BA9661
:10918800918EC206184C8355040103550400C18210
:109198003E97EFF01FE615E103458400B16593851E
:1091A80005B8EF80DFFF5945F2406244D2440561BB
:1091B80082806D1593160501F1B7814703550400A8
:1091C8006C002306F100EFA01F960545E38EA4FC72
:1091D80003458400B165938505B8EF805FFCE547DA
:1091E8002301F400B7470400938747B25CC065BF0A
:1091F8008547E9B7397126DAAE842C0022DC4AD8D3
:109208004ED606DE2A89B28965232A8421ED4A854D
:10921800EFA02FAE83D644006D1563C5A600931644
:109228000501C182984403D6240083D504004A85E9
:10923800EFF03FDC2A841DE53146A68508082306A1
:1092480001009770FB1FE78020FD83D7240022458B
:10925800B74604004E87938626AB5D466C00231EF6
:10926800F10001272285F2506254D2544259B25972
:10927800216182806FF01FF86FF0DFF7797126D2D5
:1092880006D622D44AD04ECE52CC56CA5AC88944A1
:10929800C5C159CE2E842A89BA8A368B328AEFA064
:1092A8004FA5930544008147711503D70500635204
:1092B800A70A850793F7F70FB105E318FAFE8A8521
:1092C8004A85FD21AA842DE531453305AA02916519
:1092D80093851570CD449770FB1FE78020D6AA8927
:1092E80021C931463306CA02A2859770FB1FE78061
:1092F800A0F2184483564400035624008355040002
:109308004A85EFF01FCFAA841DED0245B746040039
:1093180085475687938626AB5D464C002302F100AD
:109328004EC423064101A306010023076101152D40
:10933800B2502254268502599254F249624AD24ABE
:10934800424B456182804E859770FB1FE78040DD68
:10935800C5B7ED44F1BF79714ECE37D60600AE8958
:10936800C16526D20147AA848946130646CDFD1554
:10937800054522D406D64AD0EF10501B054431CDFE
:109388002A891307300281461146F5452685EFF0F4
:109398007FA82AC6554431C18357A900CE86014605
:1093A8002314F10091472315F10085472300F500A8
:1093B800B2472C002685A38007003247FD572301BA
:1093C800F7003247A301F700EF10100C2A8411C5EB
:1093D80032459770FB1FE780A0D42285B2502254F3
:1093E80092540259F24945618280411106C6EFF054
:1093F8008FD619C5B24041011773FB1F670043D2CE
:10940800B24041018280011106CE2AC6EF905FF476
:109418003245B727002023A6079EB727002023A898
:10942800079E9145B7270020A38CA7CEEF30006098
:10943800F24005616F20103A7971939705014AD07F
:1094480006D622D426D2C187014963DE070AB72788
:10945800002003C597CF2E89EF809F882A844DC1AD
:10946800034705009307000A6319F70885474C0866
:10947800A305F100EF90FFFAAA840DED834761017F
:1094880071476379F708138717FE1377F70F930669
:10949800000263F8E608858BD5CBB727002083A7A1
:1094A800C79E994481CB035524001306B1004C088C
:1094B8008297AA848347B10099C7084409C5977061
:1094C800FB1FE780E0C595E05247B7070001938787
:1094D80007F07D8FB707120093870710630FF70017
:1094E80003476101ED47631AF700035524008545DA
:1094F800EF304048CD476388F4002285EF802FF293
:10950800A1673349F900B25022544A85925402594E
:10951800456182803707301405073357F700058BFC
:109528003DDB372700200327079F49D70347510111
:1095380051F32306F10099472308F100035524004D
:109548006C0023170100EFA04F92ADB7B72700209A
:1095580083A7079F9DC3035524001306B1004C0839
:10956800829729D9AA8483475101A9F783476101C2
:10957800230891002306F100D1B79944EDB739715A
:1095880022DC26DA06DE4AD84ED652D456D25AD033
:10959800A5472A84B2846399F51083474502035787
:1095A8000600835A260085072302F5029307F7FF72
:1095B800B387FA025442C207C183B69703C917009A
:1095C80083C707008346C50022093369F900854728
:1095D8006390F60233075703231006008149014AB6
:1095E800130B3501931A070193DA0A0163E159074E
:1095F800C167FD176302F90C83570401637EF90AFA
:10960800050942098346C400135909012317240197
:109618000547035504009305E400639FE6002315FE
:10962800F100930720302316F100930780022314DA
:1096380021012307F1002C00EFA06FAF0345840040
:10964800B165938505B8EF809FB55945BDA083D610
:109658002400DC4083452401ED1613865900C20618
:10966800C1823E965A85EF903FD405C9630C3A01F2
:10967800C84003D62400B305350152959770FB1FE7
:10968800E78080B983D724003E9A83D70400420A32
:10969800135A0A0185072390F40083D72400BE9942
:1096A800C20993D9090199B703474600A94763102E
:1096B800F7028347450281CF0145F2506254D254E4
:1096C8004259B259225A925A025B216182808346DA
:1096D80024011309340137D506004A868945130544
:1096E800C5CCEF907FCC19C10545C1BF8346240185
:1096F80037D506004A868945130505CDEF90DFCAA0
:1097080065F58346240137D506004A868945130541
:1097180045CCEF907FC969F98346240137D5060007
:109728004A868945130505CBEF901FC855FD03C729
:109738004400BD47E3EAE7FAA56793874712B3D722
:10974800E700858BD5D38347440285072302F402BB
:1097580003D9240071BDB727002003C607D0B72757
:10976800002003A7479F81476315F6008146368589
:109778008280BA8613078702835587FDE389A5FE91
:10978800850793F7F70FCDB7011106CE2EC6EFF078
:109798009FFC01CD8347A500B24513871700639648
:1097A800E50093F707F82305F500F240056182808C
:1097B800011106CE2EC6EFF01FFA05C5B24591C1BC
:1097C80088C1834785001307E00F5D456388E7007C
:1097D8001307F00F01456383E7005945F24005611F
:1097E80082800945E5BF411122C42A84210506C6A5
:1097F80026C24AC0EFF00FAC83472400A51793F7A1
:10980800D70F91EB0347C40085476310F7061C4840
:1098180081443149A9E3FD5723010400A304F4005E
:10982800230204021305C4002244B24092440249B0
:109838006146814541011773FB1F670003A5B38784
:1098480024033E95084509C59770FB1FE780408DA6
:10985800850493F4F40F834744010848E3E1F4FED8
:109868009770FB1FE780C08B7DB7084C75F965B70B
:10987800411122C4416406C626C29307E4FF630E61
:10988800F500AA8485E1EFF01FED01E91305F4FF67
:10989800EFF07FEC19C123109500B24022449244A6
:1098A8004101828085476395F504EFF0DFEA2A8459
:1098B8006DD5FD572310F500834784001307F00F7B
:1098C8006385E7021307E00F638BE70083462400F4
:1098D8000345940001475146A685EFF0AF8F2285D6
:1098E800EFF07FF0FD572304F4002305040075B75B
:1098F8008947E394F5FA8545EF40902B59FD268575
:10990800EFF07FE52A844DF949BF39C9034785003F
:109918009307F00F6306F704011122CC06CE2A84C0
:1099280083462500835505000345950001475D469C
:10993800EFF04F8A03472400E1476319F700035506
:1099480004006C0023060100EFA0EF9DF9572304E3
:10995800F4002285EFF03FE9F2406244056182801D
:1099680082809307F00F6306F706011122CC26CAFE
:109978002A844EC6AE84B689AA859306850037A583
:1099880004004AC852C43A89328A13052591794697
:1099980006CEEFF06F91A304240123014401232292
:1099A800340185C01305C4006244F2404249B249FB
:1099B800224AA685D244614605611773FB1F6700DA
:1099C800A385F2406244D2444249B249224A056121
:1099D80082808280B7270020238CA79E82809547AB
:1099E800639CF50683474502854685072302F502F1
:1099F80083570600584203462600FD17C207C18355
:109A08006318D6048A07BA9703C7170083C70700E5
:109A18002207D98F0357E50063F9E704411106C609
:109A280022C485072316F5002A849305C50003552B
:109A38000500EF901FE603458400B165938505B8DE
:109A4800EF80EFF5B2402244D9473E85410182803C
:109A5800C946B387D70245BF83464600294785478D
:109A68006396E6000347450211C381473E8582801D
:109A78009D476392F506834745028356E5008507AF
:109A88002302F502835706005842FD178A073E97BE
:109A98008347170003470700A207D98F014763F6DA
:109AA800D704411106C622C485072A842316F50067
:109AB8009305C50003550500EFF04FC40345840026
:109AC800B165938505B8EF808FEDB24022445947C0
:109AD8003A854101828083464600A9470547639637
:109AE800F60003474502133717003A858280411173
:109AF80022C406C626C2B5472A84639BF504834759
:109B08004502B28485072302F50203550500EF904C
:109B18005F9E83D704001307F5FF014563C5E7027D
:109B28000357E400035504009305C400BA972317AC
:109B3800F400EF90DFE403458400B165938505B830
:109B4800EF80EFE55945B2402244924441018280BA
:109B5800034746009D470545E317F7FE03454402C2
:109B680013351500CDB7C547639EF5068357060024
:109B780003572600FD17B387E70203474502050789
:109B88002302E5025842C207C1833E978347370044
:109B980003472700A207D98F41677D176395E70020
:109BA80081473E858280138717002316E5000357F7
:109BB800E500E3F7E7FE411122C49305C5002A84B6
:109BC8000355050006C6EF90FFE403458400B16520
:109BD800938505B8EF80AFDCB2402244D9473E8573
:109BE800410182808346460029478547E39BE6FA80
:109BF8000347450255F775B7011122CC26CA4AC852
:109C080052C406CE4EC683C7250015472A8AAE849D
:109C180032843689639DE7043686A2852685EFF06F
:109C28001FDCAA8955E985476318F40A03474900E8
:109C3800A9476301F70203C594004A878546014690
:109C4800D285EFE03FD919E585454A85EFE0BFD0D9
:109C58001334150083C6240003C5940001476946E0
:109C6800D285EFE03FD72685EFF0FFB751A01D471B
:109C78006398E7003686A2852685EFF07FDF55B723
:109C880025476398E7003686A2852685EFF03F8F43
:109C980049BF35476398E7003686A2852685EFF0E9
:109CA8001FE541B745476398E7003686A2852685B4
:109CB800EFF07FEBBDB75D47639FE70003C7C500C3
:109CC80085473686A2852685631DF702EFF04FB9D2
:109CD8008547631BF5048549A5476317F402835735
:109CE80009009DE30544E38709F6D947E39DF9F6A2
:109CF8002285F2406244D2444249B249224A05616F
:109D08008280EFF02FC3E9B703C594004A87A28683
:109D18000146D285EFE01FCC71F5A2854A85EFE0B8
:109D28009FC313341500C1B70544D9B7397122DC74
:109D380006DE26DA4AD84ED652D456D283D7050044
:109D48001944B1E783C925002A89328A938759FEC5
:109D580093F7D70FAE84DDE7B727002083C6879F28
:109D68001307F00F938A879F19446382E602F54729
:109D78006394F904EFF03F9EAA8921C10346A50028
:109D88000DCE93178601E18763DD07000144228524
:109D9800F2506254D2544259B259225A925A21610D
:109DA8008280F5454A85EFE03FCB83C7A90093E75A
:109DB80007F82385F900D9BF814983D64400904428
:109DC80083C5140003C504003800EF90DFD62A8449
:109DD8005DFD83C6240003C50A0038000146CA8514
:109DE800EFE05FBF2A8445F5B24799C323000A0014
:109DF80083C724007547E39BE7F8E38909F82385BF
:109E0800F90071B7EFF03F95AA8A49D18547639168
:109E1800F90A83D5440088443000EF906FEF2A8414
:109E28003DF503C72A00C54763F2E70ADD4763012A
:109E3800F70CB727002003C59A0083C797CF639C08
:109E4800A70A014403C72A008D47631FF7048357F5
:109E5800810003D7CA0063F4E7002396FA0083D58C
:109E6800CA004A85EFE07FF5B727002083D747B4BB
:109E78006D47637BF70283D5CA005D476376B702F7
:109E88001387350091056349F7001307B00FBE85A6
:109E98006374F7009305B00F1166C205130606290F
:109EA800C1814A85EF8010175685EFF0DF93C5B55D
:109EB800834725001144E39C37ED5C41E38907ECB7
:109EC80083D5440088443000829791BFB7270200A9
:109ED8009387072AB3D7E700858BA1DF03C6240041
:109EE8003400D6854A85EFF03FD12300AA0045B556
:109EF80083A70A01DDB783C6240038000146CA8556
:109F0800EFE05FAD2A841DFD83C524002800EFE043
:109F18009FA405D923000A0035B7011122CC3724A4
:109F2800002006CE26CA4AC84EC652C4930984CF1A
:109F380003C589009307800291653305F50293856F
:109F48006570372900209304499F9760FB1FE780BD
:109F5800E00E03C689009307800281453306F602A6
:109F680088C09760FB1FE78040329C404D45A1C3E5
:109F7800930484CF1309499F0144130A8002FD59B1
:109F880083C78400636DF40237A50400130545D325
:109F9800EFE07FE13795040013050579EF902FC7AF
:109FA80037A5040013058587EF40A0370145F24027
:109FB8006244D2444249B249224A05618280B307C9
:109FC8004403032509006146814505041374F40F11
:109FD8003E9523103501230105002314350123057F
:109FE80005002302050231059760FB1FE780E02981
:109FF80041BF01458280B727002083C617D081471B
:10A0080063E5D70001473A8582802E87910503D6FC
:10A01800C5FFE30AA6FE8507E5B70DCD83472500F2
:10A028000547890793F7F70F6376F702411122C4B2
:10A0380006C62A8483550500034535000147F946BD
:10A048005D46EFE03F99F9572311F400B2402244EE
:10A05800410182808280B727002003C717D0FD56B0
:10A06800814763E3E70082802310D50023010500C0
:10A0780085071105FDB701458280372600201306A4
:10A088003698930700022300F60037270020FD5773
:10A098002301F79837270020A30AF79637270020CF
:10A0A800230AF7968545B72700202390B798B72746
:10A0B8000020239D079EB727002023A207A0B727CB
:10A0C800002023AA07A0B727002023A407A0B726AB
:10A0D8000020B7D7060093868697938707CCDCC203
:10A0E800B7270020238E079EB72700209387479124
:10A0F80009472380E6002380E7002388E7002380C0
:10A10800E7022388E70237D70600130747CBD4C7EF
:10A11800D8DBB7D606000D47238CE702938606CB1B
:10A1280037270020D4CB032707A037D50600B7D69A
:10A1380006001305C5CC938646CDC8C32384B70053
:10A1480023950700238CB700239D0700D0CFD4D3D5
:10A15800238407022395070223A60702239D0702EB
:10A16800D8DFB727002037A7040093874795130740
:10A17800A72323A00700D8C323A407008280411186
:10A1880006C6EFF05FE711C503452500B24041015F
:10A1980082800145E5BF411122C426C24AC006C6D5
:10A1A800AA842E893284EFF01FE511E94165CA853A
:10A1B8007D15EFF05FE4C54711C523109500230115
:10A1C80085008147B2402244924402493E854101BC
:10A1D800828029E78948354763931605011106CE21
:10A1E80022CC26CA034716000346060093C7F7FF8A
:10A1F8002207598EF18F32C68DE7C4452A84A68579
:10A20800EFF0FFF732460147630FA600228562444C
:10A21800F240A685D24405616FF0FFF72D473A85D5
:10A22800828013070008F2406244D2443A850561EF
:10A23800828083C8050009486395080303A8450080
:10A248008347180003480800A207B3E70701C207BD
:10A258000D68C187130828906395070189476FF037
:10A268005FF705458280011122CC372400201304B2
:10A2780054970347040006CE26CA4AC84EC6930719
:10A28800F00F6300F704AA892945B2842E89EF707C
:10A298003F9E05C99307100B2310F5002302050004
:10A2A800231135012313250123149500AA8503459D
:10A2B80004006244F240D2444249B24905616F70D9
:10A2C8003FAAF2406244D2444249B24905618280C1
:10A2D8004111B727002026C2AE8483A507A022C457
:10A2E80006C62A84EFF0BFE9098909C922852244F4
:10A2F800B240A685924441016FF0EF85B2402244F6
:10A308009244054541018280411122C426C24AC0B7
:10A3180006C6AA84130445001309850B8357040055
:10A328009DC3084409C59760FB1FE78060DF22854D
:10A33800314681459760FB1FE78020F53104231AD9
:10A3480004FEE31D24FDB2402244FD572390F4008F
:10A358000249924441018280B727002003C617D0E2
:10A36800B727002003A7C7A081476315F6008146D9
:10A3780036858280BA861307870B835587F4E3896D
:10A38800A5FE850793F7F70FCDB7B727002083A75A
:10A3980047A189CB03D747006314A7008847828069
:10A3A8009C43C5BF01458280411106C6EFF0FFFD01
:10A3B80009C50845B240410182800145E5BF011148
:10A3C80026CA9384450022CC4EC606CE4AC852C43B
:10A3D80056C25AC0268781490144814681473D4576
:10A3E8000356070055CED9E2035447008357270088
:10A3F800B286A297C207C18385093107E392A9FEF5
:10A4080025C82E8991659385457022859760FB1F25
:10A41800E780C0C22A8B29CD814A014A8C4485C570
:10A4280003D6440033054B019760FB1FE780C0DE6D
:10A4380083D7440088443E9A420A135A0A01976017
:10A44800FB1FE780E0CD63890A00314681452685F8
:10A458009760FB1FE78060E3850AB104E3E03AFDFB
:10A468002326690123148900054521A0630DD60020
:10A478000145F2406244D2444249B249224A924AD2
:10A48800024B0561828003562700E313F6FE03564C
:10A4980047003294B2974204C2074180C183A9BFE2
:10A4A8000545E37835FDA9BFB727002083A787A016
:10A4B80099E30145828098470357A7006315A700D1
:10A4C8001385470082809C43E5B7411106C6EFF02B
:10A4D800BFFD11C503550500B24041018280014509
:10A4E800E5BF411106C6EFF03FFC11C50345250045
:10A4F800B240410182804145E5BF411122C42A840E
:10A508002E8506C6EFF0FFFDAA8505462285EF30A9
:10A51800F04995476305F500BD476313F5002145EC
:10A52800B2402244410182804111B727002022C451
:10A5380006C603A487A08146938787A029C018442C
:10A548000356A70018406317A60285CA98C22E852D
:10A5580081C92146930544009760FB1FE780C0CB63
:10A5680022859760FB1FE780A0BB0145B2402244CB
:10A5780041018280A2863A84D1B798C3C9BF0545F4
:10A58800F5B737270020832747A10146130747A1BE
:10A59800A9C703D847009443631CA802011106CE3B
:10A5A80022CC26CA0DCA14C2AA843E852E8497607E
:10A5B800FB1FE780E0B62C002685EFF0FFF601E5EB
:10A5C80019C0B2471CC0F2406244D244056182807F
:10A5D8003E86B68775BF14C3C1BF05458280411149
:10A5E80022C42A84090506C6EFE0CFCCFD57A30193
:10A5F800F400B240224441018280B727002003C7FB
:10A6080017D0B727002083A707A12A860507814608
:10A618003E8583D707006388C700850693076500D2
:10A62800E3E8E6FE01458280411122C4416406C682
:10A6380026C29307E4FF630EF500AA8485E1EFF0D4
:10A64800DFFB01E91305F4FFEFF03FFB19C123100D
:10A658009500B24022449244410182808547639428
:10A66800F504EFF09FF92A846DD5FD572310F50006
:10A67800834724001307F00F6384E7021307E00FF2
:10A68800638AE700034534000147F9465146A68529
:10A69800EFE04FB42285EFF09FF4FD572301F4005B
:10A6A800230204007DB78947E395F5FA8545EF3025
:10A6B800305045F12685EFF05FF42A8455F951BFF3
:10A6C8001D71A6CACEC686CEA2CCCAC8D2C4D6C26E
:10A6D800DAC05EDEAE8483C52500F947AA89639790
:10A6E800F504EFF09FF12A8411ED01442285F6402C
:10A6F8006644D6444649B649264A964A064BF25B12
:10A7080025618280834725000547890793F7F70F5E
:10A71800E37DF7FC034535000147F9460146CE8540
:10A72800EFE04FAB2285EFF09FEBC1B703AB04001E
:10A73800B7070001938707F037071200B377FB00CC
:10A7480013070710B28A0149638AE7022EC6EFF0A1
:10A75800DFEA2A89B2451DC10346450005C29317A1
:10A768008601E187E3C307F84E85EFE0EFAE834744
:10A77800490093E707F82302F90085BF372A00202C
:10A7880003472A989307F00F130A2A981944E30FEE
:10A79800F7F4E147E3ECB7F493D71500FD171397E7
:10A7A8003700B7C7060093878761BA9703A80700E1
:10A7B800E30E08F283AB4700E38A0BF2420B135B0C
:10A7C8000B0163050B00C947E392F5F283D64400F9
:10A7D800904483C5140003C50400380802982A84ED
:10A7E800E31605F02C084E85829B2A8421C983C76D
:10A7F8001400E39D07EE83C72400230AA10039470C
:10A808002308F1006399E70262478347170003476B
:10A818000700A207D98F0C084E852319F100EF8095
:10A82800DFE4E30405EC14080546D9454E85EFE05E
:10A838008FC32A8465BD83578101F1BF83C6240075
:10A848009147E384F6EA03450A0038080146CE85B5
:10A85800EFE04F982A84E31B05E883C52400280805
:10A86800EFE06F8F19C123800A009840B7070001F5
:10A87800938707F07D8FB707120093870710E306C9
:10A88800F7E6E30409E683C724002302F900B9BD0B
:10A89800011106CE2EC6EFF05FD601CD83474500E5
:10A8A800B245138717006396E50093F707F823026C
:10A8B800F500F24005618280B727002003A787A032
:10A8C80019E3014615A81C4703D8A700636B0501C7
:10A8D80083584700B38608016355D50081466394C1
:10A8E80016011843F1BF3E86C10703D3A7FF6317BC
:10A8F800A30099C123900501328582808506C2068E
:10A90800C182F1BF397152D42E8A4ED69305E10126
:10A91800AA89528522DC4AD856D206DE26DA32893E
:10A9280036C63AC4BE8AEFF03FF9054435C5AA8455
:10A938000355E1013944EFF05FA539CD03284500FF
:10A94800630C08042247B246D6874A86A6854E85F8
:10A9580002982A8431E19307E00F638FFA0203C754
:10A9680004008947631AF702D84083471700034752
:10A978000700A207D98FC2070D67C1871307279061
:10A98800639CE7008347190003460900D285A207A4
:10A998005D8E4E85EFF03F8D2285F2506254D25481
:10A9A8004259B259225A925A21618280797122D42D
:10A9B800035425004ECEAA89228556CA06D626D229
:10A9C8004AD052CC5AC85EC662C4AE8AEFF0DF984D
:10A9D80001E92285EF906FE9594429E90144B9A0BA
:10A9E80003C789008547AA840144631AF702AA8528
:10A9F80013858900EFF0BF9C29CD03D7640083D667
:10AA08008400D04483D5440003D52900E147EFF002
:10AA18007FEFD9472A846318F50223A60400268508
:10AA2800EFF09F8E49C0D947E30AF4FA2285B25065
:10AA3800225492540259F249624AD24A424BB24BCA
:10AA4800224C4561828061DD83D744002390FA005F
:10AA5800F9B713894400014AB94B594C3D4B83550A
:10AA68000900D5DDE14763067A010357C90011C320
:10AA7800D94703572900835649000326890003D57F
:10AA88002900EFF03FE82A8463198501232409008F
:10AA9800050A3109E3156AFD59B77DD983570900BD
:10AAA8002390FA00F5B703D529002DB70111231714
:10AAB800C1009307E00F1306E1000147894606CE5F
:10AAC800EFF05FE4F24005618280797122D42A8434
:10AAD8000355850026D2AE849305210106D64AD0B7
:10AAE800EFF09FDD6308050E834785002AC693F7BC
:10AAF80007028DCF03552101EFF01F8BAA87B245BE
:10AB080001ED8357840039452390F400B250225454
:10AB18009254025945618280035524004946829720
:10AB280011C5835784002390F400CDB7035924003E
:10AB38004A85EFF07F8211ED41657D15EFF0DF81E9
:10AB480019E58357840025452390F400C1B72310E5
:10AB58002501130745008147BD46035607002DE62A
:10AB68003147B387E702130984003146CA85910744
:10AB78003E959750FB1FE780206A3146CA854808F2
:10AB88009750FB1FE78040690356C4000355240013
:10AB980041478146DD45EFE0EFA72ACE19E5835707
:10ABA800840045452390F40095B70C480356C4002B
:10ABB8009750FB1FE7804066035524004C08EF9030
:10ABC8008FC629D5594599B785073107E397D7F82F
:10ABD800254581BF0545B1B7797122D42A8403552B
:10ABE800850026D2AE849305E1014AD006D6328983
:10ABF800EFF09FCC51C58347850093F70702A9E77B
:10AC0800034714019307200519E38347440083563B
:10AC1800A400504483558400035524000147EFF0F5
:10AC28007FCEAA8721E98347140199E703552400B9
:10AC3800EF908FBAD94711E18147B250225492540C
:10AC480002593E85456182802AC60355E101EFF02D
:10AC5800AFF5AA8705C9B24503552400494682972E
:10AC6800AA8759DD035784002390E40003471401A1
:10AC780061F7E1B75947E317E5FE230009006DBF07
:10AC88008547CDB7B947F9BF397122DC4AD84ED6C6
:10AC980052D406DE26DAAA892E8A32C63689EFF021
:10ACA800DF95094415C5834725001307E00FAA84DB
:10ACB8005D44638FE7001307F00F5944639AE70078
:10ACC800324605E2D2854E85EF900FBE2A8415CD17
:10ACD8002285F2506254D2544259B259225A216103
:10ACE800828003550A009305E101231F0100EFF05C
:10ACF800BFBC0355E101EFF0CFFEAA8505464E859E
:10AD0800EF30C04A2A845DDDE1B79307F00FE30115
:10AD1800F9FC37A50400938624007946A685130517
:10AD28002502EFD07FD8A38124015DB73971B727F9
:10AD3800002026DA83A487A052D45AD05ECE62CCF3
:10AD480006DE22DC4AD84ED656D266CA2A8BAE8B8D
:10AD5800328C368A99E08149B9A0804483DC44006A
:10AD68000149835AA400631499018440E5B78357C5
:10AD7800A400A28963F8670105094209135909016A
:10AD88004104D5B7E3EAFBFE630C0A0083450400DF
:10AD98004840D28662863AC6EF800FE1324769DDC5
:10ADA80019C323105701F25062544E85D2544259A8
:10ADB800B259225A925A025BF24B624CD24C216130
:10ADC800828003D7050083D62500854763E9E6041A
:10ADD80039C7411183C6450026C237D5060093847A
:10ADE800550022C426862E841305C5CC894506C67F
:10ADF800EF808FDBC14711CD834644008355240083
:10AE08000355040001472686EFF05FF2814711E100
:10AE1800A947B240224492443E85410182803E8542
:10AE280082802E860355060083D52500854763E278
:10AE3800A50205C18346460041110147150606C60D
:10AE4800EFF0DFEE814711E1A947B2403E854101AD
:10AE580082803E8582802E860355060083D5250094
:10AE6800854763E2A50205C18346460041110147B3
:10AE7800150606C6EFF09FEB814711E1A947B240DE
:10AE88003E85410182803E85828039714ED683D7C6
:10AE9800250083D9050006DE22DC26DA4AD852D4FA
:10AEA80056D25AD05ECE62CC66CA6AC863E03719F9
:10AEB8008547638E0914416BAE8A2A8A23140100E0
:10AEC80002C6014401497D1B894B054CC94C054DFF
:10AED80083D52A000147814601464E852313010088
:10AEE800EFF0DFE4AA846300051209EC13072002DF
:10AEF800930661005A8695455285EFD0BFF12A84A2
:10AF0800630805120357810083C7040045C7034738
:10AF1800A100630CA70741476385E7022C0052850F
:10AF2800EF807FD909CD34001546D9455285EFD039
:10AF38009FD311C532459750FB1FE780601E81479C
:10AF4800F9A083D7A4004146130524002300F40088
:10AF580083D7A400A183A300F400CC409750FB1F23
:10AF6800E780802B4904835781008507C207C18386
:10AF78002314F10063F9270983D7A40063856709BF
:10AF88008509C20993D90901A1B7E39977F983D74C
:10AF9800A4000946130524002300F40083D7A40065
:10AFA800A183A300F400CC409750FB1FE780C02684
:10AFB800110455BF22C60359610003C7A400130535
:10AFC8002400638277033359990323057101230011
:10AFD800E40083D7A4004146A183A300F400CC4039
:10AFE8001379F90FA5BF230581012300E40083D756
:10AFF800A400135929001379F90FA183A300F400C1
:10B008000946CC4055B78357810089FBA947F250C0
:10B018006254D2544259B259225A925A025BF24BA4
:10B02800624CD24C424D3E85216182808547C5B72E
:10B03800C547F1BFB727002003C727A2854763F399
:10B04800E706011122CC26CA4AC806CE2A843289CC
:10B05800AE84EFF08FDA01C9034725009307E00FAC
:10B068005D456308F700631C0900A6852285EF90FB
:10B078008F80F2406244D24442490561828003D500
:10B0880004009305E10023170100EFF0FF82035548
:10B09800E100EFF00FC5AA8505462285EF300011C3
:10B0A80069D5C1BF5945828013F7050201C7B2852A
:10B0B8006FF0AFC4411126C24AC006C622C413F9B4
:10B0C8008500AA8463170900139785016187635D6A
:10B0D800070232853684EFF0CFC0AA850546631390
:10B0E800090001462685EF30600C01E90145B240B0
:10B0F8002244924402494101828083479400E5DB5F
:10B1080083478400E5F7E5B793F72500E5F30D4598
:10B11800F9BF7971AE8622D42A8403D50600930537
:10B12800E10106D636C6EFF02FF909CD8345850033
:10B13800B2460356E1012285EFF01FF7B2502254C0
:10B14800456182800545DDBF13F7050201C7B28559
:10B158006FF0AFBA411122C426C206C693F4850027
:10B168002A8491E413978501618763500702328529
:10B17800EFF02FB7AA85054691E0014622852244C3
:10B18800B240924441016F30600293F725000145B7
:10B1980091E30D45B2402244924441018280797185
:10B1A800AE8622D42A8403D506009305E10136C66B
:10B1B80006D6EFF06FF0B24601CD83458500035601
:10B1C800E1012285EFF05FF8B25022544561828098
:10B1D8000545DDBF797126D2AA840355A500C1674C
:10B1E80022D44AD04ECE06D623170100FD1732844A
:10B1F800B6890149630DF500050583C60400D040F2
:10B2080042051307E1004181EFF05FB22A8983C646
:10B218000400D04037D5060089451305C5CCEF801A
:10B22800AF981DC503D4A4002285EFF00FAA09C565
:10B238007D142A9442044180638409002390890084
:10B24800B25022544A8592540259F249456182808B
:10B2580083C60400D04037D506008945130505CDBF
:10B26800EF808F9461F183C60400D04037D5060083
:10B278008945130505CBEF802F9319C9E30609FA11
:10B288008357E100E39287FA0354A9007D145DB760
:10B2980003D4A40055B7397122DC26DA4AD84ED631
:10B2A80052D456D25AD062CC06DE5ECEBE8983C74F
:10B2B80085002A8AAE84C18B328C36843A89C28A48
:10B2C800468B9DE783CB04008947638BFB0462852B
:10B2D800EFF0AF8B1DC183280500638008025A88F0
:10B2E800D6874E87CA862286A6855285829839A037
:10B2F8003285EFF06F8BAA8711ED3945F250625411
:10B30800D2544259B259225A925A025BF24B624CB9
:10B31800216182802946A6855285829745D5F9BF45
:10B32800D8408347170003470700A207D98FC207F1
:10B338000D67C187930607906384D72263CEF6060C
:10B3480093062780638ED70C63C1F6021307078024
:10B35800E3CFE7F62D45E39309FADC4403C607007B
:10B36800CC432310C900228569A213073780E390D4
:10B37800E7F62D45E39409F885472310F900DC44E6
:10B38800814583C707002300F40003D5A400050501
:10B3980042054181EFF04FD2835709006317051228
:10B3A80091072310F90011468145130514009750A1
:10B3B800FB1FE78080ED29A2930627906383D718A7
:10B3C80063CED71293063790638CD718130747902C
:10B3D800E39FE7EE2D45E39309F2DC441D47231074
:10B3E800E90003C707002300E40003C71700A30010
:10B3F800E40003D727002301E40003D727002183B3
:10B40800A301E40003C747002302E40003D7670051
:10B41800A302E40083D76700A1832303F4004DA0AF
:10B428002D45E39D09ECDC446C0083C9170003C774
:10B438000700A209B3E9E90011472310E90083C70F
:10B4480007004E852300F400DC4483C71700A300DF
:10B45800F400EFF06FC6AA8435C50356C100C16574
:10B468009306E100FD158329C500EFF0BFD619ED5D
:10B4780083C60400D04037D506008945130505CD9D
:10B48800EF709FF201E5FD572317F10003C709008C
:10B4980089476310F70283A549000946130544004C
:10B4A8009750FB1FE78040D783570900890723106F
:10B4B800F9008357E1002301F400A183A301F400FC
:10B4C80001452DBD23173101EDB703470500890755
:10B4D800BA972310F9008357A500A300F4008357F7
:10B4E800A500A1832301F400034605004C41130580
:10B4F80034009750FB1FE78020D2D9B7C844975033
:10B50800FB1FE780A0DB93170501C1832A871D4530
:10B51800E3E637DF6399F90023100900CC440356AA
:10B528000900CE9589B54207B3863A01418363C7BE
:10B53800E600B38737412310F900CDB7231059012E
:10B54800F1BF2D45E39C09DACC445285EFE03FC3B7
:10B55800231079012300A4002181A300A4008DB742
:10B568002D45E39D09D8DC442310790183C70700E2
:10B578002300F400DC4483C71700A300F40089B754
:10B588001D71CAC82A8903552500A2CCCEC6D2C4CB
:10B59800D6C2DAC05EDE62DC66DA6ED686CEA6CAAF
:10B5A8006AD8AE8AEF70FFF4130CF5FF93170C01FD
:10B5B800B72B0020C1832A8A814913844BA93EC630
:10B5C800372B0020B72C0020C16D8357C90063F6C4
:10B5D800F9008357040063CC87010355290093853C
:10B5E8004BA9EF80FF932A8D15CD594D25A88327A8
:10B5F8008900139719009305E101BA9783C41700CE
:10B6080083C70700A204DD8C2685EFF0EFAAAA8580
:10B6180015E923909A004840054D09C59750FB1F2E
:10B62800E78000B0F64066446A85D6444649B64984
:10B63800264A964A064BF25B625CD25C425DB25D7A
:10B648002561828032488348490083A64CA003566E
:10B65800E1010355290081471307AB9FEFF0BFC3F2
:10B668002A8D13884CA009C523909A00484075B7C5
:10B678005C4085E703552900514781461386FDFF45
:10B68800BD45EFD02FF9B727002048C0138847A041
:10B6980009E523909A00454D71B783570400035775
:10B6A800AB9F9304AB9F3E976347470113C7F7FFD0
:10B6B80052972390E400484003D6040083250800ED
:10B6C8003E9585099750FB1FE78000B58357040016
:10B6D80003D70400C20993D90901BA972310F400CB
:10B6E800EDB5397122DC2A840355250006DE26DAF9
:10B6F8004AD84ED652D45AD05ECE62CC66CA2E8B69
:10B7080056D26AC8EF70FFDE2A8A8346C400835582
:10B71800A4000355840078001306D400130CBAFF64
:10B72800651AEFF0AFE0420A37290020AA89814460
:10B73800135A0A01B72B0020B72C0020130949A976
:10B748006386090463D48405938A4CA08348440023
:10B7580083A60A000356C100035524005288814776
:10B768001387AB9FCE85138DAB9FEFF0DFB215C566
:10B77800814A0356C1008355A4004E859306E10013
:10B78800EFF05FA5AA89639D0A065DF9E5E0835796
:10B79800840029452310FB0089A083570D00035618
:10B7A8000401E317F6FC83A50A0048489750FB1FDD
:10B7B800E780C0B355DD83274900A1E30355240082
:10B7C8004166454781467D169D45EFD0AFE405E5C6
:10B7D8008357840045452310FB00F2506254D2542D
:10B7E8004259B259225A925A025BF24B624CD24CDD
:10B7F800424D216182802322A90083DAA90095BFE6
:10B8080083274900A697238057019387140013972D
:10B81800070183274900418393DA8A00BA97238076
:10B828005701138724008326490093873400420771
:10B8380091044183C207C204C183C180369711CDE8
:10B848008356E1002300D70003274900BA9703571E
:10B85800E10021832380E700E5B5FD562300D700EA
:10B8680003274900BA972380D7000DB70355240052
:10B87800B72500208980239A95A8938545A9EF804C
:10B888002FD021DD594591BF411122C406C693F737
:10B8980005012A84328585C3EFE0BFC4AA85054621
:10B8A8002285EF20B01095476305F500BD47631D5D
:10B8B800F502214515A893F7450099CBEFE07FC223
:10B8C8000546AA8522852244B24041016F20100E08
:10B8D80093F7050489C7EFE0DFC00146DDB713F52C
:10B8E8001500133515000605B24022444101828037
:10B8F80079714AD04ECE52CC06D622D426D22A8A84
:10B90800AE89014983D749006364F9000145A1A0C4
:10B9180083A70900131419009304140033879700B0
:10B9280003470700A29703C5070022079305E10014
:10B93800598DEFE07FF805E983A7090005453E9496
:10B94800034704002380E70083A70900BE9403C7C8
:10B958000400A380E700B250225492540259F249DD
:10B96800624A45618280834585000356E10052851D
:10B97800EFF09FF105C183A709003E940347040037
:10B988002380E70083A70900BE9403C70400A380AF
:10B99800E700D1B70509420913590901A5B70111F3
:10B9A80022CC2A8403D505009305E10006CEEFE0FA
:10B9B800BFF001CD834585000356E1002285EFF0F5
:10B9C800BFECF2406244056182800545DDBF1D7110
:10B9D800CAC82A890355250086CEA2CCA6CAD2C4D5
:10B9E800D6C2DAC05EDE62DC66DA2E8ACEC66AD8D5
:10B9F8006ED6EF701FB02AC68346C9008355A900CA
:10BA08000355890078081306D900EFF02FB2B24722
:10BA1800B7240020416B938AA7FFC20AAA8B01446E
:10BA280093DA0A01372C0020B72C0020938444A90C
:10BA38007D1B63860B180356C10183C58B00035514
:10BA48002900EFF07FE4AA8D6316051683484900A4
:10BA580083A64CA00356C101035529005688814787
:10BA68001307AC9FDE85EFF01F83AA8D9309AC9F67
:10BA7800138D4CA06310051429C003D7090083D780
:10BA8800240011076397E7003247A2976D1763CA2E
:10BA9800E706B7250020938745A903D72700035554
:10BAA8002900938545A93354E40223908700EF8049
:10BAB800AFCAAA8D15C1D94D05A00355290049471C
:10BAC80081465A86C545EFD0EFB4C8C015E583D77F
:10BAD800AB00C54D2310FA00F64066446E85D64487
:10BAE8004649B649264A964A064BF25B625CD25CE6
:10BAF800425DB25D2561828083D709009107239159
:10BB0800F400DC4003D7AB009306E101A297238041
:10BB1800E7009307140013970701DC4041835E8513
:10BB2800BA9703D7AB0021832380E7000356C101EE
:10BB38008355A900EFF00FEAD440130724000356F9
:10BB4800E1014207418336972300C700D840930795
:10BB58003400C207C183BA970357E101AA8B1104C5
:10BB680021832380E700C8404204418003D60900AE
:10BB780083250D00229563950B029740FB1FE780F4
:10BB8800A06983D709003E9442044180E31304F07E
:10BB9800835789002310FA00E3900DF4A94D2DBFB7
:10BBA8009740FB1FE780406783D709003E94420413
:10BBB800418041B583D7AB002310FA00C1BF814D46
:10BBC800F1B75D71A6C2CAC0AA840359850003559E
:10BBD8002500A2C44EDE52DC5AD85ED662D466D2A4
:10BBE80086C656DA6AD06ECE2E8BEF709F90930B76
:10BBF800D5FF7115131A0501B72900200144135AFE
:10BC08000A01372C0020B72C0020938949A96359D1
:10BC1800741583C6C40083D5A4001307E1001386F6
:10BC2800D4004A85EFF08F902A8D630B05120359D3
:10BC3800A500834585000356E10003D52400EFF0F5
:10BC4800BFC46314051283C8440083A64CA00356DE
:10BC5800E10003D52400528881471307AC9FEA8589
:10BC6800EFF06FE3930DAC9F13884CA0631F050E94
:10BC78001DC883D70D0003D729008907630CF70671
:10BC8800B7250020138745A98357270003D524002B
:10BC9800938545A93354F40223108700EF800F9849
:10BCA80015C5594525A003D5240041664D47814651
:10BCB8007D16A545EFD00F96B727002023A2A9002F
:10BCC800138847A01DE123102B014545B6402644A3
:10BCD80096440649F259625AD25A425BB25B225CD8
:10BCE800925C025DF24D6161828083D70D00890705
:10BCF8002391F90083D70D00A29763D3770783A711
:10BD080049000357AD00930A2400A2972380E70057
:10BD180005049317040103A44900C183C20A3E9491
:10BD28008357AD008325080093DA0A01A183230015
:10BD3800F40003A5490003D60D0056959740FB1F54
:10BD4800E780804D03D40D00C167FD175694420467
:10BD58004180E30EF9EA050942091359090145BD75
:10BD6800294519FC23102B0195B76DDC11BF8357AA
:10BD7800050081E789473E858280411126C24441FA
:10BD880022C406C64AC083C60400D0402A8437D5D8
:10BD9800060089451305C5CCEF700FE119C9834723
:10BDA80024002547E51793F7F70F6377F702E14774
:10BDB80029A883C60400D04037D506008945130555
:10BDC80005CDEF706FDE61FD8947B2402244924491
:10BDD80002493E854101828037290020835609980F
:10BDE800854713090998F5D2035704003697C166A9
:10BDF800E3CDE6FC91659385257031459740FB1F9F
:10BE0800E780C023AA84CD4769D131468145974050
:10BE1800FB1FE780804783570400835509000146CC
:10BE28000147B386E500C206C182636BF702AE978D
:10BE3800C207C18319C22310F90023A004002146B8
:10BE4800A285138544009740FB1FE780E03CB72795
:10BE58000020938787A0984311EF84C38147B5B723
:10BE680050401315470005072A962315D6000546A6
:10BE78004DBF3E871C43F5FF04C381BF011106CEA9
:10BE880022CC26CA4AC809E98944F2406244268578
:10BE98004249D244056182802AC62A84280036890C
:10BEA8002314B1002305C100EFF07FECAA8471FDD3
:10BEB800E30D09FC8357A400E1DB91659385557078
:10BEC80031459740FB1FE780601715C58357A400CD
:10BED80023200500232425012312F500B72700207D
:10BEE800938747A1984301E788C345B73E871C431A
:10BEF800F5FF08C359BFCD4449BFB7270020938732
:10BF0800C79F03C7070015E305472380E700058996
:10BF180009CDB7260020372500209386469541464F
:10BF28009145130545916FF07FF501458280B7274C
:10BF38000020A38AA7968280C167FD176315F500C4
:10BF48002E856FE04F91411106C6EFE0CF8A11C5EB
:10BF5800FD572310F50023010500B24041018280FE
:10BF680001114AC806CE22CC26CA85472A8963937E
:10BF7800F5044A85EFE04FBE39E9C16437D60600BB
:10BF88009385F4FF1307E1008946130646CB054560
:10BF9800EFE0DFD92A84FD140DC44C444A85EFF044
:10BFA800BFF90356E10022858146A685EFF08FA2EE
:10BFB8002A84DDB789476396F5008545EF20403F21
:10BFC8004DD9F2406244D244424905618280EFE093
:10BFD800AFB365B7011126CAB7240020938484CF74
:10BFE80022CC03C59400372400201304C4A0B7272B
:10BFF80000203727002006CE4AC84EC6232004005A
:10C0080023A807A0232007A049C9138907A19307DC
:10C01800200C3305F502916593851570930907A0E7
:10C028001905420541819740FB1FE780200103C69F
:10C0380094009307200C81453306F60208C01906C0
:10C048009740FB1FE78060241C4003C7940081458C
:10C058009386870B7D5563ECE5069306800BB30644
:10C06800D7020146FD550507B6972320F900BE867D
:10C078002390B600A381B6002381B6002382060070
:10C0880005069906E366E6FEF9562390D700994619
:10C098003307D702BA9723A0F90037A50400130580
:10C0A800856CEFC0FFD037B5040013058589EF70A4
:10C0B800AFB637A5040013050563EF208026F240CC
:10C0C8006244D2444249B2490145056182802394C1
:10C0D800A6F41386C6F423100600232406003106AE
:10C0E800E31BD6FE85059386860BB5B7411106C6B8
:10C0F80022C42A84EFC00FADEFD03FF8B727002045
:10C10800238A8796B727002003A507A0EFD0BFF49E
:10C11800B7270020238187982244B24037C50400FE
:10C12800130585F641016F20C01F93970501C1874C
:10C1380063D30734B727002003C54797797122D402
:10C148005AC806D626D24AD04ECE52CC56CA2E8BC4
:10C15800EF501FB92A8429C9034705009307000B2C
:10C168006311F704B72400208547938444A0A304EF
:10C17800F1009C4023150100A9E7EF00007F9165BD
:10C18800938535709740FB1FE78040EB88C015E921
:10C198008347910099C78345440013058400EFD075
:10C1A800CFA42285EF50BFA7B25022542165334552
:10C1B800AB0092540259F249624AD24A424B456155
:10C1C8008280372A00206146814513054AA9974095
:10C1D800FB1FE780800B03494400894793044AA961
:10C1E800D289930A4AA96314F906EF0000782390CC
:10C1F800A4000355240093054AA9EF705FA70357CD
:10C20800240083D704008356840011ED63E4F6000C
:10C218002314F400835584003A85EFC01FBA2285A1
:10C22800EFC07F8CB5B763E4F6002314F40083579E
:10C238008400D945938649A90D463A852390FA008A
:10C24800EFC07FA28D4561DD138549A9D1A099472B
:10C25800631AF9029305A1002285EFF08FC8AA841A
:10C268005DDDD9476396F40E05090355240013795B
:10C27800F90FD945938649A94A86EFC0DF9ECA853A
:10C2880059DDD9B7A1476318F9009305A1002285A4
:10C29800EFF03F93E9B7A947631FF90603558400F8
:10C2A8006C00EFE06FE12A89630D05140355240043
:10C2B80041669306E10055477D16AD45EFC09FB531
:10C2C800C8C0AA8649C1834844000358E100035600
:10C2D800C10003552400814713074AA9CA85EFE026
:10C2E8009FFBAA84631E050E0355240093054AA9E3
:10C2F800EF70BFB80DD50355240093064AA92D4603
:10C30800D945EFC05F96E30C05F0AD4513054AA982
:10C31800EFD0AF8D29B7B147631BF90E03558400E1
:10C328006C00EFE06FD9AA8469CD035524004166FB
:10C338009306E10059477D16B545EFC0BFAD23A26E
:10C34800AA00AA8629E983578400C5442315F10069
:10C3580003471400D147E304F7EC8347440003552F
:10C368002400938549A92380FA008357A1002382DA
:10C378009A002391FA00EF704FAFE30205EA0355E4
:10C388002400938649A90546D945EFC0DF8DE30807
:10C3980005E8854555BD834844000358E1008357A7
:10C3A800A4000356C10003552400A68513074AA913
:10C3B800EFE07FEEAA840DE50355240093054AA912
:10C3C800EF707FB1E30D05E403552400D9459306CA
:10C3D8004AA93546EFC03F89B545E30205E4ADB546
:10C3E800D9476393F400814403A54A009740FB1F93
:10C3F800E78000D3E38504E2835784002315F10026
:10C4080081BF8357840085442315F10091B7B9474C
:10C418006318F9009305A1002285EFF06F9681B5A6
:10C42800C1476318F9009305A1002285EFF02FDAC0
:10C438003DB5C947631AF900130691009305A10099
:10C448002285EFE06FF921BDD947631DF9009305F7
:10C45800A1002285EFE06FE7AA84E31405E0A304B6
:10C46800010075BBE147E31CF9DA9305A1002285B9
:10C47800EFE0CFD3EDB301458280EDC2011152C484
:10C488002E8A854522CC4EC656C206CE26CA4AC832
:10C49800AA8AB6893284EF10B071D1471DC5B72773
:10C4A80000203727002083C707A2834617A28144AC
:10C4B80019E0B684BE8637270020032787A1939703
:10C4C8004400BA9763EDD400D547F2406244D244A1
:10C4D8004249B249224A924A3E85056182803E8994
:10C4E800C10703D727FF09C7850493F4F40FD9BF01
:10C4F80025C09565938525C0130500029740FB1F4D
:10C50800E780C0B32326A90061D113060002814544
:10C51800938404049740FB1FE78020D723119900D8
:10C5280023000900231359011DC43727002083471E
:10C5380094000326C7C52304F900118C8327C9007A
:10C5480011841180238E870023A029018147B5BF5C
:10C5580023260900F1B723044901FDB785473E8525
:10C568008280B727002083C507A2B727002003A72A
:10C5780087A181476395F5008146368582800356F9
:10C588002700BA8619C2E30AA6FE850793F7F70FB4
:10C598004107CDB7B727002003C607A2B727002059
:10C5A80003A787A181476315F600814636858280F7
:10C5B80083552700BA8689C583454700E388A5FEC9
:10C5C800850793F7F70F4107F9BFB727002083C501
:10C5D80037A2B727002003A7C7C581476395F50091
:10C5E80081463685828003560700BA8619C2E30A57
:10C5F800A6FE850793F7F70F4107CDB7B7270020A9
:10C6080003C817A2B727002083A787A1014763158E
:10C61800E80081463685828003D62700BE8619CA7F
:10C6280003D667006318A600D04709C6035626003C
:10C63800E302B6FE05071377F70FC107C9BF41111B
:10C6480022C4404526C206C6AA8415C0484409C566
:10C658009740FB1FE780C0AC484809C59740FB1FBF
:10C66800E78000AC22859740FB1FE78060AB2685FA
:10C67800414681459740FB1FE78020C1B2402244D4
:10C68800FD57A384F400924441018280011122CC19
:10C698002A840355250006CE2EC6EF10501A3246BE
:10C6A80022858145EF00B07222856244F24005611F
:10C6B8006FF0FFF80DC503572500411122C406C6C7
:10C6C8002A8411CBDD45EF00707422852244B240E4
:10C6D80041016FF0DFF6B24022444101828082803E
:10C6E800411126C2B1469304C5FFB386D402B727C9
:10C6F80000201387C7C606C622C436978356A700EC
:10C708006398B60248430DC51384C7C69307F00F54
:10C718006306F60083470500639CC7009740FB1F2C
:10C72800E78000A0B147B387F402A29723A20700CD
:10C73800B2402244924441018280411122C42E8495
:10C7480026C24946AA848145228506C69740FB1F12
:10C75800E780A0B3A5C083C7C40113974700B727D4
:10C76800002083A7C7C5BA9703D707002310E400A2
:10C7780003D7270083D767002311E4003727002059
:10C788000357E7A12312E40003D704002313E400AE
:10C7980003D724002314E40003D744002315E4003E
:10C7A80003D764002316E40003D784002318F40099
:10C7B8002317E400B2402244924441018280B72703
:10C7C800002083C507A2B727002003A8C7C5B7273D
:10C7D800002003A687A1014781476394E5003E85B1
:10C7E80082808346060081CE544691CA83C6C6011C
:10C7F8009206C2966315D500850793F7F70F0507CC
:10C808001377F70F4106D1BF130600643386C502BC
:10C8180093069500AA8537C504001305C56B6F50AC
:10C82800FFC2411122C406C62A8403459500EF5071
:10C838007FDCFD57A304F400B2402244410182800A
:10C84800011122CC4AC84EC652C456C25AC006CE9E
:10C8580026CA2A89AE890144372A0020B72A00202F
:10C868001D4B83471AA26365F40463990902B7292B
:10C878000020372A0020930AF00F83C709A26367B4
:10C88800F4061144A1442285050442041306F00F5E
:10C89800CA854180EFF0DFE4E31794FEF24062447A
:10C8A800D2444249B249224A924A024B05618280E7
:10C8B80083A78AA193144400BE9483C704009DC330
:10C8C80083D76400639027036396690103D5240026
:10C8D800EF10E07626854E868145EF00504F26857D
:10C8E800EFF0FFD505041374F40FA5BF83278AA1C1
:10C8F80093144400BE9483C704009DC383C7940067
:10C908006380570383D76400639C27012685EFF073
:10C918005FF12685D145EF00704F2685EFF03FD2B5
:10C9280005041374F40F91BF41677917630BE5028F
:10C93800411122C406C685472A846399F5002285D9
:10C948002244B240814541016FF09FEF89476396C9
:10C95800F5008545EF10D0257DD1B2402244410134
:10C96800828082809D456FF0BFEDB727002003D5F8
:10C97800E7A18280B727002003C7C7A1011106CE0F
:10C988002317A1002316B10085476318F70070002C
:10C998009305E1000545EF50B068F24005618280DB
:10C9A800A947631CF60483C7150003C70500A2073F
:10C9B800D98F2310F50083C7350003C72500A207C8
:10C9C800D98F2311F50083C7550003C74500A20777
:10C9D800D98F2312F50083C7750003C76500A20726
:10C9E800D98F2313F50083C7950003C78500A207D5
:10C9F800D98F2314F500014582800545828091472F
:10CA08006314F60283C7150003C70500A207D98F70
:10CA18002310F50083C7350003C72500A207D98F67
:10CA28002311F50001458280054582809387C5FF63
:10CA380093960701C1820D476360D7023147B387D8
:10CA4800E702372700201307C7C6BA972381A70034
:10CA58002390B700014582800945828093064020D3
:10CA680037270020AA8763F4A60093074020F11710
:10CA7800231FF7A0B72700202381B7A2B7270020DC
:10CA88002382B7A2828019059565420541119385D5
:10CA980035C0418106C69730FB1FE780205A11C573
:10CAA800B240E95541016F504F90B2404101828038
:10CAB800B7270020238107A2B727002079710547EF
:10CAC800238E07A0B72700202384E7C64ECEB727BA
:10CAD8000020B729002022D426D24AD037240020AB
:10CAE800B7240020A38207A237290020B7270020F7
:10CAF800938939A206D652CC2AC6230004A2A38061
:10CB080004A2239F07A0232C09A023800900EF106B
:10CB1800C05B3245B7270020130600032380A7C651
:10CB2800372500201305C5C681459730FB1FE780D0
:10CB3800C075372A00200345CAC9130404A2938488
:10CB480014A2130989A115CD9565938545C01205D1
:10CB58009730FB1FE780804E37270020232EA7C47D
:10CB68000DC10346CAC99307CAC983C717002380E2
:10CB7800C900814512062380F4009730FB1FE78027
:10CB8800C070B727002003C507D083C70400956588
:10CB9800938555C03E951375F50F2300A400120523
:10CBA8009730FB1FE78080492320A90049C5034629
:10CBB8000400814512069730FB1FE780006D0327AC
:10CBC800090083460400814725077D56639EF604C5
:10CBD800EF108074B1473305F5029565938565C0FC
:10CBE800420541819730FB1FE7804045B727002069
:10CBF80023A2A7C62A8401CDEF100072314633065E
:10CC0800C502814522859730FB1FE78000682254C2
:10CC1800B25092540259F249624A37D504001305BA
:10CC2800059345616F10E06F85072300C70093F7F0
:10CC3800F70F410761BF230004002380040049BFA8
:10CC480041119397050126C206C622C44AC0C1876E
:10CC5800AE8463D1070A37290020034509C6EF507F
:10CC68002F882A8429CD03470500930700096315F7
:10CC7800F70403471500CD47631CF706B7260020C5
:10CC88000348250003C536B437270020834727A269
:10CC98001306640081458146130727A2AA886318F2
:10CCA800D80299C12300F7008347070091C70345BD
:10CCB80009C68545EF506FC52285EF405FF62165AF
:10CCC800258DB24022449244024941018280834525
:10CCD8000600AE9793F5F70F93F7F80F63F4A500E6
:10CCE80093F7F50F850693F6F60F0906854545BFB8
:10CCF800012DD9B793F715000145E1D7EF00107062
:10CD080009CDB727002083C727A281CBB7270020EA
:10CD180003C507C68545EF504FBF13C5140055B767
:10CD280085462A8763FBC60483C7150003C605002A
:10CD3800A207D18F2310F500639CD70083C7350065
:10CD480083C62500A207D58F2311F50001458280EF
:10CD5800894601456394D70283C7350083C62500F9
:10CD6800A207D58F2311F70083C7550083C6450056
:10CD7800A207D58F2312F70082800545828091474C
:10CD88006314F60283C7150003C70500A207D98FED
:10CD98002310F50083C7350003C72500A207D98FE4
:10CDA8002311F5000145828005458280914763146F
:10CDB800F60283C7150003C70500A207D98F231001
:10CDC800F50083C7350003C72500A207D98F2311B3
:10CDD800F5000145828005458280A1476314F60469
:10CDE80083C7150003C70500A207D98F2310F500D4
:10CDF80083C7350003C72500A207D98F2311F50083
:10CE080083C7550003C74500A207D98F2312F50031
:10CE180083C7750003C76500A207D98F2313F500E0
:10CE280001458280054582808947631CF60083C7D7
:10CE3800150003C70500A207D98F2310F500014587
:10CE48008280054582808357260079714ECE06D6AA
:10CE580022D426D24AD01307F007AE896372F702AC
:10CE680009473AC42316F100300093F5F50FEF1087
:10CE7800E01BB250225492540259F2494561828013
:10CE880003574600D9462A89328463F8E600835757
:10CE9800660063F4F6006379F7002314010030009C
:10CEA80093F5F90F4A85E1B70355060002C4EFF080
:10CEB800CFF1AA8459C1EFF09F9083C784006369BA
:10CEC800F5001146A246CE854A85EF10A00B55B74E
:10CED800340026869305F00F4A85EFF00FDA75F1D6
:10CEE800A24703578400DC472390E7000357240038
:10CEF8002391E700035744002392E7000357640097
:10CF08002393E70003D744002394E700DC4485CB50
:10CF180093F4F90F2286A6854A858297C167FD1783
:10CF28002A86E311F5FA22459947F9452300F500C9
:10CF380023029500EFF05F8D2DBF094661B70146CA
:10CF480051B7A947631CF60483C7150003C705003A
:10CF5800A207D98F2310F50083C7350003C7250022
:10CF6800A207D98F2311F50083C7550003C74500D1
:10CF7800A207D98F2312F50083C7750003C7650080
:10CF8800A207D98F2313F50083C7950003C785002F
:10CF9800A207D98F2314F5000145828005458280B8
:10CFA80083C705002300F50083C71500A300F5001B
:10CFB80083C7350003C72500A207D98F2311F500C1
:10CFC80082802322050003C7450089476304F700D0
:10CFD8000545828083D665000D47E37BD7FE9C45D7
:10CFE800011106CE22CC26CA4AC84EC683C41700F1
:10CFF80003C60700A204D18C138644006311D6042B
:10D0080003C4370083C72700AE8922045D8C9307C9
:10D01800C4FFC207C1832A89636FF70003A589008B
:10D028002311990023108900F155EF401FB82322DE
:10D03800A900014531A02285EFF0AFD265F1054581
:10D04800F2406244D2444249B24905618280397152
:10D0580022DC2E84834704004AD806DE26DA4ED620
:10D0680019472A89B285639AE706034624002800EF
:10D07800EFF0FFD0AA8415E903558100EFF06FCED9
:10D08800AA898345140015C937E704002E861307BB
:10D0980047F634009D454A85EF00D0424E85094643
:10D0A800814535234E85EFF08FD9F250625426859D
:10D0B8004259D254B2592161828089472310F10024
:10D0C800835781000A862311F1008357A100231298
:10D0D800F1004A85EF009075C9BF4947639DE70293
:10D0E800035624002800EFF05FCFAA845DFD3725A2
:10D0F80000201305C5C68357C50099E3814475B759
:10D1080003471400834604000345E5003C0001463C
:10D11800CA85912659BF51476390E70203562400F8
:10D128002800EFF0FF87AA8449F1834514003000F6
:10D138004A85EFF05FD195BF59476393E7060356D9
:10D1480024002800EFF0BF8BAA8425F183558100C5
:10D158004A85EFF0AFCA1DC958458356A1008357C9
:10D168000700B697C207C1832310F700C1DB5C47ED
:10D17800D1D7B727002083C727A2C9D3B727002054
:10D1880003C507C68545EF405FF805B789473EC028
:10D19800835781000A86834514002312F10015BFC6
:10D1A800834514000A8623100100EF003068B9B7E0
:10D1B8005D71A6C256DA86C6A2C4CAC04EDE52DC6B
:10D1C800AA8A03C51500AE8432C6EFF0AFBCB245DB
:10D1D80001ED8144B6402644268506499644F25915
:10D1E800625AD25A61618280230205002311050028
:10D1F80083C9040085472A84639AF90003C624007A
:10D208002808EFF0FFB1AA8405492DA09D47639433
:10D21800F904034705008D47E31DF7FA03C6240008
:10D2280028080549EFF09FB8AA8409E50546814515
:10D238002285712E2285EFF0CFDE034584003C085D
:10D248000147CE862686D6853924E30509F8228546
:10D25800EFF0EFBE41B7CD47639DF90003470500E6
:10D268009147E318F7F603C624002808EFF0DFBB60
:10D2780059BFD547E39FF9F4034A05008947E31AE4
:10D28800FAF403C6240028080549EFF09FCBAA84C6
:10D2980055F183570102BDE3035781011306F003DB
:10D2A8005C44930607FCC206C182636CD600035631
:10D2B800A101D94663F7C6008356C101D94563EF7A
:10D2C800D500035524002391E7000549EF003057A6
:10D2D80003560102D2852285692CA9BF8355E10135
:10D2E8002391E7002392C7002390B7002393D70028
:10D2F80085472300F400014A0149D9BF014AC9BF43
:10D308007971AA8522D426D203542500AA84280834
:10D3180006D6EFF01FCBF24599E535E9854522851C
:10D32800EFF04FE5C1A0835781011547639BE706DE
:10D338000357A1018D4763FCE7046800EFF05FC65F
:10D348000357E100DD4763FCE7008345D100B707D9
:10D3580017008507100822853EC8EF00304D835717
:10D36800E1000357A10191076305F7002285EFF05B
:10D378006FDF8347C10072466C00858B11062285DA
:10D3880091CFEFF0FFE201C52285EFF0AFDD8844D1
:10D3980051D59730FB1FE780A0D849B7EFF03FCBB6
:10D3A800DDB711476389E7001387A7FF4207418369
:10D3B800854663EEE6023147F117B387E702372760
:10D3C80000201307C7C6BA9703D7070069D303C558
:10D3D80027003008A2850D205DF903578101914788
:10D3E800E31EF7F2B25022549254456182802C0811
:10D3F8002285812E49FDFDB701114AC82A89314588
:10D4080026CA06CE22CC2EC6B284EF407F8631C112
:10D41800B2459307000A2310F5002311B5002A84AA
:10D42800214611058DC0A6859730FB1FE780C0DE19
:10D43800A2854A85EF40DF920145F2406244D2441A
:10D4480042490561828081459730FB1FE780E0E310
:10D45800C5B70545DDB7797126D2AA841305000240
:10D4680006D622D42ECE32CC36CA3AC83EC6EF40B3
:10D478003F8031C96246F2454247D246B2472A84C4
:10D48800130520FA2300A400A300C4002311B4004C
:10D498002302E400A302D40013058400614691CF5F
:10D4A800BE859730FB1FE78020D7A2852254B25053
:10D4B8002685925445616F40BF8A81459730FB1F8E
:10D4C800E780A0DCDDB7B2502254925445618280D7
:10D4D8005845797122D406D62A84AE8649C3835723
:10D4E8002700231DF10093072006639FF504B72743
:10D4F800002003D6E7A1835767006373F600B2875D
:10D5080013F6F70F83552701834707018D8F93F78C
:10D51800F70F81E5890793F7F70FB297FD17B3C7A0
:10D52800C702231EF1008357240083556400034576
:10D538008400231CF10001473C080146EFF0BFF1CD
:10D54800B2502254456182800347C701B7270020A3
:10D5580083A7C7C51207BA9783D76700D9B72EC65E
:10D568001946814528089730FB1FE78000D2B2464C
:10D578005DBF797122D406D626D22A848DC181470F
:10D588000147930600062E868355640003458400F0
:10D59800EFF07FECB2502254925445618280B284FD
:10D5A800280059469730FB1FE78020CE23149100AE
:10D5B80089E88357240048446C002315F100EFF0F4
:10D5C800CF973C00014793060006014675BF797165
:10D5D80006D6814799ED8357250058452316C10083
:10D5E8002314F1003C0011C7835727002315F100CD
:10D5F8003C002E8683556500034585000147930648
:10D608000006EFF05FE5B25045618280411122C407
:10D6180006C68347050011472A846395E7022E86CC
:10D62800835565000345850081470147CD46EFF0E6
:10D638009FE24946835564002244B24015454101A2
:10D648006FF00F8A13F7B70F89466317D7000146A3
:10D65800EFF03FF25146F9BF0D476398E7002244C7
:10D66800B240014641016FF09FF6B24022444101A9
:10D67800828003D70500B146B7270020711733070A
:10D68800D7029387C7C6BA97D84319EBD8412395D1
:10D69800A7000145D8C303D725002394E70082805B
:10D6A80059458280797122D4404526D24AD006D67F
:10D6B800AA842E8925C0484419C59730FB1FE780E6
:10D6C80020A6232604008357040083D5640003C5DD
:10D6D80084002315F1008357240001479306400670
:10D6E8002316F100835784004A862317F1001C484B
:10D6F8003EC883D724002314F1003C00EFF0BFD5C7
:10D70800A30E240123280400B25022549254025933
:10D71800456182802800314681459730FB1FE780AC
:10D72800C0B683D7240083D5640003C584002314BE
:10D73800F10001473C00930640064A86EFF0BFD14E
:10D74800E1B7797152CC2A8A03D5050026D206D6CC
:10D7580022D44AD04ECE56CAAE84EFE09FE019E1FB
:10D768008547BDA84045AA8965DC83576500E399CC
:10D7780047FF83578400638707128346C401B72A8B
:10D78800002003A7CAC59206FD173697C20703579C
:10D798006700C1832314F4006316F700930530066D
:10D7A800EFF01FD35C48A5EFC84003491500834735
:10D7B800050022093369F90083D7240013072900DB
:10D7C800631AF702F955EF404FBEC8C023912401F0
:10D7D80003C589002686D285EFF01FC2814721E163
:10D7E800B250225492540259F249624AD24A3E85B2
:10D7F800456182809565938515C04A859730FB1FE2
:10D80800E780C08348C8C840231C2401F955EF406D
:10D81800CFB983D72400C8C0F9172391F40048482A
:10D8280059C503D624008356A401835784013308BD
:10D83800D60063C007090347C40183A7CAC5954535
:10D848001207BA9783D7270063CF0705CC403695D0
:10D858009730FB1FE780409C0357A40183D724001F
:10D86800BA97C20703578401C183231DF400E399C3
:10D87800E7EE03D7290003C5890030002314E1002F
:10D888005848D2852315F1003AC6EFF0FFB611C506
:10D8980048489730FB1FE780A088232A0400232CE0
:10D8A80004007DBD99454E85EFE05FDE55BDA54579
:10D8B800DDBF9145CDBF03D725007DC3B727002025
:10D8C80083D6E7A1ED4763EEE60C011122CC2E8446
:10D8D80026CAAA844840914506CEEF400FAD83572B
:10D8E8002400AA862300F50083572400A183A300FF
:10D8F800F500835704002301F50083570400A18332
:10D90800A301F50003562400C167F9171106420662
:10D9180041826396F4042AC4314532C6EF404FB5BC
:10D92800AA85CD471DC5930700F92300F5003246A7
:10D93800F957A2462311F50089472302F500B727B6
:10D9480000202313C50014C503C507C6EF404FC107
:10D958008147F2406244D2443E8505618280814518
:10D968002685EF40107EAA8711E9B726002003C755
:10D9780026A265D37D172381E6A2E1BF0947630488
:10D98800E5021D476303E50249476302E5027D4757
:10D99800E311E5FCB726002003C726A28147D1BFC3
:10D9A800ED473E858280D1476DB791475DB789477E
:10D9B8004DB701114AC831471309C5FF3307E902BA
:10D9C800B727002026CA9384C7C606CE22CCBA94AD
:10D9D800D84029CB1384C7C6B727002083C627A2FF
:10D9E800854795CA2314A10083D7840003D5A400D2
:10D9F8002C003AC62315F100EFF0FFEB11C5C84023
:10DA08009720FB1FE780C071B147B307F902A297BF
:10DA180023A207008547F2406244D24442493E852A
:10DA2800056182808147C5BF797126D24445372771
:10DA380000204AD083D764000359E7A152CC06D608
:10DA480022D44ECE56CA2A8A63F327013E8903D7C9
:10DA5800240142091359090183D7040141CB998F45
:10DA68004A8463D52701139407014180894522859B
:10DA7800EFF06F81AA89CD4A25C183D724002AC631
:10DA8800231581002314F10083D7240185E383D76C
:10DA98000401930925002300F50083D70401A1831D
:10DAA800A300F5006376240503D4040183D7240179
:10DAB800CC4422864E85BE959720FB1FE780C07513
:10DAC80003556A002C00EFF01FDFAA8A15C54E85A2
:10DAD8009720FB1FE780C064B250225456859254A9
:10DAE8000259F249624AD24A4561828089078DBF4C
:10DAF8007914420441805DBF03D7240183D7040011
:10DB08003A94FD17C207420403D70401C183418038
:10DB18002390F400239984006377E400D5FFFD5730
:10DB2800A38EF40055BF81455285EFF0BFB76DB79E
:10DB380079714AD03729002052CC034A59A222D4FD
:10DB480056CA5AC85EC662C406D626D24ECE52847B
:10DB5800B72A0020054B930BF00F372C002083A722
:10DB68008AA193144400BE9483C90400639D690785
:10DB7800DC44B5CBD84725CB03D7070029CBB7273B
:10DB8800002083C727A299CF2685EFF0FFE9AA8551
:10DB980015E9B727002083C717A205046351F402CB
:10DBA800A30289A2B25022544E8592540259F249D6
:10DBB800624AD24A424BB24B224C45618280A30250
:10DBC80009A2CDB72685EFF0FFAD8149E1BF83C734
:10DBD800D701639A7701930520062685EFF05F8FBA
:10DBE800DC44A38E070083471CA205041374F40FBA
:10DBF8006363F4000144E31444F7C1BF41111545C0
:10DC080006C6EFF01FDB09C50545B2404101828019
:10DC18001945EFF01FDA6DF91145EFF09FD96DF551
:10DC28001D45EFF01FD96DF1B727002083C717A254
:10DC3800E9DFB24041016FF0BFEF83D705000D4720
:10DC4800F117C207C1836365F706DC41B5C341110B
:10DC580022C42E84854526C206C6AA84912F39C9B6
:10DC68002685AD25C167F9176381F40219ED83573D
:10DC7800240081CF8356040019476393E6043727AD
:10DC880000200357E7A163FDE702B727002083C7F9
:10DC980027A2A285268599C72244B2409244410111
:10DCA8006FF07FC12244B240924441016FF07F9CE3
:10DCB800094582805145B240224492444101828004
:10DCC8006D45D5BF397126DA4ED6AA84AE895D4531
:10DCD80089454AD806DE22DC328936C63AC4EFE0E6
:10DCE8009FDA35C522472A84014511C7B246130574
:10DCF8004400B68502979357850023003401A3009A
:10DD08002401A301F4009547231CF100B727002044
:10DD180083C727A22301A4001105231DA10022CE39
:10DD28002C08268595C3EFF01FB9AA8411C5228552
:10DD38009720FB1FE780C03EF25062542685425967
:10DD4800D254B25921618280EFF0BF92F9BFCD441D
:10DD5800E5B7797126D24AD052CC56CA06D6BA8AC5
:10DD680022D44ECE19472E89B284368A639DE506A1
:10DD7800035526000944EFE0CFFE2AC62DCD5C45A9
:10DD88008359650083D727002390F400B247B7264C
:10DD9800002015472380570103C686C62391E70054
:10DDA800130716001377F70F2384E6C62382C700EC
:10DDB80001E705472384E6C65147631AE90015477A
:10DDC8002391E400DC4703D784002394E7005287BB
:10DDD800A686CA854E85EFF0FFEE2A84324515C423
:10DDE800EFE0FF8509A842867400BE85AA89EFE0A6
:10DDF800CFE82A8441DD2285B25022549254025938
:10DE0800F249624AD24A45618280F945EFE0DF9FD4
:10DE1800DDB783D705002300F50083D70500A1836C
:10DE2800A300F50083D725002301F50083D725003B
:10DE3800A183A301F5001145828083D70500230043
:10DE4800F50083D70500A183A300F50083D725003B
:10DE58002301F50083D72500A183A301F50083D70B
:10DE680045002302F50083D74500A183A302F500EE
:10DE780083D765002303F50083D76500A183A30337
:10DE8800F5002145828083D705002300F50083D75C
:10DE98000500A183A300F5000945828083D705000A
:10DEA8002300F50083D70500A183A300F50083D7DD
:10DEB80025002301F50083D72500A183A301F500E0
:10DEC80083D745002302F50083D74500A183A30229
:10DED800F50083D765002303F50083D76500A18388
:10DEE800A303F50083D785002304F50083D78500B5
:10DEF800A183A304F5002945828003D70500854640
:10DF0800AA872300E50003D705002183A300E500C5
:10DF180003D70500631DD70003D725002301E500BB
:10DF280003D725002183A301E50011458280094517
:10DF38006315A70203D7250019452381E70003D7F6
:10DF480025002183A381E70003D745002382E7004A
:10DF580003D745002183A382E700828083D7050089
:10DF68002300F50083D70500A183A300F50083D71C
:10DF780025002301F50083D72500A183A301F5001F
:10DF880011458280797126D24AD04ECEB2842A8930
:10DF9800AE8929468145480022D406D63684972082
:10DFA800FB1FE780802E231691008DEC83572400F9
:10DFB8002312F100B727002083D7E7A12314F1002B
:10DFC8005C448DC383C6C701372700200327C7C514
:10DFD800920683D787003697035727002315F10049
:10DFE8002313E10037E704004A85130747EA540082
:10DFF80013F6F90FD545EFF0FFCC2A8911C19DE042
:10E0080085472300F4002302040001468145228548
:10E01800EFF02FD6B25022544A8592540259F24951
:10E02800456182802285EFE08FE1EDB737E7040094
:10E03800B286130727F02E8685456FF0BFC80111F9
:10E048002317A100B7E60400416570000148930753
:10E05800F00F0D479386A6E199457D1506CEEFF0A2
:10E068005FCFF24005618280B7E60400B2870148BD
:10E078002E861147938626E4C9456FF09FCD37E772
:10E088000400B2861307E7E82E86CD456FF09FC3DC
:10E09800011122CC37240020130444CA26CA4AC8D6
:10E0A8004EC606CE2A89AE89930404031C4081C754
:10E0B800CE854A8582971104E31A94FEF2406244A1
:10E0C800D2444249B2490561828041113727002074
:10E0D80022C406C626C2130747B38347C7030345AE
:10E0E800D70337240020130484CFA304F400AA978D
:10E0F80093F7F70F2304F400A5CF1305C003338566
:10E10800A702A5658505B72400209720FB1FE78097
:10E11800E0F2034684009307C00381453306F60204
:10E1280023A0A4CA9720FB1FE780201683A704CA50
:10E1380083468400014789077D566341D7022244FC
:10E14800B240924437250020130600038145130589
:10E1580045CA41011723FB1F670023132390C700FB
:10E168002381070023A5070205079387C703F1B793
:10E17800B2402244924441018280B727002003C65E
:10E1880007D0B727002003A707CA81476315F60001
:10E19800814636858280BA861307C703835567FC94
:10E1A800E389A5FE850793F7F70FCDB7011122CCB8
:10E1B8002EC632C406CE2A84EFF03FFC2246B24572
:10E1C80011E9C167F9176303F4005145F24062444D
:10E1D8000561828054558347450095C213F727018E
:10E1E80041456314A700154575F2C18B3D45F9DF1C
:10E1F80083C7A6010145E3FBB7FC3145C1BFC18B0D
:10E208000145E9F71545D9B7797126D24AD0B7241F
:10E218000020416922D44ECE52CC56CA5AC806D6DE
:10E22800AA890144938484CF372A0020930AC00323
:10E238007D19054B83C784006364F400014535A844
:10E24800B307540303270ACABA9703D727006316EC
:10E25800270105041374F40FF1BF03C557003000FC
:10E2680093856700EFB091561946CE852800972010
:10E27800FB1FE780A007E31E65FDB25022549254AD
:10E288000259F249624AD24A424B45618280B72715
:10E29800002083C507D0C166B727002003A707CA97
:10E2A800FD1681476395F500014632858280035843
:10E2B80027003A866306D80003480700E307A8FE4C
:10E2C800850793F7F70F1307C703E9BF411106C680
:10E2D800EFF0BFEA11C503554501B2404101828004
:10E2E8000145E5BFB727002083C607D0B727002020
:10E2F80003A707CA0145814711076393F600828087
:10E308000346070001C605051375F50F850793F742
:10E31800F70F1307C703D5B7B727002003C507D0E2
:10E32800828037270020930647CA8147130747CAC8
:10E3380031468C4291E58A07BA9788C301458280A5
:10E3480085079106E397C7FE4D458280411106C6B1
:10E3580022C4EFF09FE21DCD2A8403552500854590
:10E36800EFF01FD3485409C59720FB1FE78040DB17
:10E3780022851306C00381459720FB1FE780E0F044
:10E38800FD572311F400230204000145B240224442
:10E39800410182800945DDBF411106C6EFF0FFDD6E
:10E3A80011C50345C500B240410182800145E5BF62
:10E3B800C167F9176304F502411122C406C62E8409
:10E3C800EFF0BFDBAA87014591C703C54700698CF9
:10E3D80033358000B2402244410182800545828065
:10E3E800011106CE2EC6EFF05FD9854711C9035734
:10E3F8004501B24585476305B700231AB500814733
:10E40800F2403E850561828031CD01114AC84EC671
:10E4180037290020C16922CC26CA52C456C206CE6A
:10E428000144AA84130989CF372A0020930AC0031C
:10E43800FD1983478900634BF400F2406244D244DB
:10E448004249B249224A924A0561828033055403FF
:10E4580083270ACA3E958357250063833701829430
:10E468000504C1BF8280B727002003C607D0B7279D
:10E47800002083A707CAC166014589070147FD1621
:10E4880091456313E600828003D807006309D8002A
:10E4980003C8A7006315B80005051375F50F050730
:10E4A8001377F70F9387C703E9BFB727002003C681
:10E4B80007D0B727002083A607CA014781479106DE
:10E4C8006310E602858393C7F7FFC207C18305453A
:10E4D8006364E50285473395A70042054181828040
:10E4E80083C5060081C583D5C602CD8F050713777E
:10E4F800F70F9386C603E9B793F61700E1FE050503
:10E5080085831375F50FE9B7797156CAAA8A2E85DE
:10E5180026D24AD04ECE52CC5AC85EC662C406D65F
:10E5280022D4AE84328B368CBA8B3E8AC289468915
:10E53800EFF0BFC449E141657D15EFF01FC42A849F
:10E54800554531CC1946DE8513056400A3028401C4
:10E558009720FB1FE78040CC8357010323119400C9
:10E56800230264012319F400835741032300540153
:10E5780023260402231AF400230644012317340136
:10E5880023182401EFF07FF22318A402232A04029F
:10E598002685232C04028145EFF09FAF0145B25038
:10E5A800225492540259F249624AD24A424BB24B1F
:10E5B800224C456182804545DDB7B727002083C6D8
:10E5C80007D0B727002003A707CA81476395F6003D
:10E5D80041657D1582803A861307C703835547FF37
:10E5E8006395A500035526008280850793F7F70FEA
:10E5F800F1BFB727002003C807D0B727002083A69C
:10E6080007CA416601477D16954811436314E8001F
:10E618000145828083D7260036856380C704CC5A9B
:10E628008DCD83C7350083C5250089CD938597FD9A
:10E6380093F5F50FE37FB3FC9387D7FA93F7D70FDA
:10E6480089EF82809385F7FD93F5F50FE3F3B8FC26
:10E658009387D7FA93F7D70FCDDF05071377F70F0F
:10E668009386C60365B7B727002083C507D04166E0
:10E67800B727002003A707CA7D168147254863945A
:10E68800F50001458280835627003A85638CC600D1
:10E69800545B89CA83C636009386E6FD93F6F60F67
:10E6A800E372D8FE850793F7F70F1307C703C1BFB7
:10E6B800011122CC2A84494506CEEF60CFFD15C151
:10E6C8002AC62285EFF07FAB09CD6244B727002028
:10E6D800324683550503F24003C5B7CF05616F3055
:10E6E800BFC1F24062440561828039714ED652D46E
:10E6F800AE892A8A93053005414526DA4AD856D28A
:10E7080006DE22DC32C63689BA8A9720FB1FE780EC
:10E71800E092CD4431C92A8489446382090432468F
:10E728008145231AC10041469720FB1FE780E0B5C9
:10E738005686CE8522859720FB1FE780E0AD2146CF
:10E74800630E0902CA8528089720FB1FE780C0AC22
:10E75800A28650082C085285EF404010AA842285D2
:10E768009720FB1FE780C09BF250625426854259D0
:10E77800D254B259225A925A21618280814528087E
:10E788009720FB1FE78060B0E1B7411122C44059D0
:10E7980026C206C6AA8429CC085409C59720FB1F9F
:10E7A800E7800098285809C59720FB1FE780409705
:10E7B800685809C59720FB1FE7808096285C09C523
:10E7C8009720FB1FE780C095685C09C59720FB1F51
:10E7D800E78000950325040809C59720FB1FE780FB
:10E7E800209422859720FB1FE780809323AA0402A8
:10E7F8002244B727002083D50403B240924403C5BE
:10E80800B7CF41016F301FD8411126C206C622C4B6
:10E81800AE84EFF09F9621C54C592A84A9C183A8DC
:10E82800C50703A88507FC59B85983C6650003D6F0
:10E83800050083C525002685EF600FEE2285EFF0E1
:10E84800DFF4EFF05FE201CD2244B7270020B240A9
:10E85800924403C5B7CF854541016F301F8BB24045
:10E868002244924441018280011122CC06CE2A849E
:10E878002EC6EFF09F905C5991CF83D70700B24521
:10E88800639A870085476397F5006244F240056103
:10E898006FF0BFEFF240624405618280411106C605
:10E8A80022C426C2EFF0FFD421C54059AA8429C04A
:10E8B800834724008DCBB727002083A787CD89C73E
:10E8C800DC4399C322858297034734009307F002FB
:10E8D8006310F702224403D52400B24092448145D4
:10E8E80041016FF07FF2B727002083A747CDC1BF52
:10E8F800B2402244924441018280411126C24AC05A
:10E9080006C622C4AA842E89EFF03F8731C1405938
:10E918005DCC83570400639C970A83473400130730
:10E928001002639CE70883472400D9C37C5403275B
:10E93800040883D7470105E713F717000DC31854D8
:10E9480003574700058B01CF93072002A301F4006A
:10E95800B24022449244024905454101828013F79E
:10E96800270009CB185403574700098B01C79307A1
:10E978004002E9BF918B89CB1C5483D74700918B08
:10E9880081C793076002D9B7B727002083A787CD2F
:10E99800E1D3DC43D5DF2285829703473400930710
:10E9A800F0028145E316F7FA2685EFF0FFE54DB74B
:10E9B800B727002083A747CDE1BF1307A0026398BC
:10E9C800E7006304090013092003CA85F1BF631C2B
:10E9D80009002685EFF06FFA19C58347450093E7CC
:10E9E80007012302F500A6854A85EF50FFE78DB79A
:10E9F800797126D29947231DB100AA842E858D45A9
:10EA080022D406D632C636C4231CF100EFE0AF8705
:10EA18002ACE4D441DC13246A246AA853285829629
:10EA28002A8419E52C082685EFF02FA12A8411C520
:10EA380072459710FB1FE780A06E2685EFF05FC731
:10EA48002285B25022549254456182804111B70602
:10EA5800050022C42E862E8493868646894506C6DE
:10EA680026C24AC02A89EFF0BFF883450400AA8469
:10EA78004A85EFF07FD9B240224426850249924464
:10EA880041018280B727002083A747CD95CB9C43BF
:10EA980085CB1D71A2CC86CE984110082A843AC82D
:10EAA800D84185453ACA829701C92306A100035572
:10EAB80024006C00EFF09FF9F640664425618280DF
:10EAC8008280AE8715C5785505C783460700238021
:10EAD800D50083461700A380D500834627012381EC
:10EAE800D50083468701584BA381D500D8C18280C1
:10EAF800414681453E851713FB1F67000379B727F9
:10EB0800002083A787CD91C703A387006303030071
:10EB1800028309458280372700200327C7ED1DC7D8
:10EB28005843AA8705450DC703A50708411106C61E
:10EB3800930605021306050C93050506130505043F
:10EB48000297B2401375F50F410182800545828016
:10EB580082804DC9357122CD2A840355050026CB04
:10EB68004AC94EC756C306CF52C55AC1DEDEB68A59
:10EB7800B2892E89EFF06FE0AA8439C50C18228576
:10EB8800EFF03FF483472400138A6400A9CBEF50C9
:10EB98001FA72A8B014583CB5400EF505FA4AA849A
:10EBA8000C100818EF10806D08542C10EF10A06D91
:10EBB800D288268A56C05E88D2875A8714103010A9
:10EBC800CE854A85EF20D028FA406A44DA444A497B
:10EBD800BA492A4A9A4A0A4BF65B0D618280EF507D
:10EBE8001FA2AA8B014503CB5400EF505F9F2ACE8A
:10EBF80008540C10EF1080682C100818EF10A0684B
:10EC0800F2484DBF8280C14709CD1455C14791CA0A
:10EC1800785501CB83C73600BD4663F4F6008347B9
:10EC280087013E858280894763090510638705103F
:10EC3800411106C622C426C2834715002E842380AC
:10EC4800F50083472500A380F5008347350023811D
:10EC5800F50083474500A381F50083475500858B60
:10EC68009396870083D7450093F7F7EFD58F2392C4
:10EC7800F5008346550093F7F7DFA20693F60620C2
:10EC8800DD8E2392D5000347550093F6F6BF220781
:10EC980013770740558F2392E50083475500FD768B
:10ECA8009386F67F8D87858B758FAE07D98F2392D4
:10ECB800F50083466500F99B858ADD8E2392D50091
:10ECC800034765009377270013F7D6FF5D8F2392DC
:10ECD800E5008347650093F647009377B7FFD58F24
:10ECE8002392F50003476500DD9B4D45218BD98FA5
:10ECF8002392F500EF602F9AAA845145EF60AF99EF
:10ED08000347340093F4F40FC947636297021375FD
:10ED1800F50F636EE500834604001147E147636819
:10ED2800D7008346140005476363D7008147B24084
:10ED3800224492443E85410182803E85828015C1ED
:10ED4800AA8709458DC141112E8541469385170033
:10ED580006C69710FB1FE780204CB24001454101D1
:10ED6800828009458280828089471DC595C54111E9
:10ED780006C603471500AE8719462380E5009305AC
:10ED88002500138517009710FB1FE780E048B24065
:10ED980081473E85410182803E85828015C1AA87D0
:10EDA80009458DC141112E8541469385170006C638
:10EDB8009710FB1FE7804046B24001454101828021
:10EDC80009458280828089471DC995C9411106C6B7
:10EDD8000347250083461500AE872207558F2390E9
:10EDE800E500214693053500138527009710FB1F82
:10EDF800E7808042B24081473E85410182803E855E
:10EE0800828015C1AA8709458DC141112E854146C9
:10EE18009385170006C69710FB1FE780E03FB240B6
:10EE2800014541018280094582808280894719C94C
:10EE380091C903471500BD46E14763E5E600238015
:10EE4800E50081473E85828015C1AA8709458DC1A5
:10EE580041112E8541469385170006C69710FB1F62
:10EE6800E780803BB24001454101828009458280AC
:10EE7800828015C1AA8709458DC141112E85414659
:10EE88009385170006C69710FB1FE780E038B2404D
:10EE98000145410182800945828082801DC1AA877F
:10EEA800094595C141112E85130600049385170065
:10EEB80006C69710FB1FE7802036B2400145410186
:10EEC800828009458280828015C1AA8709458DC143
:10EED80041112E8541469385170006C69710FB1FE2
:10EEE800E7808033B2400145410182800945828034
:10EEF80082801D71A2CC2A84084586CEA6CA230624
:10EF080001008344050035479387F4FF93F7F70F13
:10EF1800636AF70C37C706008A0713078767BA972B
:10EF28009C4382870C08EFF01FD0C9476312F50293
:10EF380099472306F100035524006C00EFF01FB138
:10EF4800F6406644D644256182800C08EFF07FEBDA
:10EF580029C98347C100E5F303552400EFF04FF5B5
:10EF6800C5B70C08EFF05FEEE5B70C08EFF01FEC43
:10EF7800C5B70C08EFF0BFDCE1BF0C08EFF0BFE449
:10EF8800C1BF0C08EFF09FE1E1B70C08EFF0DFDD3F
:10EF9800C1B70C08EFF0FFED65BF834715002308E4
:10EFA800F10003552400EFF04F9DA1470DC1034721
:10EFB800C500631BF702B727002003A787CD9D472D
:10EFC80019C7184309C71008A6850297AA872306F8
:10EFD800F10041B70C08EFF07FEC9DBF0C08EFF093
:10EFE800BFEEBDB79D47B1B7B727002003A747CDF0
:10EFF800F9B7011122CC06CE26CA4AC84EC6034725
:10F008000500930720092A84631CF712834715001B
:10F0180039476395E70A83564500096761078147C1
:10F028006398E610B729002003A589CECE84630132
:10F0380005100C4403C90500631F09008347050038
:10F0480085052146A9CF29059710FB1FE780C01C1D
:10F0580083A784CEB5C34945EF209FC12A841DC527
:10F06800930710FC2300F500A300250183A584CE97
:10F078000905414689059710FB1FE780E01983A71A
:10F0880084CEA28503C51700EF209FCD03A584CEAB
:10F098009710FB1FE780C00823A404CE31A80905F8
:10F0A8009710FB1FE7804017EF30007B05494DF1B3
:10F0B80083A789CE2380270185479DA81307E003EE
:10F0C800639EE708034725009547631FF70203552A
:10F0D8004500EFF06FAC9147E310F5FEB72700202D
:10F0E80083A747CDF1DB03A38700E30703FC03569F
:10F0F800E40003554400930564006244F240D2449E
:10F108004249B24905610283A147631EF70083455E
:10F118006400035544006244F240D2444249B24973
:10F1280005616FF08FFD930600038147E301D7FE69
:10F13800F2406244D2444249B2493E850561828028
:10F148009306000A8147E315D7FEEFF09FDA0844DB
:10F1580025D59710FB1FE780A0FCB9BF8147C9BF21
:10F16800011126CA06CE22CC89441DCD95CDAA848C
:10F178002E8468008D45EF50AF988347E1002685BF
:10F18800228693F7F70393E707046C002307F1003F
:10F19800EF200043AA8409E90D466C0013053400EA
:10F1A8009710FB1FE7804007F24062442685D2444F
:10F1B800056182805D714EDE86C6A2C4A6C2CAC041
:10F1C80052DC56DA5AD85ED6894945CD5DCA138BCA
:10F1D8004500420B135B0B01AE8A2A8A9305300562
:10F1E8005A85B2849710FB1FE78040E52A84CD49F1
:10F1F80049C9EF50AFC22A895686D285935A8900E9
:10F20800135A0901937BF90F1305440093FAFA0F77
:10F21800137AFA0F135989019710FB1FE780E01141
:10F22800A301740123015401A30044012300240114
:10F23800EF502FBEAA85414608089710FB1FE780AC
:10F24800C00F214734005A86A2850808EF20E05DE8
:10F25800AA891DE121462C0023807401A380540152
:10F2680023814401A3812401138544009710FB1FC7
:10F27800E780A00CEF504FBB22859710FB1FE7805B
:10F2880020EAB64026444E8596440649F259625A09
:10F29800D25A425BB25B6161828001114AC82A89F5
:10F2A8002E8506CE22CC26CA2EC6EFE01FED71C5EC
:10F2B800405971C4834754000947B24593F6B70FC4
:10F2C8006387E60011471305E00F6392E708835749
:10F2D80004000945639DB706930484004146CA8526
:10F2E80026859710FB1FE78020F34146CA85130542
:10F2F80084019710FB1FE78020F2034734008546FE
:10F308009307F7FE93F7F70F63E9F6041306C403B0
:10F318003285C14532C6EF40BFFE32469306C4026D
:10F32800A6852285EFF0FF828347240089CB2285BA
:10F338006244F240D244424905616F10A01B034762
:10F348003400C947E305F7FEA301F4000145F24084
:10F358006244D24442490561828093071005014501
:10F36800E317F7FE83472400FDD322856244F24069
:10F37800D244424905616F10601E0945C9BF49451D
:10F38800F9B7397152D42A8A328526DA4ED606DE82
:10F3980022DC4AD8AE8932C6EFE03FDEC94459C5FF
:10F3A8004059C94441C48357040032466390C70892
:10F3B80083475400A18BB1CB372900208327C9ED9F
:10F3C8009304E00FA5C79C47B5C393048401268521
:10F3D8004146D2859710FB1FE78000E48327C9EDDB
:10F3E8008325040826869C479385050418088146CA
:10F3F8002E858297AA844146CE8508089710FB1F60
:10F40800E780C0EE93F4F40F11E189440347340018
:10F418009307B005631CF7002285EF10E0108347BF
:10F42800240091CF9307C005A301F400F250625461
:10F4380026854259D254B259225A216182809307B3
:10F44800E005DDB729CD011126CA06CE22CCAA8453
:10F458000945A9C10D4628002E848D059710FB1F6C
:10F46800E78080DB8347A10070002C0093F7F70347
:10F4780093E7070426852305F100EF20601419E9B6
:10F488000D46A28568009710FB1FE78020E67D15D2
:10F498003335A000F2406244D244056182800945B8
:10F4A8008280011152C42A8A32854EC656C25AC079
:10F4B80006CE22CC26CA4AC82E8BB28AB689EFE07D
:10F4C800DFCB09ED8944F240624426854249D244A3
:10F4D800B249224A924A024B056182805C592A89C4
:10F4E800C544F5F34D45EF501F9B1374F50F514577
:10F4F800EF507F9AE38809FC83C78901E3E487FC1E
:10F508001375F50FE360F5FC930530051305400806
:10F518009710FB1FE78080B2232AA9022A84CD44D2
:10F528005DD11306400881459710FB1FE780E0D5A1
:10F53800A3010400230144012302640123105401A0
:10F548002326340723240402A30204008144E30C85
:10F558000AF62285EF001074AA8435D54A85EFF0A3
:10F56800CFA295B7397122DC06DE26DA4AD84ED604
:10F5780052D456D25AD05ECE62CC66CA0944630BC6
:10F58800061063090710AA8B3A89368BB28A2E8C2B
:10F59800EFE0BFBE2A8A5144630E050E930530057D
:10F5A80041459710FB1FE78060A9AA894D447DC19A
:10F5B8008344190083472900A204C207BE948347E5
:10F5C8000900BE9483473900E207BE9483278A0264
:10F5D80063E697007D5709446399E70A63070C00BF
:10F5E80083474A000544898BCDC3930C4B002146C1
:10F5F80081450A85C20C9710FB1FE78000C993DC80
:10F608000C019305300566859710FB1FE78000A362
:10F618002A8C4D443DC95A86D68511059710FB1F83
:10F62800E780A0D11146CA8562859710FB1FE78045
:10F63800C0D0414693058A014E859710FB1FE7808D
:10F64800C0CF21478A866686E2854E85EF20E01D79
:10F658002A841DE521468A8528009710FB1FE7802C
:10F66800C0CD21469305490028009710FB1FE7806D
:10F67800E0C78547631EF502A6855E85EF50FFB794
:10F6880062859710FB1FE780A0A94E859710FB1F86
:10F69800E78000A92285F2506254D2544259B259E7
:10F6A800225A925A025BF24B624CD24C2161828000
:10F6B8000544F9B779719397050122D406D626D265
:10F6C8004AD04ECEC1872E8463D50704B7240020C4
:10F6D800938484CF03C53400EF208FE02AC611CD70
:10F6E800EFF03F91B24519E503C524009307F00FE9
:10F6F800631EF5002E85EF208FD22165218DB25033
:10F70800225492540259F24945618280EF204FE514
:10F71800EDB793F7150091C7EFF04F981345140014
:10F72800F9BFA1E10145E1BF850493F4F40FEFE0CF
:10F73800BFBEE3F9A4FE33959900131905011359C7
:10F748000901B3772401EDD34A85EFE01FE7C167CC
:10F75800FD176305F500DD45EFF00F8B33452401F8
:10F7680079BF85448549E1B7B727002023A407CE90
:10F77800B727002023AC07CC37070500B7270020A0
:10F78800130707DB23AA07CCB727002023A6E7CE59
:10F79800370705009387C7CE1307C7ABD8C337E72A
:10F7A80004001307276F98C737170500B7270020ED
:10F7B8001307A7D423AEE7CC371705009387C7CD27
:10F7C8001307278BD8C337170500130767B998C7DE
:10F7D8008280B727002083C7C7CFA18B89C7B727E7
:10F7E80000209387C7CE37270020232CF7CC01456C
:10F7F8008280B727002083C7C7CF918B89C7B727D7
:10F8080000209387C7CD37270020232AF7CC01454E
:10F818008280011106CE2AC6EFF01FF53245B727C0
:10F8280000209945A38DA7CEEFD04FA0F24037F521
:10F8380004001305058705616FE0BFAE1C5581C73D
:10F84800A1473E858280011122CC26CA2A84AE8433
:10F85800130500049305300506CE9700FB1FE780CB
:10F86800E07D08D46305051013060004A6859710EB
:10F87800FB1FE780609A78548347270193F6870037
:10F88800638E0610145483C62600A18A6388061066
:10F8980083270408E9EF9305300513050010970046
:10F8A800FB1FE780A0792320A4088D4771C1A3021C
:10F8B8000400785483C714008346170081EF81EE53
:10F8C80083C72400918BDDEB83472701918BDDE70C
:10F8D800854711A889C62147A302E40099C7834731
:10F8E800540093E70701A302F4006C5483C7250171
:10F8F800858B91CF1C54054783C727008D8B639850
:10F90800E7008347640093E717002303F400832785
:10F91800040899C78347640093E787002303F4002A
:10F928008347540005476398E70C930484004146D5
:10F93800814526859710FB1FE78020954146814524
:10F94800130584019710FB1FE78020941306C40356
:10F958003285C14532C6EF40BF9A83270408324634
:10F96800BDC72285EF00903F9307000525CDA1472D
:10F97800F2406244D2443E850561828083C7040018
:10F98800834607001547B387E70237C70600130702
:10F99800C76CBA97B69783C70700B1B783C6140078
:10F9A80091C68346170099C2E14735BF83C6240034
:10F9B800D58F918B91DF83C70400834607001547D5
:10F9C800B387E70237C706001307076BD9B7228545
:10F9D8009306C402A685EFF0CF972285EF009031F9
:10F9E80059F5C14703550400A301F4008145EF50C0
:10F9F8002FEB8147B5BF13F7870149C3C18B930428
:10FA080084004146A9CB890526859710FB1FE7800E
:10FA1800A08041468145130584019710FB1FE780AC
:10FA2800C086834764001306C403328593E7470002
:10FA38002303F400C14532C6EF409F8C8327040896
:10FA480032468DC32285EF0070319307200505F1FA
:10FA5800A301F40079BF814526859710FB1FE78035
:10FA6800C08245BF9306C402A6852285EFF06F8E3B
:10FA78002285EF003028CD4761DDD5BD0947854592
:10FA88006388E70093F7D70F11476397E700894525
:10FA980003550400EF50CFE08347640093E7470025
:10FAA8002303F4008327040881C7930710054DB783
:10FAB800C54779BF8347250063830726797122D418
:10FAC80006D626D24AD083473500130750052A8424
:10FAD800639FE706034975001306C503C14593579D
:10FAE8003900AA97328583C4870032C6EF405F8108
:10FAF800B727002083A7C7EDA9C79C47B9C303252B
:10FB0800040893767900B3D6D4403246858A9305A3
:10FB18000504180893E60608130505088297137567
:10FB2800F50F05E141460C081305C4029700FB1FB9
:10FB3800E780806E2285EF00F01B93076005A30124
:10FB4800F400B2502254925402594561828013073E
:10FB580010026395E7021C550327050883D7470061
:10FB680069EB13F7071071C77855035747011377E7
:10FB7800071061C393077002A301F40083473400A0
:10FB880013077002639FE70C3C5885E39305300523
:10FB980071459700FB1FE780604A28D819C5714650
:10FBA80081459700FB1FE780406E2458B9C883C77A
:10FBB800A40191E72285EFF00F85238DA400285832
:10FBC800814541469700FB1FE780206C28583D4738
:10FBD8008345A5019387F5FF93F7F70F6364F70053
:10FBE800EF400FF2EF20EFB13C58A1452398A70052
:10FBF80013852701EF40CFF02C5803550400EF0080
:10FC0800D0409307800203550400A301F400EFE0FD
:10FC1800CFD6414611C58357E50013D617003E9647
:10FC2800B727002003C5B7CF06068545EF20CFECE0
:10FC380009BF13F7072011CB7854035747011377EF
:10FC4800072001C79307900205BF93F707409DD788
:10FC58007C5483D7470193F707408DD39307B002AD
:10FC680021BF13078002639BE7023C5889CB83D5E9
:10FC780007010355040013862701EF00903E1C542A
:10FC880083D7470013F707202DC37854035747013C
:10FC98001377072039CB93079002B5B71307900263
:10FCA800639CE700EF405F96AA8503550400EF00C8
:10FCB800503A9307A00281BF1307A0026393E70499
:10FCC800EF40FF93AA85854701456384F500814588
:10FCD80005452EC6EF40BF902A86B245035504005D
:10FCE800EF00B0331C5483D7470093F707408DC704
:10FCF8007C5483D7470193F7074099CF9307B00205
:10FD080019B71307B0026399E700EF409F90AA85DF
:10FD180003550400EF0070389307F0020DB5828098
:10FD2800411122C4405926C206C67C54AA8483D7EE
:10FD3800470113F7071019C71854035747001377DB
:10FD480007101DE313F7072019C718540357470076
:10FD58001377072011EB93F707408DCF1C5483D7F7
:10FD6800470093F707409DC793071002A301F400CB
:10FD78002285EFF03FD4034734009307F002631065
:10FD8800F702224403D52400B24092448145410140
:10FD98006FE09FA79307F002A301F400DDB7B2401C
:10FDA8002244924441018280397122DC405926DA8A
:10FDB8004AD84ED606DEAA89AE843289630F043C3F
:10FDC80003552500835704006384A700A14429A094
:10FDD8008347240091EB9D44F25062542685425992
:10FDE800D254B259216182809387E5FF93F7F70FC8
:10FDF8002D47E362F7FE37C706008A071307876EA9
:10FE0800BA979C438287B2852285EFF03FA3AA84E4
:10FE1800E1B74146CA851305C4049700FB1FE78074
:10FE2800A03F22851127AA8411C1A1448347340029
:10FE3800130740056397E70093079005A301F400B3
:10FE480061BF130760056395E7009307A005FDB739
:10FE5800D147EDB79309C4054E854146CA85970039
:10FE6800FB1FE780603B0325040855C9834734001E
:10FE7800130790056399E700228591279307E0050A
:10FE8800A301F40059A81307A0056394E708834762
:10FE9800740013D737002297834687009D8BB3D60B
:10FEA800F640B727002083A7C7ED858A93E606F8B2
:10FEB80093F6F60F81DF9C4791DB93050508180838
:10FEC8004E861305050482979374F50FE39004F0AA
:10FED80041460C081305C4049700FB1FE780004146
:10FEE800834774004D47850793F7F70FA303F40082
:10FEF8006377F7002285E1259307E00581B7B727E7
:10FF0800002003C5B7CF8545EF202FA093075005E4
:10FF180035B71307C005E381E7F6814475BD1309BA
:10FF280084004E86CA8522851408EFE09FC24146A8
:10FF38009305C40408089700FB1FE780203BE30DE6
:10FF480005E88A861306C403CE854A85EF10900417
:10FF58000DE12285EFE03FCBB72700202A8783A752
:10FF680047CF03550400814601468A858297AA84B3
:10FF780011C1A14493072002D1B583450600EFE0E3
:10FF8800BF8861BF0347340093072002E315F7E4F5
:10FF98007C5889EB9305300571459700FB1FE78076
:10FFA800E00968D86858E30805E24146CA85970021
:10FFB800FB1FE780602664582285EFE0DFC4238DAD
:10FFC800A400930730026DBD034734009307300245
:10FFD800E313F7E083570600685821469305290084
:10FFE8002318F50049059700FB1FE780E0227C54A1
:08FFF80083D7470113F727002E
:020000025000AC
:1000000035CB185403574700098B2DC7930740027F
:10001000A5BD0347340093074002E312F7DC3C5CC4
:1000200081EB85455D459700FB1FE780A00128DC3B
:10003000285CE30805EE834709004146CA85230B87
:10004000F5009700FB1FE780A01D930750022DBD10
:100050000347340093075002E313F7D8285C19468E
:100060009305190041059700FB1FE780601B7C5436
:1000700083D74701918B9DCF1C5483D74700918B29
:1000800095CB9307600209B57C5C89EB930530053D
:1000900051459700FB1FE780E0FA68DC685CE30BE2
:1000A00005D24146CA859700FB1FE78060177C5C3C
:1000B0007D5798CB4E85EFF03FC7A5B503250408C3
:1000C00013060004CA85130505049700FB1FE7808B
:1000D00020152285EFE0BFA48347340013070005F5
:1000E0006395E7009307400545B313071005639C2C
:1000F000E700B727002003C5B7CF8545EF206F8104
:100100009307500551B313072005E39CE7E0B72799
:10011000002083A7C7EDE38F07CA9C47E38C07CA7B
:1001200083250408930484001808938505088146F4
:1001300026862E858297035504001008A685EF4079
:100140009FFF9307B00589B3034734009307E00589
:10015000E317F7C88325040841464A859700FB1F2B
:10016000E7804019AD44E30D05C603250408414668
:10017000CA859700FB1FE780A00A2285EFE03FA910
:10018000B72700202A8783A747CF2C5803550400A0
:10019000814601468297AA8411C1A14493071002A7
:1001A00055B1AD47E39FF5D683460600835525003C
:1001B0001306650003450500EF402FFC9DB38947FA
:1001C00061C2DDCD2300A60083C70500A300F600B1
:1001D00083C715002301F60083C72500A301F6009D
:1001E00083C73500A30206002302F60083D745002B
:1001F000A183858BA302F60003D745001377072060
:1002000009C793E72700A302F60083D7450093F7B9
:10021000074099C78347560093E74700A302F600BB
:1002200083D745001397470163580700834756005B
:1002300093E78700A302F6002303060083C7450067
:10024000858B2303F60003D74500098B09C793E785
:1002500027002303F60083D74500918B99C7834776
:10026000660093E747002303F60003D74500814764
:10027000218B19C703476600136787002303E60035
:100280003E8582802E86AA8505456FF05FF32E8617
:10029000AA8509456FF0BFF289478DC505C5411193
:1002A00006C6AE870D47AA852380E7001385170091
:1002B00041469700FB1FE780A0F6B24081473E858C
:1002C000410182803E85828089478DC505C54111E7
:1002D00006C6AE871147AA852380E700138517005D
:1002E00041469700FB1FE780A0F3B24081473E855F
:1002F000410182803E85828089478DC505C54111B7
:1003000006C6AE871947AA852380E7001385170024
:1003100041469700FB1FE780A0F0B24081473E8531
:10032000410182803E85828089479DCD15CD411156
:1003300006C61D472380E50003570500AE8721460A
:10034000A380E5000357050021832381E500930581
:100350002500138537009700FB1FE78060ECB24053
:1003600081473E85410182803E85828089478DC5D7
:1003700005C5411106C6AE872147AA852380E7003F
:100380001385170041469700FB1FE78060E9B240E4
:1003900081473E85410182803E858280894795C99B
:1003A0000DC9411106C625472380E5000347050016
:1003B000AE871946A380E500930515001385270035
:1003C0009700FB1FE780C0E5B24081473E854101B1
:1003D00082803E85828089478DC505C5411106C64C
:1003E000AE872947AA852380E70013851700414679
:1003F0009700FB1FE780C0E2B24081473E85410184
:1004000082803E858280894795C50DC5411106C60B
:10041000AE873147AA852380E700138517001306AE
:1004200000049700FB1FE780A0DFB24081473E85B4
:10043000410182803E85828089478DC505C5411175
:1004400006C6AE873547AA852380E70013851700C7
:1004500041469700FB1FE780A0DCB24081473E8504
:10046000410182803E858280894791C909C99547AB
:100470002380F50083470500A380F50081473E8572
:100480008280894791C909C9AD472380F500834718
:100490000500A380F50081473E85828015C55D710A
:1004A0008A8586C6A2C42A84EFE02FE203550400A1
:1004B000B70605000A86938646289D45EFE0CFD310
:1004C000B6402644616182800545828015C55D7114
:1004D0008A8586C6A2C42A84EFE02FDF0355040074
:1004E000B70605000A869386E6289D45EFE0CFD043
:1004F000B640264461618280054582805D71A2C458
:100500009305C5022A8441460A8586C69700FB1FCB
:10051000E78000D103550400B70605000A869386DC
:100520008629C545EFE04FCDB64026446161828003
:100530005D71A2C49305C5032A8441460A8586C617
:100540009700FB1FE780C0CD03550400B7060500E8
:100550000A869386862CC545EFE00FCAB64026442E
:1005600061618280B727002083A7C7EDB1CB9C4390
:100570005D71A2C486C62A841305E00F95CF0325BA
:1005800004089305050C13050508829783250408C4
:10059000130600040A85938505089700FB1FE78072
:1005A00020C803550400B7060500938666400A86F6
:1005B00093051004EFE04FC4B64026446161828089
:1005C0001305E00F8280317122DD2A840355050076
:1005D00026DB06DF4AD94ED752D556D35AD15ECF45
:1005E00062CDEFD01FBA3C58AA8489EB9305300541
:1005F00071459700FB1FE780E0A428D82858CD4715
:100600000DC9714681459700FB1FE78080C803290B
:1006100004072285EFE0AFDF230DA9008347240004
:1006200037290020638A07128327C9ED85E39307E2
:10063000E00FFA506A54DA544A59BA592A5A9A5A67
:100640000A5BFA4B6A4C3E852961828083AB0701C5
:10065000E38F0BFC032B0408EF30FFFA2A8C0145D3
:10066000EF307FF883C754003858130B0B029309FF
:10067000C403130AC405938A64003AC0B337F00078
:100680002A87930801045688B33680015286CE85A6
:100690005A85829B1C5403C727002307E10203C726
:1006A0001700A306E10283C707002306F102832790
:1006B000C9EDB5DF03AB4701E30B0BF683C754006D
:1006C000B337F0003ECEEF301FF4AA8B0145EF3078
:1006D0009FF103270408F2472AC03AC2B3387001D9
:1006E00056887810930684004E86D2858800029B37
:1006F0007C5403C727012305E10203C71700A304A5
:10070000E10283C707002304F1028327C9ED03A98F
:100710004701EF305FEF2A8B0145EF30DFEC83C8F4
:1007200054009C082A883EC2B3381001B3376001D8
:100730003810930684015286CE8556C088000299EF
:1007400003550400B7060500938686439008C54507
:10075000EFE08FAAAA87F1BD83C654008327C9EDB5
:10076000032B0408B336D00083AB070136CEEF303D
:100770009FE92A8C0145EF301FE73C58F246130BE6
:100780000B02130AC4059309C403938A64002A88E0
:10079000930801044E86D2853EC05687B337800148
:1007A0005A85829B1C54130B010303C727002307A0
:1007B000E10203C71700A306E10283C7070023066F
:1007C000F1028327C9ED83AB470183C75400B337D8
:1007D000F0003ECEEF303FE32A8C0145EF30BFE022
:1007E000F2472AC0B33880015688781093068400F7
:1007F0004E86D2855AC28800829B832504084146D2
:100800005A859700FB1FE780E0AEAD47E31205EE87
:100810000DB5B70605002E869386862FC5456FE079
:10082000AF9D5D71B287A2C42300B1002A84BE854A
:1008300013051100194686C69700FB1FE780409EEE
:10084000B70605000A8622859386C639A145EFE0E2
:10085000AF9AB640264461618280B70605002E86B5
:100860009386C636C5456FE02F995D71B287A2C4E5
:100870002310B1002A84BE8513052100214686C6B7
:100880009700FB1FE780C099B70605000A862285FE
:1008900093868632AD45EFE02F96B64026446161DF
:1008A0008280B70605002E869386663DC5456FE0BB
:1008B000AF94797122D406D626D283473500130728
:1008C00030052A846384E708130750056396E70818
:1008D0009307A005A301F50083477500C14513D711
:1008E00037002A97834687009D8B1305C503B3D62F
:1008F000F640858A93E606F893F6F60F36C6EF3093
:10090000BFA0B246B727002083A7C7ED9DCB9C4769
:100910008DCB0325040818081306C40393050504AA
:100920001305050882971375F50F01ED1305C40231
:1009300041460C089700FB1FE780808E2285EFF070
:10094000FFBBB250225492544561828093079005B8
:10095000A301F50081467DB7130710026396E702F5
:100960007C550327050883D747016316070E13F745
:1009700017006302070E185503574700058B61CF18
:1009800093072002A301F4008347340013072002D9
:10099000639DE70E3C5889EB93053005714597F050
:1009A000FA1FE780206A28D82458C9C02285EFE0C2
:1009B0000FA6238DA4002858814541469700FB1FB0
:1009C000E780208D28583D478345A5019387F5FF93
:1009D00093F7F70F636DF702B727002083C777EE11
:1009E000D5C34146814508089700FB1FE780608A10
:1009F000B72500201946938505BB08089700FB1F03
:100A0000E780008230580C082E85EF00917EEF10B1
:100A1000CFCF3C58A1452398A70013852701EF307D
:100A2000BF8E2C5803550400EFF0BFDE9307300251
:100A300003550400A301F400EFD0AFF4414619C1FF
:100A40000356E500B727002003C5B7CF0606854546
:100A5000EF101F8BFDB513F7270009CB1854035770
:100A60004700098B01C79307400229BF918BE38D93
:100A700007F01C5483D74700918BE38707F0930757
:100A8000600209B7EF305F8859B713073002639AE5
:100A9000E7023C5889CB83D5070103550400138630
:100AA0002701EFF09FDC7C5483D7470113F7270021
:100AB00021CF185403574700098B39C793074002C9
:100AC00085BF13074002639CE700EF307FB4AA851F
:100AD00003550400EFF07FD89307500291BF13072E
:100AE00050026390E704EF301FB20DE981450545E0
:100AF0002EC6EF305FAF2A86B24503550400EFF0F3
:100B00005FD27C5483D74701918B9DC71C5483D7F8
:100B10004700918B95C39307600219BF8545014536
:100B2000C1BF130760026399E700EF301FAFAA85CA
:100B300003550400EFF0FFD67C540327040883D745
:100B4000470119EF13F7071001CF18540357470057
:100B50001377071011C793077002A301F400D5B3F0
:100B600013F7072011CB18540357470013770720BA
:100B700001C793079002D5B793F7074091CB1C5458
:100B800083D7470093F7074081C79307B002F1B7B7
:100B90009307F002D9B7397122DC26DA4ED652D447
:100BA00006DE4AD8AE89328AAA84EFD08FDD40595A
:100BB000414681450A8597F0FA1FE780806D25C878
:100BC0000359040063159906034734009307100284
:100BD000631FF7028327040899CF2C58A9C94A85B7
:100BE000EF1050490545F2506254D2544259B2595F
:100BF000225A216182808A861306C4059305C403A4
:100C000013058400EF0090391DE18A85C9BF2C5877
:100C100099CD83D70501639C47012146C9054E85BF
:100C200097F0FA1FE780006D19C12C584DBF26853B
:100C3000EFD02FD52A8405455DD44C54A1C983D764
:100C40000501639547052146C9054E8597F0FA1FB2
:100C5000E780406A8547631BF502B727002083C7FA
:100C6000B79891C74C5483C7B501639BA70CBD458A
:100C70002685EF10703AB727002083A747B60145B5
:100C8000BDD31D45894582970145B1BFB7270020D7
:100C900003C787EEB7290020938949B3058B3E89A6
:100CA00031C3B72700200347540083C707EE631BF7
:100CB000F702B72500201946938515EE1305640049
:100CC00097F0FA1FE78000638547631DF50083A74F
:100CD000090381C791451D458297BD452685EF10C3
:100CE000B03309B737270020034777EE83A70903FE
:100CF00031CB034789EE098B09CB81C795451D454B
:100D000082972685EF105037F1BD81C78D451D456F
:100D1000829741468145080897F0FA1FE78060579F
:100D2000B72500201946938505BB080897F0FA1FE0
:100D3000E780004F0C082E850A86EF00914B8A85CC
:100D4000268579BD8545C5FF6DBF797122D440598F
:100D50004AD04ECE52CC06D626D2AA892E8A3289C5
:100D6000630D046A0355250083570400638CA700B4
:100D7000A144B2502254268502599254F249624A43
:100D8000456182808344240099C09D44DDB79387E8
:100D9000F5FF93F7F70F3147E369F7FE37C7060012
:100DA0008A0713078771BA979C4382871C54E9F31B
:100DB000930530051305000497F0FA1FE78080289B
:100DC00008D45DD503470900914763F4E7008D44DB
:100DD0004DB7034719008547E3EBE7FE1306000410
:100DE000CA8597F0FA1FE780A0430C547054A30201
:100DF0000400D4415C4A858AFD8E83574601F99BE5
:100E0000D58F231AF600D841544AF59B0583058BEC
:100E10008582F98E8606DD8E231AD600DC41584A7B
:100E2000ED9A8983858B09837D8F0A07558F231A55
:100E3000E600D4415C4A5D9B8D82858A8D83F58F67
:100E40008E07D98F231AF600D841544A93F7F7EF4B
:100E50002183058BA182F98EA206DD8E231AD6008E
:100E6000DC41584AA583858B25837D8F9317970096
:100E700013F7F6DF5D8F231AE600D4415C4AA9829E
:100E8000858AA983F58F9396A7009377F7BFD58FAF
:100E9000231AF600D441584AAD82858A2D83758F76
:100EA000FD769386F67F2E07F58FD98F231AF600ED
:100EB0008347260103250408A18B6387071083C796
:100EC0002500A18B63820710E31405EA9305300522
:100ED0001305001097F0FA1FE780C0162320A4081E
:100EE000E30705EE7C54A30204000347190083C600
:100EF000170089EA45C38347540093E70701A3021B
:100F0000F40029A0A147A302F40075F72285EFF0B1
:100F1000EFDB6C5483C72501858B81CF1C5483C7BD
:100F200027008D8B99C78347640093E7170023033D
:100F3000F4008327040899C78347640093E7870078
:100F40002303F4008347540005476393E70C4146AD
:100F500081451305840097F0FA1FE78080334146EE
:100F600081451305840197F0FA1FE7808032C1455F
:100F70001305C403EF304FB9032704089307000596
:100F800011E3C14703550400A301F4008145EF407C
:100F9000AF91C5B303C72701118B19E70347290098
:100FA000118B19E38547A1BF83C707001547834607
:100FB0000900B387E70237C706001307C76CBA9763
:100FC000B69783C7070025BF19C597F0FA1FE780BA
:100FD000A015232004087C5403C7170011C703473A
:100FE000190019C3E14721BF03C72701118B09E786
:100FF00003472900118B5DD783C707001547834638
:101000000900B387E70237C706001307076B45BF20
:1010100013F7870131CFC18B130584004146A9C363
:10102000890597F0FA1FE780A01F41468145130507
:10103000840197F0FA1FE780C02583476400C1450B
:101040001305C40393E747002303F400EF30CFAB4D
:101050008327040881CF93072005A301F40011BB67
:10106000814597F0FA1FE780C022C1B7CD47F5B799
:10107000094789456386E70011476398E70085457E
:1010800003550400EF404F8221A01947E389E7FE92
:101090008347640093E747002303F4008327040891
:1010A00081C79307100555BFC54745BF4146CA854F
:1010B0001305C40497F0FA1FE780801683473400B5
:1010C00013076005639CE700B727002003C5B7CF6F
:1010D0008545EF100F849307500541B7454763835B
:1010E000E7029306C4021306C40393058400228515
:1010F000EFD0BFA62285EFF06FC0AA8411C1A14432
:10110000D147A1BFC94791BF9309C4054E85414648
:10111000CA8597F0FA1FE780A0100325040861CD67
:1011200083473400130790056398E7002285EFF0AA
:101130002FC09307E00515B71307A005639EE706C8
:10114000B727002083A7C7EDE38107C403A8870062
:10115000E30D08C283477400930505084E8613D734
:1011600037002297834687009D8B0A87B3D6F640C7
:10117000858A93E6060813050504029841468A8588
:101180001305C40497F0FA1FE780C01611E1D2845A
:101190002285EFF0EFB983477400CD461307E005D1
:1011A000850793F7F70FA303F40063E4F600130732
:1011B0006005A301E40075BE1307C005E39BE7BA11
:1011C000B727002083A7C7EDE38107BC9C47E38EC8
:1011D00007BA93050508130984000A8781464A86E1
:1011E0002E858297035504000A86CA85EF30BFF426
:1011F0009307B0059DB58A864E86930584002285A7
:10120000EFD0BF9541469305C4040A8597F0FA1FB5
:10121000E780400E8547D284E31DF5B42285EFF0C8
:101220002FB1AA84E31605B4930710023DB5034716
:10123000340093077002E31AF7B47C5889EB9305E6
:101240003005714597F0FA1FE780C0DF68D868580D
:10125000E30D05B2CA85414697F0FA1FE78040FCCE
:10126000032944072285EFD09F9A230DA9009307F5
:101270008002E5B30347340093078002E317F7B019
:101280008357060068582146930529002318F50066
:10129000490597F0FA1FE780A0F87C5483D74701EF
:1012A00013F7072025CF185403574700137707205B
:1012B00035C79307900255B3034734009307900254
:1012C000E315F7AC3C5C89EB930530055D4597F081
:1012D000FA1FE78020D728DC285CE30805AA4146EE
:1012E000CA8597F0FA1FE780A0F39307A002B5B371
:1012F000034734009307A002E319F7A883470600C9
:10130000285C194693051900230BF500410597F059
:10131000FA1FE780E0F07C5483D7470193F707403A
:10132000B1C71C5483D7470093F70740A1C3930765
:10133000B00225B3034734009307B002E317F7A4C4
:101340007C5C89EB93053005514597F0FA1FE780E7
:1013500060CF68DC685CE30D05A04146CA8597F064
:10136000FA1FE780E0EB7C5C7D5798CB03D5290022
:101370008145EFD0EFC9F5BA034734009307F00475
:10138000E3F8E79E03250408E304059E1306000422
:10139000CA851305050497F0FA1FE78060E82285E7
:1013A000EFF04F9CAA842285EFD06FF7834734007B
:1013B00013070005639FE700B727002003D6E90065
:1013C00003C5B7CF85450606EF009FF393073005A9
:1013D00069B1130710056395E70093076005B5B978
:1013E00013072005E397E7989307C005BDB10347AE
:1013F00034009307E005E31DF796032504084146F2
:10140000CA8597F0FA1FE780A0E12285EFF0AF9B35
:10141000AA8419BD83450600A9BF85478144E39A84
:10142000F594032846008347360003472600834689
:10143000160083552500034606000145EF308FCA8C
:101440000DBA8147C1463307F500B388F50003475D
:10145000070083C808003308F600850733471701E3
:101460002300E800E391D7FE82800147BD471308BF
:10147000F00F3306F50083460600B388F500FD172C
:101480008606558F2380E8000347060093F7F70F81
:101490001D83E39007FF82808147930800F841484D
:1014A00093F6F70F3387F50063FCC600B306F5002B
:1014B00083C606002300D7008507E39307FF8280D9
:1014C0006395C60023001701C5BF23000700EDB7D1
:1014D00001114AC856C22E89AA8A93053005414592
:1014E00006CE22CC26CA4EC652C4328A97F0FA1FC4
:1014F000E78040B5AA8493053005414597F0FA1F6F
:10150000E78040B42A84CD49A5C431CD4146814508
:1015100097F0FA1FE780E0D72686A2855685EF0070
:10152000414DAA8929E18387040063D30706A28578
:101530002685EFF09FF3B7C506004A869385C574EC
:101540002285EFF01FF08307090063D80704A28506
:101550004A85EFF09FF1B7C5060052869385C574A2
:101560002285EFF01FEE268597F0FA1FE780C0BBBB
:1015700011C4228597F0FA1FE78000BBF240624455
:101580004E85D2444249B249224A924A056182803C
:10159000CA852685EFF07FED7DB7D2854A85EFF0CD
:1015A000DFECD1B781474146B306F5003387F5003C
:1015B0000347070003C80600850733470701238058
:1015C000E600E393C7FE8280011126CA4EC6AE84B0
:1015D000AA8993053005130500034AC806CE22CC1C
:1015E000328997F0FA1FE780E0A52DC513060003A6
:1015F00081452A8497F0FA1FE780A0C94146CE852D
:10160000228597F0FA1FE780C0D3A6850D46130503
:10161000D40197F0FA1FE780C0D2130604029305A5
:1016200004012285EF00E13CAA840D469305D40213
:101630004A8597F0FA1FE780C0D0228597F0FA1FFD
:10164000E78080AEF240624426854249D244B249E6
:1016500005618280CD44FDB75D714EDE62D4AE89F6
:101660002A8C9305300513050003A6C2CAC052DCBC
:1016700056DA5AD85ED686C6A2C4B28B368BBA84E6
:10168000BE8A4289468A97F0FA1FE780A09B6305CD
:1016900005101306000381452A8497F0FA1FE7809E
:1016A00040BF4146E285228597F0FA1FE78060C976
:1016B000414681450A8597F0FA1FE78080BD1D46A7
:1016C000DE850A8597F0FA1FE780A0C71D46DA85F8
:1016D0001305710097F0FA1FE780A0C63339200187
:1016E000B334900041468145080823072101A30730
:1016F000910097F0FA1FE780C0B91946D6854808CF
:1017000097F0FA1FE780E0C31946D2851305A101BF
:1017100097F0FA1FE780E0C2930404014146CE85AA
:10172000268597F0FA1FE780C0C18A852685EFF0ED
:101730007FE7930904024E86A6852285EF00612B80
:101740002A890DE94146CE85268597F0FA1FE78064
:1017500020AD0C082685EFF0FFE44E86A685228595
:10176000EF0021292A8946454146CE8597F0FA1F88
:10177000E78020BD228597F0FA1FE780E09AB64007
:1017800026444A8596440649F259625AD25A425B27
:10179000B25B225C616182804D49D5B7011126CAD6
:1017A00052C4AA842E8A13050003930530054AC843
:1017B0004EC606CE22CC3289B68997F0FA1FE78052
:1017C000608835C52A84A685414697F0FA1FE780D0
:1017D00040B7930404012146D285268597F0FA1F6D
:1017E000E78020B6CA8521461305840197F0FA1FC9
:1017F000E78020B513090402A6854A862285EF00FA
:10180000411FAA844146CA854E8597F0FA1FE7809A
:1018100040B3228597F0FA1FE7800091F2406244BE
:1018200026854249D244B249224A05618280CD448C
:10183000F5B739715AD05ECE2A8BAE8B41459305F0
:10184000300506DE26DA52D456D262CC66CA6AC8A1
:10185000368C328DBA8C22DC4AD84ED697E0FA1FED
:10186000E780407EAA8A93053005414597E0FA1F3C
:10187000E780407D2A8ACD44638E0A0859C52A86AE
:10188000D6855A85EFF0DFC4AA8441E1930530057F
:10189000414597E0FA1FE780E07A2A8993053005F1
:1018A000414597E0FA1FE780E079AA89630A090EAB
:1018B0006306050E1304FD0011841376FD0049C074
:1018C0007D144204418035EE131544004E86D685C2
:1018D0005E95EFF01FB7414681454A8597F0FA1FA4
:1018E000E780209B014D93170D01C18363F48708A6
:1018F000BDC04A8597F0FA1FE7800083638709001F
:101900004E8597F0FA1FE7802082568597F0FA1FE0
:10191000E780808163070A00528597F0FA1FE7800D
:10192000A080F250625426854259D254B259225AAC
:10193000925A025BF24B624CD24C424D2161828042
:101940000144131544008A855E95EFF0FFB44E867E
:10195000D2850A85BDBF93154D000A86DE954A855E
:10196000EFF03FAE4A868A855A85EF008108AA8447
:10197000050D95BFBDFC0A86CE854A85EFF07FAC8C
:101980004A868A855A85EF00C106AA846686CA857A
:10199000628597F0FA1FE780A088A1BFCD4491BF70
:1019A000CD44A9BF397162CC2A8C594526DA4AD870
:1019B0004ED652D456D25AD05ECE06DE22DCAE8B44
:1019C000328BB68A3AC63E8AC2894689834401046C
:1019D000EF008FAA49C19167938717E92310F5009B
:1019E00085472301F5002A8432472105630C0C0446
:1019F00093071003A301F4001946814597F0FA1FDD
:101A0000E780208923036401A3035401230A94007F
:101A100023127401231744012318340123192401CC
:101A2000A285B72700206254F250D2544259B259CD
:101A3000225A925A025BF24B624C03C587CF216156
:101A40006F008FB2A30104001946BA8597E0FA1F10
:101A5000E780007D45BFF2506254D2544259B259DA
:101A6000225A925A025BF24B624C21618280797158
:101A700056CAAA8A1305100326D24AD04ECE52CC9B
:101A800006D622D42EC6328AB684BA893E89EF00A1
:101A9000AF9E2DC1B245374602019307850013065C
:101AA00016E92A845CC110C123045501A304B500C2
:101AB0001946D285290597E0FA1FE7806076CE8522
:101AC0002308940013051401268697E0FA1FE78087
:101AD000207523082403A285B72700202254B25082
:101AE00092540259F249624AD24A03C587CF4561EE
:101AF0006F008FA7B250225492540259F249624AA1
:101B0000D24A45618280011122CC2A84314506CE19
:101B10002EC632C436C23AC0EF000F9629C1916773
:101B2000938717E92310F500B245224692460247F3
:101B30008D472301F500A30185006244B7270020EB
:101B40002312B5002313C5002314D5002315E50087
:101B5000F240AA8503C587CF05616F00EFA0F24070
:101B600062440561828001114AC82A89394526CA22
:101B700006CE22CC2EC6B284EF000F9031C1B24502
:101B80009167938727E92310F50091472301F5001A
:101B9000A30125012312B5002A84A6851905214633
:101BA00097E0FA1FE780C067A285B727002062444C
:101BB000F240D244424903C587CF05616F00CF9AF6
:101BC000F2406244D24442490561828001114AC810
:101BD0002A89414526CA06CE22CC2EC6B284EF0001
:101BE000AF8929C19167B245938727E92310F50092
:101BF00095472A842301F500231225012146190562
